:020000040800F2
:100000000000032081550008B1340008BD34000809
:10001000C5340008CD340008D534000800000000C5
:10002000000000000000000000000000E553000890
:10003000DD34000800000000C9540008195500080C
:10004000CD550008CD550008CD550008CD55000808
:10005000CD550008CD550008E9340008CD550008FD
:10006000CD550008CD550008CD550008CD550008E8
:10007000CD550008CD550008CD550008CD550008D8
:10008000CD550008CD550008CD550008CD550008C8
:10009000CD550008CD550008CD550008CD550008B8
:1000A000CD550008CD550008CD550008CD550008A8
:1000B00001350008CD550008CD550008CD55000884
:1000C000CD550008CD550008CD550008CD55000888
:1000D000CD550008CD550008CD550008CD55000878
:1000E000CD550008951E0008CD550008CD550008D7
:1000F000CD550008CD550008CD550008CD55000858
:10010000CD550008CD55000819350008CD5500081B
:10011000CD550008CD550008CD550008CD55000837
:10012000CD5500087D350008CD550008CD55000897
:10013000CD550008CD550008CD550008CD55000817
:10014000CD550008CD550008CD550008CD55000807
:10015000CD550008CD550008CD550008CD550008F7
:10016000CD550008CD550008CD550008CD550008E7
:10017000CD5500080D350008CD550008CD550008B7
:10018000CD550008CD550008CD550008CD550008C7
:10019000CD550008CD550008CD550008CD550008B7
:0C01A00089350008CD5500089535000891
:1001B00081F0004102E000BF83F0004330B54FEA18
:1001C00041044FEA430594EA050F08BF90EA020F85
:1001D0001FBF54EA000C55EA020C7FEA645C7FEA18
:1001E000655C00F0E2804FEA5454D4EB5555B8BF3B
:1001F0006D420CDD2C4480EA020281EA030382EAAC
:10020000000083EA010180EA020281EA0303362D3D
:1002100088BF30BD11F0004F4FEA01314FF4801C10
:100220004CEA113102D0404261EB410113F0004F22
:100230004FEA03334CEA133302D0524263EB4303D9
:1002400094EA050F00F0A780A4F10104D5F1200E77
:100250000DDB02FA0EFC22FA05F2801841F10001D2
:1002600003FA0EF2801843FA05F359410EE0A5F1A6
:1002700020050EF1200E012A03FA0EFC28BF4CF0D7
:10028000020C43FA05F3C01851EBE37101F000458D
:1002900007D54FF0000EDCF1000C7EEB00006EEB9A
:1002A0000101B1F5801F1BD3B1F5001F0CD3490824
:1002B0005FEA30004FEA3C0C04F101044FEA44527B
:1002C00012F5800F80F09A80BCF1004F08BF5FEA02
:1002D000500C50F1000041EB045141EA050130BDE2
:1002E0005FEA4C0C404141EB010111F4801FA4F185
:1002F0000104E9D191F0000F04BF01460020B1FADA
:1003000081F308BF2033A3F10B03B3F120020CDA11
:100310000C3208DD02F1140CC2F10C0201FA0CF0EF
:1003200021FA02F10CE002F11402D8BFC2F1200C54
:1003300001FA02F120FA0CFCDCBF41EA0C0190400A
:10034000E41AA2BF01EB0451294330BD6FEA040453
:100350001F3C1CDA0C340EDC04F11404C4F120023E
:1003600020FA04F001FA02F340EA030021FA04F350
:1003700045EA030130BDC4F10C04C4F1200220FAA7
:1003800002F001FA04F340EA0300294630BD21FAE5
:1003900004F0294630BD94F0000F83F4801306BFAB
:1003A00081F480110134013D4EE77FEA645C18BF9F
:1003B0007FEA655C29D094EA050F08BF90EA020F36
:1003C00005D054EA000C04BF1946104630BD91EA2E
:1003D000030F1EBF0021002030BD5FEA545C05D131
:1003E0004000494128BF41F0004130BD14F5800470
:1003F0003CBF01F5801130BD01F0004545F0FE41E4
:1004000041F470014FF0000030BD7FEA645C1ABF18
:10041000194610467FEA655C1CBF0B46024650EA4F
:10042000013406BF52EA033591EA030F41F400217B
:1004300030BD00BF90F0000F04BF0021704730B501
:100440004FF4806404F132044FF000054FF00001D6
:1004500050E700BF90F0000F04BF0021704730B597
:100460004FF4806404F1320410F0004548BF40426C
:100470004FF000013EE700BF42004FEAE2014FEAC1
:1004800031014FEA02701FBF12F07F4393F07F4F9C
:1004900081F06051704792F0000F14BF93F07F4FCE
:1004A000704730B54FF4607401F0004521F0004111
:1004B00020E700BF50EA010208BF704730B54FF097
:1004C00000050AE050EA010208BF704730B511F09C
:1004D000004502D5404261EB41014FF4806404F1D4
:1004E00032045FEA915C3FF4DCAE4FF003025FEA56
:1004F000DC0C18BF03325FEADC0C18BF033202EBDE
:10050000DC02C2F1200300FA03FC20FA02F001FA37
:1005100003FE40EA0E0021FA02F11444C1E600BFD6
:1005200070B54FF0FF0C4CF4E06C1CEA11541DBF89
:100530001CEA135594EA0C0F95EA0C0F00F0DEF854
:100540002C4481EA030621EA4C5123EA4C5350EA39
:10055000013518BF52EA033541F4801143F480138A
:1005600038D0A0FB02CE4FF00005E1FB02E506F01B
:100570000042E0FB03E54FF00006E1FB03569CF070
:10058000000F18BF4EF0010EA4F1FF04B6F5007F76
:1005900064F5407404D25FEA4E0E6D4146EB0606E8
:1005A00042EAC62141EA55514FEAC52040EA5E5071
:1005B0004FEACE2EB4F1FD0C88BFBCF5E06F1ED81B
:1005C000BEF1004F08BF5FEA500E50F1000041EB52
:1005D000045170BD06F0004646EA010140EA0200FF
:1005E00081EA0301B4EB5C04C2BFD4EB0C0541EA21
:1005F000045170BD41F480114FF0000E013C00F336
:10060000AB8014F1360FDEBF002001F0004170BD59
:10061000C4F10004203C35DA0C341BDC04F1140472
:10062000C4F1200500FA05F320FA04F001FA05F2FE
:1006300040EA020001F0004221F0004110EBD370CB
:1006400021FA04F642EB06015EEA430E08BF20EAF7
:10065000D37070BDC4F10C04C4F1200500FA04F39A
:1006600020FA05F001FA04F240EA020001F000412C
:1006700010EBD37041F100015EEA430E08BF20EA9F
:10068000D37070BDC4F1200500FA05F24EEA020EE7
:1006900020FA04F301FA05F243EA020321FA04F016
:1006A00001F0004121FA04F220EA020000EBD370CD
:1006B0005EEA430E08BF20EAD37070BD94F0000FCD
:1006C0000FD101F00046400041EB010111F4801F01
:1006D00008BF013CF7D041EA060195F0000F18BFB2
:1006E000704703F00046520043EB030313F4801FEE
:1006F00008BF013DF7D043EA0603704794EA0C0FA8
:100700000CEA135518BF95EA0C0F0CD050EA4106BD
:1007100018BF52EA4306D1D181EA030101F000413A
:100720004FF0000070BD50EA410606BF1046194662
:1007300052EA430619D094EA0C0F02D150EA01366E
:1007400013D195EA0C0F05D152EA03361CBF1046AF
:1007500019460AD181EA030101F0004141F0FE414E
:1007600041F470014FF0000070BD41F0FE4141F4D2
:10077000780170BD70B54FF0FF0C4CF4E06C1CEAD2
:1007800011541DBF1CEA135594EA0C0F95EA0C0F87
:1007900000F0A7F8A4EB050481EA030E52EA033542
:1007A0004FEA013100F088804FEA03334FF0805563
:1007B00045EA131343EA12634FEA022245EA111590
:1007C00045EA10654FEA00260EF000419D4208BF41
:1007D000964244F1FD0404F5407402D25B084FEAEE
:1007E0003202B61A65EB03055B084FEA32024FF49A
:1007F00080104FF4002CB6EB020E75EB030E22BFF7
:10080000B61A754640EA0C005B084FEA3202B6EBB6
:10081000020E75EB030E22BFB61A754640EA5C0065
:100820005B084FEA3202B6EB020E75EB030E22BFF5
:10083000B61A754640EA9C005B084FEA3202B6EBF6
:10084000020E75EB030E22BFB61A754640EADC00B5
:1008500055EA060E18D04FEA051545EA16754FEA17
:1008600006164FEAC30343EA52734FEAC2025FEA35
:100870001C1CC0D111F4801F0BD141EA00014FF0C4
:1008800000004FF0004CB6E711F4801F04BF014395
:100890000020B4F1FD0C88BFBCF5E06F3FF6AFAEB1
:1008A000B5EB030C04BFB6EB020C5FEA500C50F141
:1008B000000041EB045170BD0EF0004E4EEA1131C4
:1008C00014EB5C04C2BFD4EB0C0541EA045170BDCB
:1008D00041F480114FF0000E013C90E645EA060E0F
:1008E0008DE60CEA135594EA0C0F08BF95EA0C0F3D
:1008F0003FF43BAF94EA0C0F0AD150EA01347FF485
:1009000034AF95EA0C0F7FF425AF104619462CE75B
:1009100095EA0C0F06D152EA03353FF4FDAE1046BE
:10092000194622E750EA410618BF52EA43067FF40F
:10093000C5AE50EA41047FF40DAF52EA43057FF49F
:10094000EBAE12E74FF0FF3C06E000BF4FF0010CAA
:1009500002E000BF4FF0010C4DF804CD4FEA410C0E
:100960007FEA6C5C4FEA430C18BF7FEA6C5C1BD0DB
:1009700001B050EA410C0CBF52EA430C91EA030F5C
:1009800002BF90EA020F0020704710F1000F91EAB9
:10099000030F58BF994208BF90422CBFD8176FEA87
:1009A000E37040F0010070474FEA410C7FEA6C5C55
:1009B00002D150EA013C07D14FEA430C7FEA6C5C5C
:1009C000D6D152EA033CD3D05DF8040B704700BF88
:1009D0008446104662468C461946634600E000BFD6
:1009E00001B5FFF7B7FF002848BF10F1000F01BDA8
:1009F0004DF808EDFFF7F4FF0CBF012000205DF873
:100A000008FB00BF4DF808EDFFF7EAFF34BF0120F7
:100A100000205DF808FB00BF4DF808EDFFF7E0FF90
:100A200094BF012000205DF808FB00BF4DF808EDE1
:100A3000FFF7CEFF94BF012000205DF808FB00BF48
:100A40004DF808EDFFF7C4FF34BF012000205DF82A
:100A500008FB00BF4FEA410212F5001215D211D572
:100A60006FF47873B3EB625212D94FEAC12343F0AB
:100A7000004343EA505311F0004F23FA02F018BF2D
:100A8000404270474FF00000704750EA013005D1F6
:100A900011F0004008BF6FF0004070474FF00000B9
:100AA000704700BF4FEA4102B2F1E04324BFB3F503
:100AB000001CDCF1FE5C0DD901F0004C4FEAC002D5
:100AC0004CEA5070B2F1004F40EB830008BF20F0B9
:100AD0000100704711F0804F21D113F13872BCBF73
:100AE00001F00040704741F480114FEA5252C2F1C8
:100AF0001802C2F1200C10FA0CF320FA02F018BF11
:100B000040F001004FEAC1234FEAD32303FA0CFC63
:100B100040EA0C0023FA02F34FEA4303CCE77FEAF2
:100B2000625307D150EA01331EBF4FF0FE4040F43C
:100B30004000704701F0004040F0FE4040F40000EB
:100B4000704700BF844641EA000313F003036DD1F0
:100B5000403A41D351F8043B40F8043B51F8043B80
:100B600040F8043B51F8043B40F8043B51F8043B87
:100B700040F8043B51F8043B40F8043B51F8043B77
:100B800040F8043B51F8043B40F8043B51F8043B67
:100B900040F8043B51F8043B40F8043B51F8043B57
:100BA00040F8043B51F8043B40F8043B51F8043B47
:100BB00040F8043B51F8043B40F8043B51F8043B37
:100BC00040F8043B51F8043B40F8043B51F8043B27
:100BD00040F8043B403ABDD2303211D351F8043BC7
:100BE00040F8043B51F8043B40F8043B51F8043B07
:100BF00040F8043B51F8043B40F8043B103AEDD276
:100C00000C3205D351F8043B40F8043B043AF9D2C6
:100C1000043208D0D2071CBF11F8013B00F8013B99
:100C200001D30B8803806046704700BF082A13D3A6
:100C30008B078DD010F003038AD0C3F10403D21ABE
:100C4000DB071CBF11F8013B00F8013B80D331F8F2
:100C5000023B20F8023B7BE7043AD9D3013A11F872
:100C6000013B00F8013BF9D20B7803704B784370DD
:100C70008B788370604670474BB942B9002908BF32
:100C8000002802D04FF0FF31084600F03BB882B098
:100C9000EC462DE9005000F01DF8DDF804E002B04C
:100CA0000CBC70472DE97043069E14461D468046D5
:100CB000894600F029F804FB01F300FB0533A4FB8F
:100CC00000451D44B8EB040469EB0505C6E9004581
:100CD000BDE870832DE97043069E14468046894620
:100CE0001D4600F05DF900FB05F504FB0153A0FB78
:100CF00004451D44B8EB040469EB0505C6E900454D
:100D0000BDE87083704700BF00292DE9F00FC0F2E5
:100D10009F800024002BC0F29680154606460F46A1
:100D2000002B3ED18A4257D9B2FA82F34BB1C3F1BC
:100D3000200201FA03F720FA02F29D40174300FA5D
:100D400003F6290CB7FBF1F2330C01FB127CA8B2BD
:100D500043EA0C4700FB02F3BB4209D97F1902F1B9
:100D6000FF3C80F00181BB4240F2FE80023A2F44FA
:100D7000FF1AB7FBF1F3B6B201FB137146EA01416A
:100D800000FB03F0884208D9491903F1FF3780F0CE
:100D9000ED80884240F2EA80023B43EA02420023AF
:100DA00003E08B420AD900231A461046194614B1B3
:100DB000404261EB4101BDE8F00F7047B3FA83F8A0
:100DC000B8F1000F40F084808B4202D3824200F2DF
:100DD000DE8000230122E8E712B90123B3FBF2F51C
:100DE000B5FA85F2002A39D17F1B280C1FFA85FC41
:100DF0000123B7FBF0F1320C00FB117742EA074701
:100E00000CFB01F2BA4207D97F1901F1FF3802D277
:100E1000BA4200F2C1804146BF1AB7FBF0F2B6B247
:100E200000FB127046EA00400CFB02FC844507D927
:100E3000401902F1FF3702D2844500F2AB803A46F6
:100E400042EA0142B1E7E443524263EB430364E701
:100E5000404261EB41014FF0FF345BE79540C2F146
:100E6000200327FA03F1280C26FA03F39740B1FB7D
:100E7000F0F81F433B0C00FB18111FFA85FC43EAF6
:100E800001410CFB08F38B4206FA02F608D9491916
:100E900008F1FF3279D28B4277D9A8F102082944B0
:100EA000C91AB1FBF0F3BFB200FB131147EA0147C7
:100EB0000CFB03F2BA4207D97F1903F1FF3160D26C
:100EC000BA425ED9023B2F44BF1A43EA084390E777
:100ED000C8F1200203FA08FC25FA02F343EA0C0CDD
:100EE0004FEA1C4921FA02F301FA08F720FA02F24C
:100EF000B3FBF9F1174309FB11333A0C1FFA8CFBD2
:100F000042EA03430BFB01FA9A4505FA08F008D9B7
:100F100013EB0C0301F1FF3235D29A4533D9023974
:100F20006344CAEB0303B3FBF9F209FB1233BFB20C
:100F300047EA03470BFB02F9B94508D917EB0C0741
:100F400002F1FF331BD2B94519D9023A674442EA8C
:100F50000145A5FB0001C9EB07078F424FF00003D5
:100F60000AD305D02A4620E7624601E73B4614E74C
:100F700006FA08F68642F5D26A1E002315E71A46DD
:100F8000E5E70B46A0E71146CBE7904688E74346E6
:100F900042460AE7023A53E702392F443CE700BFD2
:100FA0002DE9F00F144605460E46002B43D18A4228
:100FB00053D9B2FA82F757B1C7F1200620FA06F6E4
:100FC00001FA07F302FA07F41E4300FA07F5210CB1
:100FD000B6FBF1F22B0C01FB1267A0B243EA074605
:100FE00000FB02F3B34209D9361902F1FF3780F052
:100FF000F680B34240F2F380023A2644F61AB6FB7A
:10100000F1F3ADB201FB136145EA014100FB03F0CE
:10101000884208D9091903F1FF3680F0E28088423E
:1010200040F2DF80023B43EA0242002310461946A9
:10103000BDE8F00F70478B424AD8B3FA83F6002E12
:101040004DD18B4202D3824200F2D680002301228E
:1010500010461946BDE8F00F704712B90124B4FBE1
:10106000F2F4B4FA84F2002A7CD1091B260CA7B250
:101070000123B1FBF6F02A0C06FB101142EA0141F4
:1010800007FB00F28A4207D9091900F1FF3C02D29E
:101090008A4200F2C3806046891AB1FBF6F2ADB213
:1010A00006FB121145EA014507FB02F7AF4208D9DA
:1010B0002C1902F1FF3180F09680A74240F2938014
:1010C000023A42EA004210461946BDE8F00F704766
:1010D00000231A4610461946BDE8F00F7047C6F1C6
:1010E000200522FA05F4B3401C434FEA144821FAC4
:1010F00005F301FA06F720FA05F5B3FBF8FC2F43D8
:1011000008FB1C333D0C1FFA84FA45EA03430AFB33
:101110000CF9994502FA06FB04D91B190CF1FF32B0
:101120006DD39446C9EB0303B3FBF8F508FB153305
:10113000BFB247EA03470AFB05F8B84504D93F198F
:1011400005F1FF3361D31D4645EA0C4CACFB0B2384
:10115000C8EB07079F424FF0000549D345D06246D0
:101160002B4663E79440C2F1200321FA03FC260CCE
:1011700020FA03F301FA02F5BCFBF6F843EA050195
:101180000B0C06FB18CCA7B243EA0C4C07FB08F388
:10119000634500FA02F509D91CEB040C08F1FF3293
:1011A0003AD2634538D9A8F10208A444C3EB0C0C29
:1011B000BCFBF6F389B206FB13CC41EA0C4107FBFA
:1011C00003F28A4207D9091903F1FF3022D28A4279
:1011D00020D9023B2144891A43EA084349E73A46A9
:1011E0000CE733461FE70A466BE7B0409042B6D2A1
:1011F0000CF1FF32002319E73346324616E79945D2
:101200008FD9ACF1020C23448CE7B8459BD9023D41
:10121000274499E70346DEE79046C7E702382144B2
:101220003AE700BF90B484B000AF02460B46FA71B3
:10123000BB710023FB60BB7903F003039B000F220B
:1012400002FA03F3FB60154BBA799208D2B2134944
:10125000B8798008C0B2023051F82000F968C9435B
:101260000140023243F822100C4BBA799208D2B2F4
:101270000A49B8798008C0B2023051F82000FC79E0
:10128000B97901F00301890004FA01F10143023246
:1012900043F822101037BD4690BC7047003801401B
:1012A00080B500AF00F0C8F900F00CFA00F074F857
:1012B0000346002B01D0042308E000F087F801204A
:1012C000012100F0ADF800F0D3F80023184680BDEE
:1012D00080B584B000AF402000F0C4FA034603F0AC
:1012E00080039AB2294B1A80284B1B88002B30D0E0
:1012F00000F030F90346FB6000F060F90346BB6084
:10130000234B1B68FA689A4204D9214B1B68FA6880
:10131000D31A03E01E4B1A68FB68D31A7B601D4B7F
:101320001B68BA689A4204D91A4B1B68BA68D31A68
:1013300003E0184B1A68BB68D31A3B607A683B68B5
:101340001344052B05D9124BFA681A60114BBA6881
:101350001A600F4B1B689AB20C4B5A800D4B1B68DE
:101360009AB20A4B9A8000F053F903461A46074B8B
:10137000DA804B20012100F0C7F94B20002100F05A
:10138000C3F9024B18461037BD4680BD985F002058
:10139000300A0020340A002080B500AF00F026F8A3
:1013A00003461A4640F611039A4209D0064B1B68C1
:1013B000002B03D100F02AFC034602E0012300E0E9
:1013C0000023184680BD00BF0000002080B500AF9C
:1013D0000320022100F098F9022000F04DFC0320C8
:1013E000002100F091F90023184680BD80B582B03D
:1013F00000AF0023FB80002000F034FA0346FB809E
:10140000FB881B02FB80012000F02CFA03461A46E1
:10141000FB881343FB80FB8818460837BD4680BD18
:1014200080B584B000AF02460B46FA71BB71002351
:10143000FB73042000F016FA0346FB73BB79002B04
:1014400007D0FB79DB43DAB2FB7B1340DBB2FB73E3
:1014500003E0FA7BFB791343FB73FB7B0420194603
:1014600000F052F9002318461037BD4680BD00BF7A
:1014700080B500AF02200121FFF7D2FF20204921D3
:1014800000F042F9022000F0F7FB2120012100F0DA
:101490003BF91E20002100F035F841209A2100F090
:1014A00033F94A20012100F02FF94B20012100F0EF
:1014B0002BF94B20002100F027F95620012100F0E4
:1014C00023F95820012100F01FF94020032100F0EA
:1014D0001BF90B20FF2100F017F9094B0022DA80DD
:1014E000074BDA88064B9A80054B9A88044B5A8042
:1014F000034B5A88024B1A800023184680BD00BF58
:10150000985F002080B584B000AF02460B46FA71A8
:10151000BB710023FB73172000F0A4F90346FB7393
:10152000BB79002B04D0FA7BFB791343FB7306E0F5
:10153000FB79DB43DAB2FB7B1340DBB2FB73FB7B53
:101540001720194600F0E0F8002318461037BD4672
:1015500080BD00BF80B582B000AF4D2000F070FAB2
:1015600003467B607A6840F6B8339A4205DC7B68B4
:10157000C3F571630E337B6004E07B68C3F56D6374
:1015800008337B607B680C4A82FB03121A44D2103A
:10159000DB17D31A3B603B68002B02DC00233B6067
:1015A00004E03B68F02B01DDEF233B603B689BB21E
:1015B00018460837BD4680BD8988888880B582B0C6
:1015C00000AF4F2000F03CFA03463B603B68A3F5B8
:1015D000B4733B603B680D4A82FB03125210DB1769
:1015E000D31A7B607B68002B02DC00237B6006E063
:1015F0007B68B3F5A07F02DD40F23F137B607B6820
:101600009BB218460837BD4680BD00BFE9A28B2EAD
:1016100080B582B000AF512000F012FA03467B6023
:101620007B68002B01D100237B607B689BB218464E
:101630000837BD4680BD00BF80B582B000AF4FF413
:101640000000012101F054FA40F20510012101F0DF
:1016500013FA4FF48040012101F068FA4FF40000C2
:10166000012101F081FA4FF40000002101F07CFA21
:1016700012480821042202F043FE114809210422E5
:1016800002F03EFE4FF480733B6002233B71022365
:101690007B710123BB710023FB713B460748194650
:1016A00002F06CFD4FF400733B603B460448194662
:1016B00002F064FD0837BD4680BD00BF0000024057
:1016C0000008024080B584B000AF0023BB804BF619
:1016D000FF73FB8000233B814FF480637B814FF4D9
:1016E0008043BB81064B3B603B460648194604F0ED
:1016F00025F90448012104F0E3F91037BD4680BD07
:10170000A0860100005C004080B584B000AF0246B6
:101710000B46FA71BB710023FB604C48012104F0B9
:10172000EFF94B4B4FF440521A600AE0484B1B68EC
:10173000591E474A1160002B03D100F067FA034697
:1017400080E04248434904F0B9FA0346002BEDD04B
:101750003E488221002204F013FA3D4B4FF44052E0
:101760001A600AE03A4B1B68591E394A1160002B77
:1017700003D100F04BFA034664E03448364904F0E4
:101780009DFA0346002BEDD0304B1B8B304B4FF4B2
:1017900040521A600AE02E4B1B68591E2C4A1160F9
:1017A000002B03D100F032FA03464BE027482B49C7
:1017B00004F084FA0346002BEDD0FB792348194648
:1017C00004F05EFA224B4FF440521A600AE0204BBC
:1017D0001B68591E1E4A1160002B03D100F016FA37
:1017E00003462FE019481D4904F068FA0346002B10
:1017F000EDD0BB791548194604F042FA144B4FF46A
:1018000040521A600AE0124B1B68591E104A1160C0
:10181000002B03D100F0FAF9034613E00B480F49FF
:1018200004F04CFA0346002BEDD008480C4904F0B4
:1018300045FA0346002BE6D00448012104F080F964
:10184000FB68DBB218461037BD4680BD005C004027
:1018500000000020010000100200001080000010B5
:101860000400001080B584B000AF0346FB71002374
:10187000FB736C48012104F043F96B4B4FF4405269
:101880001A600AE0684B1B68591E674A1160002BFA
:1018900003D100F0BBF90346C0E06248634904F09D
:1018A0000DFA0346002BEDD05E48002104F086F9C6
:1018B0005C488221002204F063F95B4B4FF44052F4
:1018C0001A600AE0584B1B68591E574A1160002BDA
:1018D00003D100F09BF90346A0E05248544904F0BC
:1018E000EDF90346002BEDD04E4B1B8B4E4B4FF4C6
:1018F00040521A600AE04C4B1B68591E4A4A11605C
:10190000002B03D100F082F9034687E0454849499E
:1019100004F0D4F90346002BEDD0FB794148194679
:1019200004F0AEF9404B4FF440521A600AE03E4BCF
:101930001B68591E3C4A1160002B03D100F066F968
:1019400003466BE037483B4904F0B8F90346002BE7
:10195000EDD03448384904F0B1F90346002BE6D005
:101960003048012104F0CCF82F4B4FF440521A605C
:101970000AE02D4B1B68591E2B4A1160002B03D126
:1019800000F044F9034649E02648284904F096F956
:101990000346002BEDD023488221012204F0F0F809
:1019A000214B4FF440521A600AE01F4B1B68591E2E
:1019B0001D4A1160002B03D100F028F903462DE0E9
:1019C00018481B4904F07AF90346002BEDD0154B5B
:1019D0001B8B154B4FF440521A600AE0124B1B68E8
:1019E000591E114A1160002B03D100F00FF9034674
:1019F00014E00C48114904F061F90346002BEDD0C6
:101A00000848012104F09CF8064804F049F903460F
:101A1000FB730448012104F0D1F8FB7B1846103712
:101A2000BD4680BD005C00400000002001000010A9
:101A300002000010800000100400001040000010A0
:101A400080B584B000AF786000233B7300237B73C4
:101A50006848012104F054F8674B4FF440521A6073
:101A60000AE0654B1B68591E634A1160002B03D1C5
:101A700000F0CCF80346B9E05E48604904F01EF976
:101A80000346002BEDD05B488221002204F078F859
:101A9000594B4FF440521A600AE0574B1B68591ECD
:101AA000554A1160002B03D100F0B0F803469DE0C9
:101AB0005048534904F002F90346002BEDD04D4B3A
:101AC0001B8B4D4B4FF440521A600AE04A4B1B6887
:101AD000591E494A1160002B03D100F097F80346C4
:101AE00084E04448474904F0E9F80346002BEDD070
:101AF0007B68DBB23F48194604F0C2F83D4801213B
:101B000003F0FEFF3C4B4FF440521A600AE03A4BA0
:101B10001B68591E384A1160002B03D100F076F87B
:101B2000034663E03348354904F0C8F80346002B08
:101B3000EDD030488221012204F022F82E4B4FF4E0
:101B400040521A600AE02C4B1B68591E2A4A116049
:101B5000002B03D100F05AF8034647E025482849F6
:101B600004F0ACF80346002BEDD02248002104F02D
:101B700025F820484FF4006104F062F81D4B1B8BE0
:101B80001D4B4FF440521A600AE01B4B1B68591E54
:101B9000194A1160002B03D100F038F8034625E004
:101BA0001448194904F08AF80346002BEDD0114877
:101BB000012103F0C5FF0F4804F072F803467B7360
:101BC0000C4804F06DF803463B730A48012103F00A
:101BD000F5FF08484FF2FF7104F032F83B7B1A46DC
:101BE0007B7B1B029BB213439BB29BB21846103700
:101BF000BD4680BD005C00400000002001000010D8
:101C000002000010800000100400001080B584B0B5
:101C100000AF1748012103F093FF1548012103F09D
:101C2000EDFF1348002103F0E9FFFFF705FD104821
:101C300003F04AFE0023BB804BF6FF73FB80332387
:101C40003B814FF480637B814FF48043BB81094B20
:101C50003B600748012103F033FF3B460448194627
:101C600003F06CFE002318461037BD4680BD00BF50
:101C7000005C0040A086010080B485B000AF7860B1
:101C80000023FB607B68084A02FB03F3FB6002E071
:101C9000FB68013BFB60FB68002BF9D11437BD46A4
:101CA0005DF8047B704700BFA086010080B500AFDF
:101CB00002484FF4083115F01DFE80BDA05F0020E2
:101CC00080B483B000AF78600B46FB70FB78002BCC
:101CD00006D0094B084A11687A680A431A6006E080
:101CE000054B054A11687A68D2430A401A600C37DE
:101CF000BD465DF8047B704700B0024080B483B0FD
:101D000000AF0346FB71044BFA791A600C37BD46ED
:101D10005DF8047B704700BF20000E4280B500AF25
:101D2000214B00221A704FF08050012100F0E0FE9C
:101D30000120FFF7E3FF012000F060FD00BF6120FC
:101D400000F04EFF0346002BF9D04FF4007000F076
:101D500037FE012000F062FE04F048FF134B7F22A3
:101D60005A60124BFF229A60104B00221A600F48F3
:101D700004F0B8FE00F01EF802460D4B1A600B4B43
:101D80007F225A600A4B1B68DB095A1E074B9A6078
:101D9000064B00221A60054804F0A4FE024B1B7893
:101DA0005BB2184680BD00BF380A0020A47F022025
:101DB0003C0A002080B584B000AF012000F01EFD79
:101DC00000BF612000F00CFF0346002BF9D0082073
:101DD000012100F08DFE2A48402105F06BFF2848C4
:101DE0000021012205F000FE0C233B8000237B80B4
:101DF0000123BB800C23FB8000233B813B46204812
:101E0000194605F025FE32233B7300237B73002324
:101E1000BB730123FB7307F10C03184604F004FEA7
:101E20001748012105F0F4FD154B00221A821448D1
:101E30001021012205F0E0FE00BF124B1B68022BAF
:101E4000FBD10F4805F0F2FC0F4B9B6803F4E05305
:101E5000002B08D10D4B1B689A080D4B1B68B2FB79
:101E6000F3F3DB0008E0094B1B689B085A00084BA2
:101E70001B68B2FBF3F3DB0018461037BD4680BD8C
:101E8000000C0040400A00200038024020000020E2
:101E9000440A002080B500AF4FF4003004F0A4FDE8
:101EA0004FF4805004F0DEFE0346002B0CD00120DE
:101EB00004F056FF054B00221A704FF4805004F0D6
:101EC00005FF034B01221A7080BD00BF08000020EF
:101ED000A07F022080B489B000AF78600023FB614E
:101EE0000023BB6100237B6100233B610023FB6077
:101EF0000023BB603F4A3F4B99683F4B0B409360C8
:101F00007B681B691B04FB613A4B3A4A91687A680B
:101F10005069FA6902430A439A60364A354BD968D8
:101F2000354B0B40D3607B689B691B04BB61314B15
:101F3000304AD1687A68D069BA6902430A43DA60E4
:101F40002C4A2C4B19692C4B0B4013617B681B6A84
:101F50001B047B61274B274A11697A68506A7A69AA
:101F600002430A431A61234A224B5969224B0B4010
:101F700053617B689B6A1B043B611E4B1D4A516980
:101F80007A68D06A3A6902430A435A61194A194B7E
:101F900099691A4B0B409361164B164A91697A68FE
:101FA00010687A68526810437A68926810437A68B9
:101FB000D26802430A439A617B685B6B1B02FB6039
:101FC0007B681B6B1B04BB600A4B0A4AD26A02F097
:101FD0007F42DA62074B074AD16AB868FA68104351
:101FE0007A68926B02430A43DA622437BD465DF891
:101FF000047B70470068014000F800F08F88FE0FF6
:1020000080B483B000AF0346FB71FB79002B06D090
:10201000084B084A926942F001029A6105E0054BBB
:10202000044A926922F001029A610C37BD465DF8BC
:10203000047B70470068014080B483B000AF7860D3
:10204000034B7A685A620C37BD465DF8047B7047D3
:102050000068014080B489B000AF78603960002327
:10206000FB610023BB6100237B6100233B610023F4
:10207000FB600023BB603B685B681B04FB617B6803
:102080005B6803F470427B685A603B681A68FB69BE
:102090001A437B685A603B68DB681B04BB617B6842
:1020A0009B6803F470427B689A603B689A68BB69DE
:1020B0001A437B689A607B681B6923F007027B6880
:1020C0001A613B681A697B681A613B68DB691B020D
:1020D0007B613B681B6A1B043B613B685B6A1B06B8
:1020E000FB607B689B697B6800229A613B689A6908
:1020F0007B691A433B691A43FB681A437B689A6100
:102100007B685B6923F0FF027B685A613B685A6910
:102110007B685A617B68DB6923F4E06323F0070383
:102120007A68D3613B689A6A3B68DB6A1A437B68CA
:10213000DA617B689B6A7B6800229A623B681A6B53
:102140007B689A623B689B6B1B04BB607B68DB6AA5
:1021500003F0E0227B68DA623B685A6BBB681A4383
:102160007B68DA627B681B6B23F4FF6323F0070351
:102170007A6813633B68DA6B7B681A632437BD4661
:102180005DF8047B704700BF80B483B000AF786017
:102190000B46FB70FB78002B06D07B681B6843F076
:1021A00001027B681A6005E07B681B6823F001026E
:1021B0007B681A600C37BD465DF8047B704700BF32
:1021C00080B483B000AF78600B46FB70FB78002BC7
:1021D00006D0094B084A516B7A680A435A6306E0F5
:1021E000054B054A516B7A68D2430A405A630C3753
:1021F000BD465DF8047B70470068014080B58CB037
:1022000000AF4FF48070012100F090FC0420012108
:1022100000F032FC08233B6003233B710023FB7179
:102220003B461A48194601F0A9FF00F09FFF002322
:102230003B6200237B620023BB624FF47063FB624E
:1022400007F12003184600F0F3FF0023BB600023D2
:102250003B7300237B7300237B6100233B610023DE
:10226000BB6101233B7707F108030948194600F0D9
:102270008BFF0748012101F003F805480D210122D9
:10228000062301F019F83037BD4680BD0008024032
:102290000020014090B585B004AF4FF4407004F0C9
:1022A000B1FB0020002104F091FDFFF7A7FF0923F7
:1022B0000093184B019300230293002303931648C5
:1022C000164940F6E832002301F06AF9144B0093F6
:1022D000144832210122012300F0E2FC0246124B95
:1022E0001A60114B1B68002B0CD00F4B1C6801F0BF
:1022F000E5FA034600220092204600211A460023F8
:1023000000F0FEFC01F020FA002318460437BD4619
:1023100090BD00BFB07F0220E9230008D02C020846
:10232000E1270008E02C0208B47F022080B500AF4E
:10233000084801F085F800BF0648022101F09EF828
:102340000346002BF8D0034801F08AF803461846EC
:1023500080BD00BF0020014080B58CB002AF786026
:1023600039603B68022B33D11B4A07F1180307CAB7
:1023700083E80700194811F069FF12F0BBF9786291
:1023800007F11003184608F049FF07F108037868C1
:10239000194608F0C7FE3B8A9AB27B6A9BB2134487
:1023A0009BB29BB2BB824FF4004011F097FF07F144
:1023B000180318461DF016F8034607F1180107F137
:1023C00010020748009008461146022213F022FA34
:1023D0002837BD4680BD00BFE82C02085C570208C4
:1023E000380100200000000080B5B6B006AF78606C
:1023F0000023C7F8BC3003F0E5F913F00FFEC8481E
:1024000008F058F9C74807F0C7FA09F05BF8034627
:102410000093022301930023029300230393C24BF2
:102420000493002305930A201E21DC22E62307F0F3
:102430003BFFC7F8B800D7F8B80009F051F8C7F863
:10244000B400D7F8B800B94907F0C2FAD7F8B80015
:10245000022107F03DFFD7F8B43000930223019327
:10246000002302934FF40873039305200521C8222B
:10247000782306F073FEC7F8B00000230093D7F866
:10248000B00028210022002306F080FFD7F8B0001A
:102490000F2106F019FFD7F8B0000A2106F030FF2F
:1024A000D7F8B000012106F0F1FED7F8B000022104
:1024B00006F0AAFFD7F8B000022106F0C3FFD7F854
:1024C000B0009B4906F086FF4FF47F40C8210022F0
:1024D000002306F0A5F8C7F8AC00D7F8AC000A2135
:1024E00006F008F9D7F8B000D7F8AC1006F07EFE79
:1024F0002620012101221E2305F016FFC7F8A8009F
:10250000D7F8A8008B4905F07BFFD7F8A800012178
:1025100005F0A2FFD7F8A8000A2105F039FFD7F887
:10252000A800002105F050FFD7F8B000D7F8A81098
:1025300006F084FED7F8B430009302230193002301
:1025400002934FF4B07303937B4B04930A208C21C6
:102550006422142305F0EAFDC7F8A400D7F8B430CC
:102560000093022301930023029340F2611303932B
:10257000724B04930A20A0216422142305F0D6FD97
:10258000C7F8A000D7F8B4300093022301930023CA
:1025900002934FF4B1730393694B04930A20B4215F
:1025A0006422142305F0C2FDC7F89C00D7F8B430AC
:1025B0000093022301930023029340F263130393D9
:1025C000604B0493A020A0211422142305F0AEFD3B
:1025D000C7F89800D7F898005B4905F0D1FCD7F808
:1025E000B80008F00DF8D7F8BC305A1CC7F8BC206A
:1025F000052B40F2E7800023C7F8BC30002004F030
:10260000C7FBFFF793FE0346A7F89630B7F896305E
:102610001846FDF70FFF02460B46104619463CA32D
:10262000D3E90023FDF77CFF02460B46C7E92223CE
:10263000D7E922014FF00002444BFEF79BF8024617
:102640000B46C7E92023D7E9220133A3D3E90023AE
:10265000FDF7B2FD02460B46104619464FF0000248
:102660003B4BFEF787F802460B46C7E91E23D7E926
:102670001E014FF00002364BFEF77CF802460B4677
:10268000C7E91C23D7E920014FF00002314BFDF7C9
:1026900047FF02460B4610461946FEF7DBF9034694
:1026A0009BB21BB2D7F8AC00194606F001F807F14F
:1026B0000C0318462849D7E920231CF00FFE07F128
:1026C0000C03D7F8A400194605F02AFC07F10C0307
:1026D00018462249D7E91E231CF000FE07F10C031F
:1026E000D7F8A000194605F01BFC07F10C031846AB
:1026F0001B49D7E91C231CF0F1FD07F10C03D7F8A7
:102700009C00194605F00CFC2CE000BFAFF30080E4
:102710008FE4F21FD26FE73F000000000070974087
:102720008080FF0081940008D02C02083047020806
:1027300059230008022B073DF42C0208F82C02084C
:10274000FC2C0208042D0208383E020800408F408D
:102750000000244000003E40082D0208182D020809
:10276000282D0208D7E91E014FF00002174BFEF793
:1027700067F90346002B0BD0D7F89800144905F0F1
:10278000CFFBD7F898004FF47F0105F0AFFB19E0BD
:10279000D7E91E014FF000020E4BFEF733F9034656
:1027A000002B0AD0D7F898000B4905F0B9FBD7F8F1
:1027B0009800FF2105F09AFB04E0D7F8980007493C
:1027C00005F0AEFB0A2011F097FB0CE70000144067
:1027D000382D0208000014C03C2D0208042D020808
:1027E00080B582B000AF786003F00EF80837BD46C0
:1027F00080BD00BF80B400AFFEE700BF80B483B0EF
:1028000000AF0346FB71044BFA791A600C37BD46E2
:102810005DF8047B704700BF800E474280B485B0EE
:1028200000AFF860B9607A60074BFA689101BA6846
:10283000120611437A6812070A43C3F88820143736
:10284000BD465DF8047B70470038024080B483B019
:1028500000AF0346FB71044BFA791A600C37BD4692
:102860005DF8047B704700BF7000474280B489B0B8
:1028700000AF78600023BB6100237B610023FB6114
:1028800002233B610023FB600223BB60484B9B6833
:1028900003F00C03BB61BB69042B07D0082B09D0E4
:1028A000002B3FD17B68434A1A603FE07B68424A75
:1028B0001A603BE03E4B5B6803F480039B0DFB60BA
:1028C0003B4B5B6803F03F03BB60FB68002B0DD004
:1028D000394ABB68B2FBF3F2354B596847F6C0730F
:1028E0000B409B0903FB02F3FB610CE0314ABB6820
:1028F000B2FBF3F22E4B596847F6C0730B409B09AD
:1029000003FB02F3FB612A4B5B6803F440331B0CAF
:1029100001335B003B61FA693B69B2FBF3F27B6810
:102920001A6003E07B68234A1A6000BF204B9B6853
:1029300003F0F003BB61BB691B09BB611F4ABB69A4
:1029400013441B78DBB27B617B681A687B69DA40D1
:102950007B685A60164B9B6803F4E053BB61BB690C
:102960009B0ABB61154ABB6913441B78DBB27B61D0
:102970007B685A687B69DA407B689A600C4B9B687D
:1029800003F46043BB61BB695B0BBB610B4ABB6972
:1029900013441B78DBB27B617B685A687B69DA4041
:1029A0007B68DA602437BD465DF8047B704700BF62
:1029B000003802400024F40000127A000C000020CD
:1029C00080B485B000AF78600023FB607B6803F4BF
:1029D0004073B3F5407F11D10F4B9B68FB60FB68E0
:1029E00023F4F813FB607B6823F0704323F44073F7
:1029F000FA681343FB60084BFA689A60064B064A74
:102A0000116F7A68C2F30B020A431A671437BD4686
:102A10005DF8047B704700BF0038024080B483B08B
:102A200000AF0346FB71044BFA791A600C37BD46C0
:102A30005DF8047B704700BF3C0E474280B485B010
:102A400000AF78600023FB600A4BD3F88C30FB604A
:102A5000FB6823F44033FB60FA687B681343FB6038
:102A6000044BFA68C3F88C201437BD465DF8047B2C
:102A7000704700BF0038024080B483B000AF786078
:102A80000B46FB70FB78002B06D0094B084A116BF4
:102A90007A680A431A6306E0054B054A116B7A68A7
:102AA000D2430A401A630C37BD465DF8047B704779
:102AB0000038024080B483B000AF78600B46FB70F2
:102AC000FB78002B06D0094B084A916B7A680A43C1
:102AD0009A6306E0054B054A916B7A68D2430A4037
:102AE0009A630C37BD465DF8047B7047003802409E
:102AF00080B483B000AF78600B46FB70FB78002B8E
:102B000006D0094B084A116C7A680A431A6406E039
:102B1000054B054A116C7A68D2430A401A640C3797
:102B2000BD465DF8047B70470038024080B483B036
:102B300000AF78600B46FB70FB78002B06D0094B8A
:102B4000084A516C7A680A435A6406E0054B054A04
:102B5000516C7A68D2430A405A640C37BD465DF81E
:102B6000047B70470038024080B483B000AF7860C7
:102B70000B46FB70FB78002B06D0094B084A116A04
:102B80007A680A431A6206E0054B054A116A7A68B8
:102B9000D2430A401A620C37BD465DF8047B704789
:102BA0000038024080B483B000AF78600B46FB7001
:102BB000FB78002B06D0094B084A516A7A680A4311
:102BC0005A6206E0054B054A516A7A68D2430A40C8
:102BD0005A620C37BD465DF8047B704700380240EE
:102BE00080B487B000AF0346FB710023FB60002375
:102BF0007B610023FB74FB795B09DBB2FB60FB6844
:102C0000012B03D1124B1B687B6109E0FB68022B8F
:102C100003D10F4B1B6F7B6102E00D4B5B6F7B6140
:102C2000FB7903F01F03FB60FB687A6922FA03F368
:102C300003F00103002B02D00123FB7401E0002309
:102C4000FB74FB7C18461C37BD465DF8047B70475F
:102C50000038024080B586B004AF00237B6000F0EE
:102C60005BFA0C4B1B68002B0ED00A230093002349
:102C7000019300230293002303930748074980220E
:102C8000002300F08DFC78607B6818460837BD464D
:102C900080BD00BF780A0020F12D0008402D0208F9
:102CA00080B586B000AFF860B9607A603B60BB6801
:102CB000002B02D100237B611CE0282004F062FC81
:102CC00078617B69002B15D000F026FA7B69FA68E1
:102CD0001A607B69BA689A617B697A68DA617B6994
:102CE0003A681A627B693A6A5A627B690433184609
:102CF00001F040FD7B6918461837BD4680BD00BF16
:102D000080B588B000AFF860B9607A603B6000239E
:102D1000FB611D4B1B68002B30D0BB683B617B689F
:102D20007B61FB68BB613B68002B1CD101F012F991
:102D30000346012B0BD1144B1A6807F11003104600
:102D40001946BA6A002302F07BF8F86116E00E4BD0
:102D50001A6807F11003104619460022002302F0FA
:102D60006FF8F8610AE0084B1A6807F11003104683
:102D700019463A68002302F0E9F8F861FB69184641
:102D80002037BD4680BD00BF780A002080B586B0E0
:102D900002AF78603960154B1B68DB68DB68FB604D
:102DA000FB680433184601F051FDFB68DB69012B19
:102DB00015D1FB689A697B681344F86819463A682C
:102DC0007B6800F0A3F80346012B08D10023009391
:102DD000F86800217A680023FFF792FFB860FB686B
:102DE0005B6AF86898471037BD4680BD700A0020BE
:102DF00080B584B000AF786007F10803184600F092
:102E00003FF8F860BB68F868194600F003F800F076
:102E1000BFF8F1E780B584B000AF7860396000F0AA
:102E2000C5FC07F10803184600F04EF8F860BB68CF
:102E3000002B1ED13B68002B0AD17A68FB689A42AE
:102E400006D800F0C1FC7868F968FFF79FFF12E030
:102E50000A4B1A687968FB68CB1A1046194602F0CB
:102E600067FA00F0B1FC0346002B04D102F0F8FA37
:102E700001E000F0A9FC1037BD4680BD780A0020B3
:102E800080B485B000AF78600E4B1B681B68002BC8
:102E900014BF00230123DBB21A467B681A607B68EB
:102EA0001B68002B05D1074B1B68DB681B68FB60A8
:102EB00001E00023FB60FB6818461437BD465DF84F
:102EC000047B7047700A002080B584B000AF786042
:102ED00000F0F4FCF8600C4B1B68FA689A4208D2C8
:102EE000094B1B68184600F0C3F87B6801221A6082
:102EF00002E07B6800221A60034BFA681A60FB68E4
:102F000018461037BD4680BD7C0A002080B586B0CB
:102F100000AFF860B9607A603B6000237B61FB68BA
:102F2000BA685A60FB68FA681A61BA687B689A42A4
:102F300012D87A683B68D21AFB689B699A4202D31E
:102F400001237B611BE0104B1A68FB6804331046B9
:102F5000194601F043FC12E07A683B689A4206D2B7
:102F6000BA683B689A4202D301237B6107E0074BB2
:102F70001A68FB6804331046194601F02FFC7B6980
:102F800018461837BD4680BD740A0020700A00201C
:102F900080B58AB002AF3B1D1846FFF795FFF86178
:102FA00053E03B69BB61BB69002B08D0BB695B691F
:102FB000002B04D0BB690433184601F047FCBB6802
:102FC000032B41D801A252F823F000BFDD2F0008E7
:102FD000493000082530000841300008FA68BB6914
:102FE0009B691A44FB68B8691146FA69FFF78EFFBE
:102FF0000346012B15D1BB695B6AB8699847BB6969
:10300000DB69012B0DD1FA68BB699B69134400226F
:103010000092B86900211A460023FFF771FE78611B
:1030200013E012E0FA68BB699A61BB699A69FB69AF
:103030001344B8691946FA69FB69FFF767FF04E0B2
:10304000B86904F045FB00E000BF084B1A6807F1BF
:103050000803104619460022002301F0B7FF03467B
:10306000002B9ED12037BD4680BD00BF780A0020CE
:1030700080B58AB002AF786037E0254B1B68DB680B
:103080001B68FB61224B1B68DB68DB68BB61BB69AB
:103090000433184601F0DAFBBB695B6AB8699847EC
:1030A000BB69DB69012B20D1BB699A69FB691344B9
:1030B0007B617A69FB699A420ED9BB697A695A6069
:1030C000BB69BA691A61124B1A68BB6904331046AE
:1030D000194601F083FB08E000230093B869002142
:1030E000FA690023FFF70CFE3861094B1B681B6867
:1030F000002BC2D1064B1B68FB60064B1A68044BC1
:103100001A60044BFA681A602037BD4680BD00BFC4
:10311000700A0020740A002080B500AF02F0ACF9FC
:103120000D4B1B68002B13D10C4801F003FB0C481E
:1031300001F000FB0B4B094A1A600B4B084A1A605E
:103140000A200C21002201F0FDFD0246024B1A600C
:1031500002F0A4F980BD00BF780A0020480A0020D0
:103160005C0A0020700A0020740A002080B500AFBD
:103170004FF480700121FFF715FD4FF4807000219E
:10318000FFF710FD80BD00BF80B485B000AF786050
:1031900039600023FB600023FB727B685B68FB6087
:1031A000FB6823F0407323F48073FB603B681B795A
:1031B0001A023B681B681343FA681343FB607B6881
:1031C000FA685A607B689B68FB60FA68174B13408B
:1031D000FB603B681A693B68DB681A433B689B6885
:1031E0001A433B685B795B001343FA681343FB6047
:1031F0007B68FA689A607B68DB6AFB60FB6823F493
:103200007003FB603B681B7D013BDAB2FB7A134322
:10321000FB72FB7A1B05FA681343FB607B68FA6854
:10322000DA621437BD465DF8047B7047FDF7FFC0D6
:1032300080B485B000AF78600023FB600E4B5B6804
:10324000FB60FA680D4B1340FB607B681A687B6873
:103250005B681A437B689B681A437B68DB6813438F
:10326000FA681343FB60044BFA685A601437BD4692
:103270005DF8047B704700BF00230140E030FCFF95
:1032800080B483B000AF78600B46FB70FB78002BF6
:1032900006D07B689B6843F001027B689A6005E07A
:1032A0007B689B6823F001027B689A600C37BD46FF
:1032B0005DF8047B704700BF80B485B000AF7860D4
:1032C000F970BA707B700023FB600023BB60FB7851
:1032D000092B23D97B68DB68FB60FB78A3F10A022A
:1032E00013465B001344072202FA03F3BB60BB687A
:1032F000DB43FA681340FB607978FB78A3F10A029C
:1033000013465B00134401FA03F3BB60FA68BB6821
:103310001343FB607B68FA68DA601EE07B681B6918
:10332000FB60FA7813465B001344072202FA03F3AA
:10333000BB60BB68DB43FA681340FB607978FA78BE
:1033400013465B00134401FA03F3BB60FA68BB68E1
:103350001343FB607B68FA681A61BB78062B21D89F
:103360007B685B6BFB60BB785A1E13469B00134463
:103370001F2202FA03F3BB60BB68DB43FA68134009
:10338000FB60F978BB785A1E13469B00134401FA80
:1033900003F3BB60FA68BB681343FB607B68FA68A1
:1033A0005A6347E0BB780C2B21D87B681B6BFB6012
:1033B000BB78DA1F13469B0013441F2202FA03F363
:1033C000BB60BB68DB43FA681340FB60F978BB78ED
:1033D000DA1F13469B00134401FA03F3BB60FA683B
:1033E000BB681343FB607B68FA681A6322E07B6862
:1033F000DB6AFB60BB78A3F10D0213469B0013440C
:103400001F2202FA03F3BB60BB68DB43FA68134078
:10341000FB60F978BB78A3F10D0213469B001344BF
:1034200001FA03F3BB60FA68BB681343FB607B6877
:10343000FA68DA621437BD465DF8047B704700BF56
:1034400080B483B000AF78607B689B6843F08042B3
:103450007B689A600C37BD465DF8047B704700BFFF
:1034600080B483B000AF78607B68DB6C9BB2184699
:103470000C37BD465DF8047B704700BF80B485B053
:1034800000AF78600B46FB700023FB737B681A6803
:10349000FB781340002B02D00123FB7301E00023D3
:1034A000FB73FB7B18461437BD465DF8047B704701
:1034B00080B400AFBD465DF8047B704780B400AFB8
:1034C000FEE700BF80B400AFFEE700BF80B400AFEE
:1034D000FEE700BF80B400AFFEE700BF80B400AFDE
:1034E000BD465DF8047B704780B500AF034B0122F9
:1034F0001A60012003F078FA80BD00BF800A002026
:1035000080B400AFBD465DF8047B704780B400AF67
:10351000BD465DF8047B704798B500AF1348102195
:1035200004F08EFB0346002B1ED0114B1B681C467B
:10353000621C0F4B1A600D4804F0DEFA03469AB283
:103540000C4B23F814200948102104F0A3FB084B6E
:103550001B68012B08D9074B5A88064B1B88D31AC6
:103560009BB21A46044B1A6098BD00BF000C004085
:10357000400A0020840A0020440A002080B400AFE2
:10358000BD465DF8047B704780B500AF02F0FAFFDE
:1035900080BD00BF80B500AF02F0E8FF80BD00BF76
:1035A00080B58AB002AFF860B9603B601346FB801B
:1035B000FB881846396B00F07BFCB861BB69002BB7
:1035C00074D0BB691A6BFB8803F18043013B9B00FD
:1035D00013447B617B6923F007037B61FB880093C5
:1035E000B869B968BA6A7B6B00F07EFB7869F968E4
:1035F0003A6801F0C7FE0246BB691A60FB6A002BFD
:1036000002D0FB6ABA691A6001F036FF334B1B68BF
:103610005A1C324B1A60324B1B68002B09D1304BBD
:10362000BA691A602D4B1B68012B0FD100F092FB79
:103630000CE02C4B1B68002B08D1294B1B68DA6A65
:10364000BB6A9A4202D8264BBA691A60BB69DA6A29
:10365000254B1B689A4203D9BB69DA6A224B1A6070
:10366000224B1A68BB695A64204B1B685A1C1F4BBB
:103670001A60BB69DA6A1E4B1B689A4203D9BB69A0
:10368000DA6A1B4B1A60BB69DA6A13469B00134463
:103690009B00184A1A44BB6904331046194601F0CE
:1036A00075F80123FB6101F0F9FE02E04FF0FF33F2
:1036B000FB61FB69012B0BD10A4B1B68002B07D068
:1036C000074B1B68DA6ABB6A9A4201D201F0C8FE56
:1036D000FB6918462037BD4680BD00BFEC0B0020BB
:1036E000880A0020FC0B0020F40B0020100C0020A6
:1036F000F80B00208C0A002080B584B000AF786001
:103700000023FB607B68002B12D000F04FF80C4BBD
:103710001A687B681344BB600A4B1B680433184665
:1037200001F094F8B86800F08DFB00F04DF8F860F7
:10373000FB68002B01D101F093FE1037BD4680BD20
:10374000F00B0020880A002080B586B004AF00236B
:1037500000930023019300230293002303930F4857
:103760000F4980220023FFF71BFF78607B68012B45
:1037700002D1FFF76FFA78607B68012B0BD14FF015
:10378000500080F31188074B01221A60064B00227B
:103790001A6001F03FFE0837BD4680BDC53C0008F9
:1037A000482D0208FC0B0020F00B002080B400AF75
:1037B000044B1B685A1C034B1A60BD465DF8047B22
:1037C000704700BF000C002090B583B000AF00230D
:1037D0007B6001F051FE314B1B685A1E2F4B1A6063
:1037E0002E4B1B68002B52D12D4B1B68002B4ED04B
:1037F00000233B6027E02B4BDB68DC6804F11803F7
:10380000184601F023F8231D184601F01FF8E26A5C
:10381000254B1B689A4202D9E26A234B1A60E26A7E
:1038200013469B0013449B00204A1A44231D104654
:10383000194600F0ABFFE26A1D4B1B68DB6A9A4237
:1038400001D301233B60174B1B68002BD3D1194BCD
:103850001B68002B0DD006E000F042F8154B1B68EA
:103860005A1E144B1A60134B1B68002BF4D1012312
:103870003B603B68012B03D00F4B1B68012B06D12B
:1038800001237B600C4B00221A6001F0E9FD01F07E
:1038900005FE7B6818460C37BD4690BD000C002025
:1038A000EC0B0020AC0B0020F80B00208C0A002051
:1038B000880A0020040C0020080C002080B582B08B
:1038C00000AF01F0D9FD054B1B687B6001F0E6FD00
:1038D0007B6818460837BD4680BD00BFF00B00204E
:1038E00080B584B000AF444B1B68002B73D1434BB1
:1038F0001B685A1C414B1A60404B1B68002B21D19E
:103900003F4B1B68FB603F4B1A683D4B1A603D4BB9
:10391000FA681A603C4B1B685A1C3B4B1A60384BC8
:103920001B681B68002B04D1384B4FF0FF321A6024
:1039300008E0334B1B68DB68DB68BB60BB685A6818
:10394000324B1A602D4B1A68304B1B689A4241D398
:103950002B4B1B681B68002B04D12C4B4FF0FF3204
:103960001A6037E0264B1B68DB68DB68BB60BB680E
:103970005B687B60214B1A687B689A4203D2234BB9
:103980007A681A6026E0BB680433184600F05EFFD0
:10399000BB689B6A002B04D0BB681833184600F044
:1039A00055FFBB68DA6A1A4B1B689A4203D9BB6899
:1039B000DA6A174B1A60BB68DA6A13469B00134435
:1039C0009B00144A1A44BB6804331046194600F0A1
:1039D000DDFEBDE706E0104B1B685A1C0E4B1A605B
:1039E00003F0BCFE0C4B1B68002B01D103F0B6FEAC
:1039F0001037BD4680BD00BF000C0020F00B00203A
:103A0000A40B0020A80B00200C0C00201C000020A0
:103A1000F80B00208C0A0020040C002080B582B036
:103A200000AF1F4B1B68002B03D01E4B01221A60F6
:103A300032E003F0D9FE04E01B4B1B685A1E1A4B00
:103A40001A60194B1A68194913469B0013449B00CE
:103A50000B441B68002BEFD0134B1A6813469B00D6
:103A600013449B00114A13447B607B685B685A686F
:103A70007B685A607B685A687B6808339A4204D135
:103A80007B685B685A687B685A607B685B68DA6849
:103A9000074B1A6003F094FE0837BD4680BD00BF97
:103AA000000C0020080C0020F80B00208C0A0020DD
:103AB000880A002080B584B000AF78603960124B6E
:103AC0001B6818337868194600F088FE0E4B1B6897
:103AD0000433184600F0BAFE3B68B3F1FF3F07D14C
:103AE000094B1B6804330948194600F04FFE07E0F4
:103AF000074B1A683B681344FB60F86800F0A2F9B2
:103B00001037BD4680BD00BF880A0020D80B0020BA
:103B1000F00B002080B584B000AF786039600C4BAA
:103B20001B6818337868194600F030FE084B1B6894
:103B30000433184600F08AFE064B1A683B681344AB
:103B4000FB60F86800F07EF91037BD4680BD00BF0D
:103B5000880A0020F00B002080B584B000AF7860A8
:103B60007B68DB68DB68BB60BB681833184600F015
:103B70006DFE1C4B1B68002B1DD1BB68043318461F
:103B800000F064FEBB68DA6A174B1B689A4203D9DF
:103B9000BB68DA6A144B1A60BB68DA6A13469B008A
:103BA00013449B00114A1A44BB680433104619465B
:103BB00000F0ECFD05E0BB6818330D48194600F035
:103BC000E5FDBB68DA6A0B4B1B68DB6A9A4202D3DD
:103BD0000123FB6001E00023FB60FB6818461037FF
:103BE000BD4680BD000C0020F80B00208C0A002090
:103BF000AC0B0020880A002080B483B000AF78604E
:103C0000064B1A687B681A60054B1A687B685A6015
:103C10000C37BD465DF8047B704700BF0C0C0020DC
:103C2000F00B002080B584B000AF7860396001F0FF
:103C300023FC3B681B68B3F1FF3F02D10023FB600C
:103C400029E07B681A68174B1B689A4208D07B688A
:103C50005A68154B1B689A4202D80123FB601AE090
:103C6000114B1A687B685B68D21A3B681B689A42E2
:103C70000FD23B681A687B6859680B4B1B68CB1ADC
:103C80001A443B681A607868FFF7B6FF0023FB60B0
:103C900001E00123FB6001F001FCFB6818461037CE
:103CA000BD4680BD0C0C0020F00B002080B400AF9E
:103CB000034B01221A60BD465DF8047B704700BFCC
:103CC000080C002080B582B000AF786000F080F86A
:103CD000044B1B68012B01D901F0C2FB03F030FD3E
:103CE000F4E700BF8C0A002080B584B000AFF86014
:103CF000B9607A603B60FB6834331846B9681022BB
:103D00001BF0A0FBFB68002283F843207B680B2B91
:103D100001D90B237B60FB687A68DA62FB687A68FA
:103D2000DA64FB680433184600F024FDFB6818339E
:103D3000184600F01FFDFB68FA681A617B68C3F142
:103D40000C02FB689A61FB68FA685A621037BD463C
:103D500080BD00BF80B582B000AF00237B600CE067
:103D60007A6813469B0013449B00114A134418467B
:103D700000F0E0FC7B6801337B607B680B2BEFD9A4
:103D80000C4800F0D7FC0C4800F0D4FC0B4800F0C5
:103D9000D1FC0B4800F0CEFC0A4800F0CBFC0A4BEB
:103DA000044A1A60094B044A1A600837BD4680BDB0
:103DB0008C0A00207C0B0020900B0020AC0B002014
:103DC000C00B0020D80B0020A40B0020A80B002063
:103DD00080B582B000AF184B1B68002B28D0FFF7CE
:103DE000E5FC164B1B68002B14BF00230123DBB23C
:103DF0007B60FFF7E9FC7B68002B19D101F03CFBED
:103E00000E4BDB68DB683B603B680433184600F010
:103E10001DFD0B4B1B685A1E094B1A60064B1B6895
:103E20005A1E054B1A6001F039FB386800F072F831
:103E30000837BD4680BD00BFD40B0020C00B00205A
:103E4000EC0B002080B582B000AF7860134B1B688C
:103E50007A685A60124B1B687A689A4209D2114BF1
:103E60001A680E4B1B6804331046194600F0B6FC66
:103E700010E00D4B1A68094B1B68043310461946B5
:103E800000F0ACFC094B1B687A689A4202D2074BDF
:103E90007A681A600837BD4680BD00BF880A0020D6
:103EA000F00B0020A80B0020A40B00201C00002019
:103EB00080B584B000AF03463960FB80502003F02A
:103EC00061FBF860FB68002B1FD03B68002B06D11C
:103ED000FB889B00184603F055FB034600E03B6857
:103EE000FA681363FB681B6B002B05D1F86803F0BD
:103EF000EFFB0023FB6008E0FB681A6BFB889B006C
:103F00001046A5211A461BF09FF9FB68184610378A
:103F1000BD4680BD80B582B000AF78607B681B6B0A
:103F2000184603F0D5FB786803F0D2FB0837BD468E
:103F300080BD00BF80B483B000AF054B1B687B60C1
:103F40007B6818460C37BD465DF8047B704700BFA0
:103F5000880A002080B483B000AF0B4B1B68002B95
:103F600002D100237B6008E0084B1B68002B02D1C4
:103F700001237B6001E002237B607B6818460C37DD
:103F8000BD465DF8047B7047FC0B0020000C002050
:103F900080B584B000AF78607B68FB60FB68DA6A4C
:103FA000214B1B68DB6A9A423AD21F4B1B68DB6AC3
:103FB000C3F10C02FB689A61FB685969FB68DA6A15
:103FC00013469B0013449B00184A1344994222D184
:103FD000FB680433184600F039FC134B1B68DA6A9F
:103FE000FB68DA62FB68DA6A114B1B689A4203D9F4
:103FF000FB68DA6A0E4B1A60FB68DA6A13469B00AC
:1040000013449B00094A1A44FB68043310461946BE
:1040100000F0BCFB04E0044B1B68DA6AFB68DA6260
:104020001037BD4680BD00BF880A00208C0A0020E2
:10403000F80B002080B584B000AF78607B68FB602F
:104040007B68002B2CD0FB68DA6AFB68DB6C9A4239
:1040500026D0FB680433184600F0F8FBFB68DA6CE6
:10406000FB68DA62FB68DB6AC3F10C02FB689A61E9
:10407000FB68DA6A0C4B1B689A4203D9FB68DA6A60
:10408000094B1A60FB68DA6A13469B0013449B00D5
:10409000064A1A44FB6804331046194600F076FBC2
:1040A0001037BD4680BD00BFF80B00208C0A0020F1
:1040B00080B500AFFFF702FC0346184680BD00BF85
:1040C00080B582B000AF78607B681846FFF714FBBC
:1040D0000837BD4680BD00BF80B400AFBD465DF867
:1040E000047B704780B500AF012000F067FE0246F8
:1040F0000B4B1A6001200021032200F023FE024630
:10410000084B1A60074B1B68002B07D0054B1B6838
:10411000184600210022002300F092FE80BD00BF5F
:10412000480C00204C0C002080B500AF044B1B68ED
:10413000184600210022002300F082FE80BD00BF4F
:10414000480C002080B500AF074B1B68002B01D145
:10415000FFF7C8FF044B1B68184600214FF0FF32E1
:10416000002300F033FF80BD480C002080B500AF75
:10417000FFF7E0FE0346184680BD00BF80B487B05D
:1041800000AF7860396000237B6100233B6100232E
:10419000FB6000237B6176E07B69012202FA03F376
:1041A0003B613B681A683B691340FB60FA683B69F6
:1041B0009A4265D17B681A687B695B00032101FA2A
:1041C00003F3DB431A407B681A607B681A683B681C
:1041D0001B7919467B695B0001FA03F31A437B687C
:1041E0001A603B681B79012B03D03B681B79022BBB
:1041F0002ED17B689A687B695B00032101FA03F387
:10420000DB431A407B689A607B689A683B685B79FD
:1042100019467B695B0001FA03F31A437B689A60D5
:104220007B685A687B699BB2012101FA03F3DB4387
:104230001A407B685A607B685A683B689B791946CC
:104240007B699BB201FA03F39BB21A437B685A6005
:104250007B68DA687B699BB25B00032101FA03F398
:10426000DB431A407B68DA607B68DA683B68DB799D
:1042700019467B695B0001FA03F31A437B68DA6035
:104280007B6901337B617B690F2B85D91C37BD4668
:104290005DF8047B704700BF80B483B000AF7860E6
:1042A0000B467B807B687A881A830C37BD465DF8A5
:1042B000047B704780B483B000AF78600B467B808E
:1042C0007B687A885A830C37BD465DF8047B70475B
:1042D00080B483B000AF786013460A467A807B7062
:1042E0007B78002B03D07B687A881A8302E07B6896
:1042F0007A885A830C37BD465DF8047B704700BF4F
:1043000080B485B000AF786013460A467A807B702F
:104310000023FB600023BB607A787B8803F00703EF
:104320009B0002FA03F3FB607B88DB089BB21A4612
:104330007B88DB089BB219467B68083153F8211053
:104340007B8803F007039B000F2000FA03F3DB4395
:1043500019407B68083243F822107B88DB089BB247
:104360001A467B68083253F82220FB681343BB606F
:104370007B88DB089BB21A467B680832B96843F831
:1043800022101437BD465DF8047B704780B592B0AB
:1043900000AF00F035F801200121FEF78BFB02236E
:1043A0003B6007237B600423BB600723FB60022381
:1043B0003B6102237B610223BB610123FB6100237C
:1043C0003B6204237B621023BB624023FB624FF4F9
:1043D000C0733B6300237B634FF40063BB63002324
:1043E000FB634FF400533B643B467B6407F11C03C3
:1043F000184600F03BFB00F00DF94837BD4680BD84
:1044000080B582B000AF7E200121FEF735FB02238C
:104410003B7102237B710023BB710023FB71774842
:1044200005210C22FFF76CFF744806210C22FFF7D0
:1044300067FF60233B603B4670481946FFF79EFECE
:104440006F4800210C22FFF75BFF01233B603B46D6
:104450006B481946FFF792FE6A4800210C22FFF7CD
:104460004FFF684801210C22FFF74AFF65480821E9
:104470000C22FFF745FF634809210C22FFF740FF9C
:1044800060480A210C22FFF73BFF5E480E210C22F8
:10449000FFF736FF5B480F210C22FFF731FF4CF28C
:1044A00003733B603B4657481946FFF767FE564883
:1044B00000210C22FFF724FF534801210C22FFF7B3
:1044C0001FFF514807210C22FFF71AFF4E48082111
:1044D0000C22FFF715FF4C4809210C22FFF710FFB3
:1044E00049480A210C22FFF70BFF47480B210C22F9
:1044F000FFF706FF44480C210C22FFF701FF42485A
:104500000D210C22FFF7FCFE3F480E210C22FFF785
:10451000F7FE3D480F210C22FFF7F2FE4FF68373A2
:104520003B603B4638481946FFF728FE37480021D4
:104530000C22FFF7E5FE354801210C22FFF7E0FED3
:10454000324802210C22FFF7DBFE304803210C2207
:10455000FFF7D6FE2D4804210C22FFF7D1FE2B4891
:1045600005210C22FFF7CCFE28480B210C22FFF777
:10457000C7FE26480C210C22FFF7C2FE23480D215E
:104580000C22FFF7BDFE21480E210C22FFF7B8FEDA
:104590001E480F210C22FFF7B3FE4FF63F033B608E
:1045A0003B461A481946FFF7E9FD194800210C223D
:1045B000FFF7A6FE164801210C22FFF7A1FE1448C2
:1045C00004210C22FFF79CFE114805210C22FFF765
:1045D00097FE0F4808210C22FFF792FE0C480F218E
:1045E0000C22FFF78DFE48F233133B603B46084830
:1045F0001946FFF7C3FD0837BD4680BD00040240E1
:1046000000080240000C024000100240001402406A
:104610000018024080B586B000AF00237B61012303
:104620007B600823BB600123FB6000233B6100BF6C
:104630000120202100F0FAFA0346002BF8D13B1D9F
:10464000184600F0C1FA0A2000F05AF802237B60F5
:104650000823BB600123FB6000233B6100BF0120F6
:10466000202100F0E3FA0346002BF8D13B1D184649
:1046700000F0AAFA03237B600823BB600423FB60DD
:1046800000233B6100BF0120202100F0CFFA034648
:10469000002BF8D13B1D184600F096FA00BF012010
:1046A000202100F0C3FA0346002BF8D13B1D184629
:1046B00000F08AFA40F231237B6104237B600823F7
:1046C000BB600123FB607B693B6100BF01202021AF
:1046D00000F0ACFA0346002BF8D13B1D184600F061
:1046E00073FA40F2AB2000F08FFA00BF01202021C6
:1046F00000F09CFA0346002BF8D11837BD4680BD68
:1047000080B485B000AF78600023FB607B68084A06
:1047100002FB03F3FB6002E0FB68013BFB60FB680C
:10472000002BF9D11437BD465DF8047B704700BFFC
:10473000A086010080B483B000AF78607B6803F18D
:1047400008027B685A607B684FF0FF329A607B6892
:1047500003F108027B68DA607B6803F108027B687A
:104760001A617B6800221A600C37BD465DF8047B35
:10477000704700BF80B483B000AF78607B680022D0
:104780001A610C37BD465DF8047B704780B485B074
:1047900000AF786039607B685B68FB60FB685A68D3
:1047A0003B685A607B685A683B689A60FB685B6844
:1047B0003A689A60FB683A685A607B683A685A605F
:1047C0003B687A681A617B681B685A1C7B681A60B0
:1047D0001437BD465DF8047B704700BF80B485B0D8
:1047E00000AF786039603B681B68BB60BB68B3F1A1
:1047F000FF3F03D17B681B69FB600CE07B680833DB
:10480000FB6002E0FB685B68FB60FB685B681A6842
:10481000BB689A42F6D9FB685A683B685A603B68A5
:104820005B683A689A603B68FA689A60FB683A6825
:104830005A603B687A681A617B681B685A1C7B68FF
:104840001A601437BD465DF8047B704780B485B0AC
:1048500000AF78607B685B687A6892689A607B6872
:104860009B687A6852685A607B681B69FB60FB68CA
:104870005A687B689A4203D17B689A68FB685A60E1
:104880007B6800221A61FB681B685A1EFB681A606D
:104890001437BD465DF8047B704700BF80B500AF9C
:1048A000154B154AD2F8882042F47002C3F88820CC
:1048B000124B124A126842F001021A600F4B00229A
:1048C0009A600E4A0D4B1B6823F0847323F48033E7
:1048D00013600A4B0A4A5A60084B084A126822F4CD
:1048E00080221A60054B0022DA6000F00BF8024BC0
:1048F0004FF000629A6080BD00ED00E00038024099
:104900001030002480B483B000AF00237B6000230C
:104910003B60424B414A126842F480321A603F4B7E
:104920001B6803F400333B607B6801337B603B68AA
:10493000002B03D17B68B3F5A04FF0D1374B1B6838
:1049400003F40033002B02D001233B6001E000237D
:104950003B603B68012B02D1304B314A5A602F4BF0
:104960002E4A126C42F080521A642E4B2D4A126865
:1049700042F440421A60294B284A92689A60274BB9
:10498000264A926842F400429A60244B234A926875
:1049900042F4A0529A60214B204A126842F0807281
:1049A0001A6000BF1D4B1B6803F00073002BF9D089
:1049B0001C4B1C4A126842F480321A6000BF194B2B
:1049C0005B6803F48033002BF9D0164B154A12684C
:1049D00042F400321A6000BF124B5B6803F40033EC
:1049E000002BF9D0104B40F205721A600B4B0B4AAA
:1049F000926822F003029A60084B084A926842F0DB
:104A000002029A6000BF054B9B6803F00C03082B61
:104A1000F9D10C37BD465DF8047B70470038024081
:104A2000085A400700700040003C024080B485B046
:104A300000AF78600B4B1B68002B02D1094B0A4A70
:104A40001A60084B1B68FB60064B1A687B681A44A7
:104A5000044B1A60FB6818461437BD465DF8047BAA
:104A6000704700BF500C00202881022080B487B01E
:104A700000AF786000237B6100233B610023FB6073
:104A80000023BB607B685A687B689B681A437B681D
:104A9000DB681A437B681B691A437B685B691A43AE
:104AA0007B689B691A437B68DB691A437B681B6AD6
:104AB0001A437B685B6A13437B617B681B68002B2E
:104AC00006D1404B7A681268796943F8221011E0E8
:104AD0007B68DA697B681B6A1A437B685B6A1343ED
:104AE000FB60384BFA681A60364B7A68126879694D
:104AF00043F822107B681B68002B30D17B689B6ACF
:104B00001B685A1E7B689B6A5B68013B1B011A434A
:104B10007B689B6A9B68013B1B021A437B689B6A0C
:104B2000DB68013B1B031A437B689B6A1B69013BE3
:104B30001B041A437B689B6A5B69013B1B051A4394
:104B40007B689B6A9B69013B1B0613433B611D4BC2
:104B50007A6812680232396943F822102CE07B68C7
:104B60009B6A1B685A1E7B689B6A5B68013B1B0142
:104B70001A437B689B6A9B68013B1B021A437B6854
:104B80009B6A1B69013B1B0413433B617B689B6A67
:104B9000DB68013B1A037B689B6A5B69013B1B0571
:104BA0001343BB60074BBA689A60064B7A68126879
:104BB0000232396943F822101C37BD465DF8047B88
:104BC000704700BF400100A080B485B000AF78609E
:104BD0000023FB607B681A687B685B681A437B680C
:104BE0009B68013B5B011A437B68DB685B021343F4
:104BF000FB60044BFA681A611437BD465DF8047B0C
:104C0000704700BF400100A080B483B000AF78605F
:104C1000054B054A51697A6852000A435A610C37BC
:104C2000BD465DF8047B7047400100A080B485B0AC
:104C300000AF786039600023FB730023BB607B68A2
:104C4000102B03D1144B5B68BB6012E07B68B3F59B
:104C5000807F03D1114B5B68BB600AE07B68B3F5D2
:104C6000805F03D10E4B5B68BB6002E00D4B9B691C
:104C7000BB60BA683B681A403B689A4202D0002386
:104C8000FB7301E00123FB73FB7B18461437BD4621
:104C90005DF8047B704700BF600000A0800000A0AA
:104CA000A00000A0400100A080B584B000AF7860F3
:104CB00039600123FB603B68012B0BD07B685B6A8A
:104CC000002B01D00023FB607B681B69002B01D007
:104CD0000023FB60FB68012B2FD17B681A687B687F
:104CE000DB6B7968096C01FB03F31A447B685A603B
:104CF0007B6800229A637B681A687B689A607B688D
:104D00001A687B68DB6B013B7968096C01FB03F374
:104D10001A447B68DA607B684FF0FF325A647B6824
:104D20004FF0FF329A647B6810331846FFF702FD9C
:104D30007B6824331846FFF7FDFCFB6818461037E4
:104D4000BD4680BD80B588B000AFF860B96013463D
:104D5000FB710023FB61FB68002B2AD0502002F07E
:104D600011FCB861BB69002B23D0FB68BA6802FB59
:104D700003F301337B61786902F004FC0246BB69EE
:104D80001A60BB691B68002B10D0BB69FA68DA6334
:104D9000BB69BA681A64B8690121FFF785FFBB696E
:104DA000FA7983F84D20BB69FB6102E0B86902F033
:104DB0008FFCFB6918462037BD4680BD80B584B0A6
:104DC00000AF0346FB71502002F0DCFBF860FB688B
:104DD000002B30D0FB6800225A60FB6800221A606A
:104DE000FB6800229A60FB680022DA60FB68002200
:104DF0009A63FB680122DA63FB6800221A64FB688D
:104E00004FF0FF325A64FB684FF0FF329A64FB6840
:104E1000FA7983F84D20FB6810331846FFF78AFCB7
:104E2000FB6824331846FFF785FCF8680021002250
:104E3000002300F005F8FB6818461037BD4680BD1A
:104E400080B588B000AFF860B9607A603B6000233D
:104E5000FB6100F011FBFB689A6BFB68DB6B9A420D
:104E600016D2F868B9683A6800F066F9FB685B6AC0
:104E7000002B09D0FB6824331846FEF76DFE03466D
:104E8000012B01D100F0ECFA00F008FB012359E0FE
:104E90007B68002B03D100F001FB002352E0FB698B
:104EA000002B06D107F114031846FEF7A5FE0123D7
:104EB000FB6100F0F3FAFEF779FC00F0DDFAFB6825
:104EC0005B6CB3F1FF3F02D1FB6800225A64FB68C0
:104ED0009B6CB3F1FF3F02D1FB6800229A6400F0A3
:104EE000DDFA07F114023B1D10461946FEF79AFE43
:104EF0000346002B1ED1F86800F002FA0346002B8F
:104F000012D0FB6803F110027B6810461946FEF7C9
:104F1000D1FDF86800F092F9FEF756FC0346002B2D
:104F20000FD100F09DFA0CE0F86800F087F9FEF769
:104F30004BFC8EE7F86800F081F9FEF745FC002392
:104F400000E086E718462037BD4680BD80B586B0B4
:104F500000AFF860B9607A603B6000233B614FF0BE
:104F6000500080F31188FB689A6BFB68DB6B9A42F8
:104F700021D2F868B9683A6800F0DEF8FB689B6CEB
:104F8000B3F1FF3F0FD1FB685B6A002B10D0FB68C9
:104F900024331846FEF7E0FD0346002B08D07B685B
:104FA00001221A6004E0FB689B6C5A1CFB689A643F
:104FB00001237B6101E000237B614FF0000080F35F
:104FC00011887B6918461837BD4680BD80B588B00A
:104FD00000AFF860B9607A603B600023FB6100F0CD
:104FE0004BFAFB689B6B002B3BD0FB68DB68BB611B
:104FF000F868B96800F0FCF83B68002B1CD1FB682E
:105000009B6B5A1EFB689A63FB681B68002B04D1DC
:10501000FEF790FF0246FB685A60FB681B69002B95
:105020001BD0FB6810331846FEF796FD0346012B94
:1050300013D100F015FA10E0FB68BA69DA60FB687A
:105040005B6A002B09D0FB6824331846FEF784FD09
:105050000346002B01D000F003FA00F01FFA0123F1
:1050600066E07B68002B03D100F018FA00235FE0B4
:10507000FB69002B06D107F110031846FEF7BCFDB3
:105080000123FB6100F00AFAFEF790FB00F0F4F94F
:10509000FB685B6CB3F1FF3F02D1FB6800225A64EE
:1050A000FB689B6CB3F1FF3F02D1FB6800229A645E
:1050B00000F0F4F907F110023B1D10461946FEF707
:1050C000B1FD0346002B2BD1F86800F003F903462D
:1050D000002B1FD0FB681B68002B08D100F0CCF917
:1050E000FB685B681846FEF753FF00F0D7F9FB68D2
:1050F00003F124027B6810461946FEF7DBFCF868D2
:1051000000F09CF8FEF760FB0346002B0FD100F087
:10511000A7F90CE0F86800F091F8FEF755FB5EE7A0
:10512000F86800F08BF8FEF74FFB002300E056E72D
:1051300018462037BD4680BD80B584B000AFF8600A
:10514000B9607A60FB681B6C002B0CD1FB681B6894
:10515000002B45D1FB685B681846FEF76BFFFB68C8
:1051600000225A603CE07B68002B1AD1FB689A68E9
:10517000FB681B6C1046B9681A46FBF7E3FCFB683A
:105180009A68FB681B6C1A44FB689A60FB689A6813
:10519000FB685B689A4223D3FB681A68FB689A60D5
:1051A0001EE0FB68DA68FB681B6C1046B9681A469B
:1051B000FBF7C8FCFB68DA68FB681B6C5B421A44AF
:1051C000FB68DA60FB68DA68FB681B689A4207D202
:1051D000FB685A68FB681B6C5B421A44FB68DA6028
:1051E000FB689B6B5A1CFB689A631037BD4680BDF9
:1051F00080B582B000AF786039607B681B68002B97
:1052000019D07B68DA687B681B6C1A447B68DA60AB
:105210007B68DA687B685B689A4203D37B681A68AC
:105220007B68DA607B68DA687B681B6C38681146DB
:105230001A46FBF787FC0837BD4680BD80B582B0B3
:1052400000AF786000F018F914E07B685B6A002B0F
:105250000FD07B6824331846FEF77EFC0346002BF4
:1052600001D0FEF723FD7B689B6C5A1E7B689A6415
:1052700000E003E07B689B6C002BE6DC7B684FF072
:10528000FF329A6400F00AF900F0F6F814E07B6847
:105290001B69002B0FD07B6810331846FEF75CFCAF
:1052A0000346002B01D0FEF701FD7B685B6C5A1EA4
:1052B0007B685A6400E003E07B685B6C002BE6DCF3
:1052C0007B684FF0FF325A6400F0E8F80837BD46BB
:1052D00080BD00BF80B584B000AF786000F0CCF82E
:1052E0007B689B6B002B14BF00230123DBB2FB60A8
:1052F00000F0D4F8FB6818461037BD4680BD00BFEB
:1053000080B584B000AF786000F0B6F87B689A6B27
:105310007B68DB6B9A4214BF00230123DBB2FB6086
:1053200000F0BCF8FB6818461037BD4680BD00BFD2
:1053300080B582B000AF7860396000F09DF87B687E
:105340005B6CB3F1FF3F02D17B6800225A647B683B
:105350009B6CB3F1FF3F02D17B6800229A6400F09E
:105360009DF87B689B6B002B05D17B682433184626
:105370003968FEF7CFFB7868FFF760FF0837BD4656
:1053800080BD00BF80B485B000AFF860B9607A60BE
:10539000FB68043BFB60FB684FF080721A60FB689F
:1053A000043BFB60BA68FB681A60FB68043BFB6067
:1053B000FB6800221A60FB68143BFB607A68FB689C
:1053C0001A60FB68043BFB60FB686FF002021A6026
:1053D000FB68203BFB60FB6818461437BD465DF850
:1053E000047B7047054B19680868B0E8F04F80F3FC
:1053F00009884FF0000080F311887047880A002068
:1054000003480068006880F3088862B600DF00BFC8
:1054100008ED00E080B500AF0E4B0E4A126842F472
:1054200070021A600B4B0B4A126842F070421A600D
:1054300000F08AF8084B00221A6000F097F8074B3A
:10544000064A126842F040421A60FFF7D9FF002373
:10545000184680BD20ED00E03400002034EF00E06D
:1054600080B400AF034B4FF080521A60BD465DF828
:10547000047B704704ED00E080B400AF4FF05000B3
:1054800080F31188044B1B685A1C034B1A60BD46FD
:105490005DF8047B704700BF3400002080B400AF8B
:1054A000084B1B685A1E074B1A60064B1B68002BE3
:1054B00003D14FF0000080F31188BD465DF8047BF6
:1054C000704700BF34000020EFF30980114B1A68C9
:1054D0001EF0100F08BF20ED108A20E9F04F106079
:1054E0002DE908404FF0500080F31188FEF796FA3E
:1054F0004FF0000080F31188BDE808401968086883
:10550000B0E8F04F1EF0100F08BFB0EC108A80F327
:1055100009887047880A002080B582B000AF094B27
:105520004FF080521A6000237B604FF0500080F3F0
:105530001188FEF7D5F94FF0000080F31188083785
:10554000BD4680BD04ED00E080B400AF044B054AC9
:105550001A60054B07221A60BD465DF8047B704750
:1055600014E000E01FBF020010E000E0DFF80C00D4
:10557000016841F4700101607047000088ED00E0AF
:10558000002100F004B80C4B5B58435004310B4829
:105590000B4B42189A42FFF4F6AF0A4A00F003B8E8
:1055A000002342F8043B084B9A42FFF4F9AFFFF79F
:1055B00075F9FCF76FFE7047C47602080000002002
:1055C0002C0A0020300A002028810220FFF7FEBFAD
:1055D00080B582B000AF78607A682D4B9A420AD1CC
:1055E0004FF480500121FDF7DDFA4FF48050002187
:1055F000FDF7D8FA49E07A68264B9A420AD14FF46F
:1056000080400121FDF7B0FA4FF480400021FDF702
:10561000ABFA3AE07A68204B9A420AD14FF4004044
:105620000121FDF7A1FA4FF400400021FDF79CFA9B
:105630002BE07A68194B9A420AD14FF400500121AD
:10564000FDF7B0FA4FF400500021FDF7ABFA1CE073
:105650007A68134B9A420AD14FF480100121FDF76A
:10566000A1FA4FF480100021FDF79CFA0DE07A6852
:105670000C4B9A4209D14FF400100121FDF792FA28
:105680004FF400100021FDF78DFA0837BD4680BDAC
:105690000030014000380040003C00400034014030
:1056A000005001400054014080B485B000AF7860E4
:1056B00039600023FB817B681B88FB81FB8903F435
:1056C0004153FB813B681A883B685B8813439AB25D
:1056D0003B689B8813439AB23B68DB8813439AB2BA
:1056E0003B681B8913439AB23B685B8913439AB2A8
:1056F0003B689B8913439AB23B68DB8913439AB298
:10570000FB891343FB817B68FA891A807B689B8B3A
:105710009BB223F400639AB27B689A833B681A8A2F
:105720007B681A821437BD465DF8047B704700BF62
:1057300080B483B000AF78600B46FB70FB78002B21
:1057400008D07B681B889BB243F040039AB27B6809
:105750001A8007E07B681B889BB223F040039AB253
:105760007B681A800C37BD465DF8047B704700BF2C
:1057700080B483B000AF78600B467B807B687A880A
:105780009A810C37BD465DF8047B704780B485B0C4
:1057900000AF78600B467B800023FB737B681B891E
:1057A0009AB27B8813409BB2002B02D00123FB737B
:1057B00001E00023FB73FB7B18461437BD465DF800
:1057C000047B704780B500AF002001F09BFA0120F8
:1057D00001F098FA00F00EF8FEF7D8FDFCF79EFAFB
:1057E00000F04CF84FF480500121FDF745F90023FB
:1057F000184680BD80B500AF72B6FBF751FD62B6AA
:105800000023184680BD00BF80B584B000AFFFF70D
:1058100033FEFBF75DFDF860FFF740FE154B1B689C
:10582000002B06D1FB685B883B60FB689B887B6034
:1058300007E0FB685B887B60FB689B88C3F5A0730F
:105840003B60FB681B88802B14BF00230123DBB265
:105850003B723A7A084B1B789A4208D03A7A064B48
:105860001A7000237B723B4618460EF0ABFC1037D3
:10587000BD4680BD540C0020580C002080B584B07B
:1058800000AF72B64FF4003001F0AEF84FF40033C1
:105890007B6000233B7208237B720123BB723B1D9C
:1058A000184601F033F829233B7300237B73002350
:1058B000BB730123FB7307F10C03184601F0B4F826
:1058C00062B61037BD4680BD80B582B000AF78604B
:1058D0007A68174B9A420AD14FF400100121FDF764
:1058E00043F94FF400100021FDF73EF91CE07A68FF
:1058F000104B9A420AD14FF480000121FDF734F990
:105900004FF480000021FDF72FF90DE07A680A4B73
:105910009A4209D14FF400000121FDF725F94FF417
:1059200000000021FDF720F90837BD4680BD00BF0B
:105930000054004000580040005C004080B58AB030
:1059400000AF786039600023FB8400237B8404234C
:10595000BB84574BFB617B689B88FB84FB8C23F0EB
:105960003F03FB8407F10C031846FCF77FFF7B69BC
:10597000FB61FA694F4BA3FB02139B0C7B84FA8CEF
:105980007B8C1343FB847B68FA8C9A807B681B8832
:105990009BB223F001039AB27B681A800023FB8438
:1059A0003B681A68444B9A4215D83B681B685B00F9
:1059B000FA69B2FBF3F3BB84BB8C032B01D804233D
:1059C000BB84FA8CBB8C1343FB847B8C01339AB26F
:1059D0007B681A8440E03B68DA884BF6FF739A4292
:1059E00009D13B681A6813465B001344FA69B2FB9D
:1059F000F3F3BB840EE03B681A6813469B00134424
:105A00009A001344FA69B2FBF3F3BB84BB8C43F4F2
:105A10008043BB84BB8CC3F30B03002B03D1BB8C33
:105A200043F00103BB84BA8CFB8C13439BB26FEA37
:105A300043436FEA5343FB847B8C4FF4967202FB23
:105A400003F31E4A82FB03129211DB17D31A9BB297
:105A500001339AB27B681A847B68FA8C9A837B68DC
:105A60001B889BB243F001039AB27B681A807B6863
:105A70001B88FB84FB8C23F4816323F00203FB84EB
:105A80003B689A883B685B8913439AB2FB8C13434B
:105A9000FB847B68FA8C1A803B689A893B681B8977
:105AA00013439AB27B681A812837BD4680BD00BF78
:105AB00000127A0083DE1B43A0860100D34D6210E2
:105AC00080B483B000AF78600B46FB70FB78002B8E
:105AD00008D07B681B889BB243F001039AB27B68B5
:105AE0001A8007E07B681B889BB223F001039AB2FF
:105AF0007B681A800C37BD465DF8047B704700BF99
:105B000080B483B000AF78600B46FB70FB78002B4D
:105B100008D07B681B889BB243F480739AB27B6881
:105B20001A8007E07B681B889BB223F480739AB2CB
:105B30007B681A800C37BD465DF8047B704700BF58
:105B400080B483B000AF78600B46FB70FB78002B0D
:105B500008D07B681B889BB243F400739AB27B68C1
:105B60001A8007E07B681B889BB223F400739AB20B
:105B70007B681A800C37BD465DF8047B704700BF18
:105B800080B483B000AF786013460A46FA70BB70E9
:105B9000BB78002B04D0FB7843F00103FB7003E0DB
:105BA000FB7823F00103FB70FB789AB27B681A82C2
:105BB0000C37BD465DF8047B704700BF80B483B0EE
:105BC00000AF78600B46FB70FB78002B08D07B6839
:105BD0001B889BB243F480639AB27B681A8007E00B
:105BE0007B681B889BB223F480639AB27B681A801F
:105BF0000C37BD465DF8047B704700BF80B483B0AE
:105C000000AF78600B46FB70FB78002B0AD07B68F6
:105C10001B889BB26FEA43436FEA53439AB27B6897
:105C20001A8007E07B681B889BB2C3F30E039AB20D
:105C30007B681A800C37BD465DF8047B704700BF57
:105C400080B483B000AF78600B467B807B88B3F56F
:105C5000006F08D17B681B889BB243F400639AB243
:105C60007B681A8007E07B681B889BB223F4006383
:105C70009AB27B681A800C37BD465DF8047B70478A
:105C800080B483B000AF78600B46FB70FB789AB2AB
:105C90007B681A820C37BD465DF8047B704700BFF5
:105CA00080B483B000AF78607B681B8A9BB2DBB2A4
:105CB00018460C37BD465DF8047B704780B487B04A
:105CC00000AF786039600023FB7500233B6100233F
:105CD000FB607B68FB603B681B0F3B613B6823F00C
:105CE0007F433B603B69002B03D0FB681433FB60B0
:105CF00005E03B681B0C3B60FB681833FB60FB68EE
:105D00001A683B681340002B02D00123FB7501E0A9
:105D10000023FB75FB7D18461C37BD465DF8047BF0
:105D2000704700BF80B483B000AF0346FB71084BDF
:105D300097F907205209F97901F01F01012000FAB3
:105D400001F143F822100C37BD465DF8047B704723
:105D500000E100E080B483B000AF03463960FB711E
:105D600097F90730002B0BDA0D49FB7903F00F038D
:105D7000043B3A68D2B21201D2B20B441A7609E05F
:105D8000084997F907303A68D2B21201D2B20B44EF
:105D900083F800230C37BD465DF8047B704700BFD5
:105DA00000ED00E000E100E080B485B000AF786075
:105DB0007B68002B01D0002335E01E4B7A6853F836
:105DC0002230FB60FA681C4B9A4201D100232AE082
:105DD000FA681A4B9A4201D1012324E0FA68184B61
:105DE0009A4201D102231EE0FA68164B9A4201D171
:105DF000032318E0FA68144B9A4201D1042312E0FD
:105E0000FA68124B9A4201D105230CE0FA68104B54
:105E10009A4201D1062306E0FA680E4B9A4201D15C
:105E2000072300E0FEE718461437BD465DF8047B03
:105E3000704700BF40000020986A0208686A0208A4
:105E4000B06A0208E06A0208C86A0208106B020819
:105E5000286B0208F86A020880B584B000AF786049
:105E6000396078680BF076FCF860FB683A6802FBF2
:105E700003F30733002B00DA0733DB10BB60BB688A
:105E800018461037BD4680BD80B483B000AF78603F
:105E900039603B68002B06D07B681B6843F0020228
:105EA0007B681A6005E07B681B6823F002027B6850
:105EB0001A60044B02225A620C37BD465DF8047B1F
:105EC000704700BF0068014080B483B000AF7860C5
:105ED00039603B68002B06D07B681B6843F01002DA
:105EE0007B681A6005E07B681B6823F010027B6802
:105EF0001A60044B02225A620C37BD465DF8047BDF
:105F0000704700BF0068014080B58AB000AFF860FC
:105F1000B9607A60F8680BF0E5FB7862F8680BF01E
:105F2000EFFB3862BB681E33FB61BB6803F11D02E7
:105F30007B6A1344BB617B6804337B617B68DA1C3A
:105F40003B6A13443B61184BFA6853F82230164AF7
:105F5000F96852F82120526802F470425A60124BDC
:105F6000FA6853F82230BA691104FA690A435A6090
:105F70000D4BFA6853F822300B4AF96852F8212089
:105F8000926802F470429A60074BFA6853F8223024
:105F90003A6911047A690A439A600220FCF74CF8C6
:105FA0002837BD4680BD00BF3800002080B582B0D4
:105FB00000AF786039600D4B7A6853F822300B4A95
:105FC000796852F82120526922F0FF025A61074B8A
:105FD0007A6853F822303A68C2F1FF025A61012010
:105FE000FCF72AF80837BD4680BD00BF3800002006
:105FF00080B588B000AFF860B9607A60BB68DBB28A
:106000001B04FB61BB6803F47F43BB61BB681B0CD3
:10601000DBB27B617B681B063B610E4BFA6853F871
:1060200022301B6C0B4BFA6853F8223000221A64A2
:10603000084BFA6853F82230F969BA6911437A6952
:1060400011433A690A431A640120FBF7F5FF203730
:10605000BD4680BD3800002080B586B000AFF86036
:10606000B9607A603B60F868FFF79EFE7861154B77
:106070004FF400721A60134BBA68DA60114B7A68F9
:10608000DA63104B7A6A1A610E4B7A6A1A640D4B06
:106090007A69DA610B4B3A68120411463A6A92B295
:1060A0000A435A64074B074A126842F001021A6019
:1060B00000BF044B1B6803F00103002BF9D1183714
:1060C000BD4680BD00B0024080B586B000AFF8602C
:1060D000B9607A603B60F868FFF766FE7861134B41
:1060E000134A1A60114B7A6A9A63104BBA68DA63E2
:1060F0000E4B3A6A1A640D4B7A695A630B4B7A68F5
:10610000120411463A6892B20A435A64074B074A8E
:10611000126842F001021A6000BF044B1B6803F0D2
:106120000103002BF9D11837BD4680BD00B00240F5
:106130000002030080B500AF01F0B4F80120FBF7C6
:106140005FFF80BD80B592B000AF786007F10802B4
:106150004023104600211A4619F076F87B68012B7F
:1061600000F2C180614B1B68002B1ED15F4B0122E6
:106170001A6000F075FE01200121FCF721F858207B
:106180000021FFF7E7FD5820FFF7CCFD4FF400702A
:106190000121FBF795FD5A200021FFF7DBFD5A2076
:1061A000FFF7C0FD524B02229A6078680BF09AFA12
:1061B0000246504B1A6078680BF0A2FA02464E4B2A
:1061C0001A601E23BB604B4B1B681D33FB6004230E
:1061D0003B61494B1B6803337B617868FFF7E4FD43
:1061E0000246464B1A60454B1B68BB61FF23FB61AF
:1061F00000233B6200237B620023BB620023FB621F
:106200003C4B1B6878681946FFF726FE02463C4B5C
:106210001A604FF480633B6305237B63384B1B6834
:106220000333FB63364B1B683B64334B1B687B6457
:10623000344B7A6853F82230BB63334B7A6853F897
:10624000222007F1080310461946FBF703FF786880
:106250000BF080FA02462D4B1A602C4B1B68082B62
:1062600008DC294B7A6853F8223018460121FFF7E1
:106270002BFE2DE0264B7A6853F82220254B9A42BC
:1062800026D1214B7A6853F8223018460121FFF7B6
:106290001BFE214B00221A6016E0204B5B681E4A51
:1062A00012681046984702461D4B1A601C4B1A682C
:1062B000194B1B68786811461A46FFF799FE164B72
:1062C0001B685A1C144B1A60134B1B68FF2BE4DD30
:1062D0000D4B7A6853F8223018460121FBF754FF22
:1062E0000120FBF7A9FE4837BD4680BD700C002099
:1062F00000B00240740C0020780C00207C0C0020C0
:10630000800C0020682D020838000020840C00203A
:1063100040000020F86A0208880C0020106B020878
:106320008C0C002080B485B000AF78600B4B7A688D
:1063300053F822300A4A796852F8212002FB03F30D
:10634000084A796852F8212002FB03F3FB60FB68DE
:1063500018461437BD465DF8047B7047640C002076
:10636000680C00206C0C002090B58BB002AFF86078
:10637000B9607A60F868FFF7D5FFF861134BFA68E7
:1063800053F82220BB68F96901FB03F31344BB6196
:106390000E4BFA6853F822207B68F96901FB03F37E
:1063A00013447B61B9697A69094BF86853F8203066
:1063B0000848FC6850F82400009000200190F8681C
:1063C000FFF74AFE2437BD4690BD00BF682D020886
:1063D000640C0020680C002080B58AB002AFF86021
:1063E000B9607A603B60F868FFF79CFFF861284B62
:1063F000FA6853F82220274BF96853F8213079685E
:1064000001FB03F1BB680B442349F86851F82010E5
:1064100001FB03F31946214BF86853F82030F86963
:1064200000FB03F30B441344BB61194BFA6853F8A8
:106430002220184BF96853F82130B96A01FB03F1A7
:106440003B680B441449F86851F8201001FB03F332
:106450001946124BF86853F82030F86900FB03F333
:106460000B4413447B61BA697B690A49F86851F8A7
:106470002000F96A411A386B00900191F8681146C2
:106480001A46FB6AFFF7E8FD2037BD4680BD00BF16
:10649000682D0208640C00206C0C0020600C0020A9
:1064A00080B58AB002AFF860B9607A603B600EF0E8
:1064B0002BF90346012B10D1F868192100220AF0AC
:1064C00075FAB86879683A68BB6A0BF023FCF8681B
:1064D0001921214A0AF06AFA3BE03A68BB68D31AEC
:1064E0000133FB61BA6A7B68D31A0133BB61F86878
:1064F000FFF718FF7861194BFA6853F82220184B00
:10650000F96853F82130796801FB03F1BB680B444B
:106510001449F86851F8201001FB03F31946124B97
:10652000F86853F82030786900FB03F30B441344F8
:106530003B613B690A4AF96852F82110FA698A1AE4
:106540000092FA6A0192F8681946FA69BB69FFF786
:10655000BBFD2037BD4680BDA1640008682D020840
:10656000640C00206C0C0020600C002080B400AF94
:10657000034B02229A60BD465DF8047B704700BF62
:1065800000B0024080B582B000AF2D4B0122DA632B
:1065900000237B604EE02B4B7A6853F82230002BAF
:1065A00045DB294B7A6853F82220284B796853F849
:1065B00021302749786851F8201001FB03F3214965
:1065C000786851F8201001FB03F32249786851F8EC
:1065D000201001FB03F313443B601F4B7A6853F810
:1065E00022309B6A1C4B7A6853F8223000229A6250
:1065F000194B7A6853F822303A689A620120FBF707
:106600001BFD104B7A6853F82230786819460EF05B
:106610001DF80C4B7A6853F82210104B7A6843F837
:106620002210084B7A684FF0FF3143F822107B6844
:1066300001337B607B68002BADDD0837BD4680BD34
:10664000006801405C0C0020682D0208640C0020EA
:10665000680C00206C0C002038000020600C00202A
:1066600090B593B000AFF860B9607A6000237B64A6
:10667000BB68013B0D2B00F2D68001A252F823F03B
:10668000B966000827680008C3660008116700089B
:106690002B67000831670008756700085B67000812
:1066A00037670008B767000827680008CB6700084D
:1066B000EF670008FF660008FB681846FFF742FD19
:1066C000B4E07B683B645C4BFA6853F822305B4A69
:1066D000F96852F821103A6C52685948FC6850F831
:1066E000240000FB02F25748FC6850F8240000FB2D
:1066F00002F20A449A620220FBF79EFC96E07B6855
:10670000FB63FB6B1968504BFA6843F822108DE06D
:106710007B68BB63F968BB6B1A68BB6B1B79084667
:1067200011461A46FFF764FC80E0FFF703FD7DE0A9
:1067300000F0BEFD7AE07B687B633F4BFA6853F85C
:1067400022207B6B1B68002B0CBF00230123DBB2D4
:1067500010461946FBF718FD68E07B683B63F96853
:106760003B6B1A683B6B5B68084611461A46FFF79D
:10677000CBFB5BE007F1180207F11403F868114640
:106780001A460DF0FFFD7B68FB62FB6A19682C4B13
:10679000FA6843F82210FB6A59682C4BFA6843F8F0
:1067A0002210F968BA697B69084611461A46FFF754
:1067B000ABFB00BF3AE07B68BB62FA68BB6A1B6850
:1067C00010461946FFF7F2FB30E07B687B621A4BFC
:1067D000FA6853F822207B6A1B68002B0CBF002349
:1067E0000123DBB210461946FFF74EFB1EE07B6823
:1067F0003B623B6A1B6803F47F031A0C3B6A1B680D
:1068000003F47F431A433B6A1B68DBB21B04134348
:10681000FB61094BFA6853F82230FA69DA6002200A
:10682000FBF70AFC02E04FF0FF337B647B6C1846F9
:106830004C37BD4690BD00BF38000020682D0208CF
:10684000640C00206C0C00205C0C0020680C002004
:1068500080B582B000AF25482549002200230FF003
:1068600093FA0020F0214FF4A0720AF03FF80020C4
:10687000F0214FF4A0720AF021F800237B602EE093
:106880001C4B7A684FF0FF3143F822101A4B7A689C
:1068900053F822307868194609F0FAFF78680AF050
:1068A00059FF0346D910154B7A6843F822107868CF
:1068B0002121134A0AF07AF878682321114A0AF054
:1068C00075F87868FFF770FA0346042B04D87868E7
:1068D00019210D4A0AF06AF87B6801337B607B68F6
:1068E000002BCDDD0837BD4680BD00BF986802088B
:1068F000986A02085C0C0020682D02086C0C0020CD
:1069000069630008D9630008A164000880B485B0F9
:1069100000AF78600023FB60324BFB607B689B79A3
:10692000002B4DD02F4B2F4A11687A681268D24342
:106930000A401A602B4B2B4A51687A681268D2437E
:106940000A405A607B681B79FA681344FB60FB6855
:10695000FA6811687A6812680A431A60214B214A62
:1069600091687A681268D2430A409A601D4B1D4AAA
:10697000D1687A681268D2430A40DA607B685B7932
:10698000102B0ED1174B174A91687A6812680A4388
:106990009A60144B134AD1687A6812680A43DA6025
:1069A0001BE0104BFB607B685B79FA681344FB606B
:1069B000FB68FA6811687A6812680A431A600CE08A
:1069C0007B681B79FA681344FB60FB68FA681168FE
:1069D0007A681268D2430A401A601437BD465DF8DF
:1069E000047B7047003C014080B483B000AF786006
:1069F000034B7A685A610C37BD465DF8047B7047DB
:106A0000003C014080B483B000AF7860054A7B68E9
:106A100043F0BF6343F40033D3600C37BD465DF8E9
:106A2000047B704700ED00E080B485B000AF786073
:106A30000023FB730023BB730F237B737B68DB781E
:106A4000002B37D0254BDB68DB4303F4E0631B0AE4
:106A5000FB73FB7BC3F10403BB737A7BFB7B42FAC2
:106A600003F37B737B685B781A46BB7B02FA03F304
:106A7000FB737B689A787B7B1340DAB2FB7B134312
:106A8000FB73FB7B1B01FB73154A7B681B7813446C
:106A9000FA7B83F80023124B7A6812785209D2B23B
:106AA0007968097801F01F01012000FA01F143F82B
:106AB00022100EE00A4B7A6812785209D2B2796835
:106AC000097801F01F01012000FA01F1203243F89A
:106AD00022101437BD465DF8047B704700ED00E0DE
:106AE00000E100E080B584B000AF78600023FB7364
:106AF000194BCA225A62184B53225A6200F02EF8E0
:106B00000346002B02D10023FB731CE0124B124AF8
:106B1000926822F040029A600F4B0F4A91687A689F
:106B200012680A439A600C4B7A6892681A610A4BA1
:106B3000094A11697A68526812040A431A6100F01E
:106B400047F80123FB73044BFF225A62FB7B184674
:106B50001037BD4680BD00BF0028004080B485B01E
:106B600000AF00237B600023FB730023BB60174B47
:106B7000DB6803F04003002B1ED1144B4FF0FF32B3
:106B8000DA60124BDB6803F04003BB607B680133C3
:106B90007B607B68B3F5803F02D0BB68002BF0D0F0
:106BA0000A4BDB6803F04003002B02D00123FB7388
:106BB00004E00023FB7301E00123FB73FB7B184619
:106BC0001437BD465DF8047B704700BF00280040C5
:106BD00080B400AF044B044AD26822F08002DA602D
:106BE000BD465DF8047B70470028004080B485B046
:106BF00000AF00237B600023FB730023BB60184BB6
:106C0000CA225A62164B53225A62154B144AD26852
:106C100022F0A002DA60124BDB6803F02003BB60B5
:106C20007B6801337B607B68B3F5003F02D0BB68B3
:106C3000002BF0D00A4BDB6803F02003002B02D0BE
:106C40000123FB7301E00023FB73054BFF225A6213
:106C5000FB7B18461437BD465DF8047B704700BFC8
:106C60000028004080B487B000AF78600023FB7537
:106C700000233B610023FB60134B1B6C03F00403F8
:106C80003B61114B9A687B681A407B68D90B3B6962
:106C90000B401343FB600C4BDA687B681B09134005
:106CA0003B61FB68002B06D03B699BB2002B02D0F6
:106CB0000123FB7501E00023FB75FB7D18461C37A3
:106CC000BD465DF8047B70470028004080B485B065
:106CD00000AF78600023FB607B681B09FB60084BFA
:106CE000FA6892B242F08002D143054AD26802F0BB
:106CF00080020A43DA601437BD465DF8047B7047B2
:106D00000028004080B584B000AF0346FB71FA79DB
:106D1000104B53F8223018460121FBF7ADFEFA79EB
:106D20000D4B33F81230BB6001233B730023BB7360
:106D30000123FB7302237B73FA79084B53F822205B
:106D400007F1080310461946FDF718FA1037BD463B
:106D500080BD00BF742D0208702D02084400002081
:106D600080B483B000AF0346FB71FA79064B53F849
:106D70002230F979054A32F811201A830C37BD46C2
:106D80005DF8047B704700BF44000020702D0208AE
:106D900080B483B000AF0346FB71FA79094B53F816
:106DA0002230F979074A52F821205169F879064AC8
:106DB00032F810204A405A610C37BD465DF8047B1A
:106DC000704700BF44000020702D020880B588B0D5
:106DD00000AF02460B46FA71BB7101231846012130
:106DE000FBF74AFE4FF480400121FBF79FFE002392
:106DF0003B770023FB770123BB61FA79174B53F8EC
:106E0000222007F1180310461946FDF7B7F9BB79A0
:106E1000012B1FD10022002310461946FAF702FA6F
:106E200001233B6100233B7508237B750123BB7560
:106E300007F110031846FFF769FD06233B730F2384
:106E40007B730F23BB730123FB7307F10C031846FD
:106E5000FFF7EAFD2037BD4680BD00BF4C00002093
:106E600080B592B000AF08200121FBF705FE4FF47A
:106E700000537B6002237B7201233B720023BB72B1
:106E80000023FB723B1D2D481946FDF777F900F0F2
:106E900015FA002000F054F8012000F051F800F03D
:106EA0003FFA00F0B7F84FF080600121FBF73EFE9B
:106EB0004FF400000121FBF7DFFD00F093FAFDF72E
:106EC00065FA0023FB6000233B6100237B61002304
:106ED000BB610023FB6300233B6400237B64C02071
:106EE00007210422FBF79AFC4FF40030FBF7A6FDC4
:106EF0000120FBF7ABFC00BF3D20FBF771FE034612
:106F0000002BF9D00923FB6101233B621D237B6227
:106F10000323BB6240F20D13FB6240F243133B6359
:106F200040F217137B6340F24713BB6307F10C0376
:106F30001846FAF7CFFF4837BD4680BD000C024027
:106F400080B582B000AF0346FB71FB79002B04D102
:106F500005480421FDF7AEF903E003480421FDF7DD
:106F60009BF90837BD4680BD0008024080B582B05D
:106F700000AF0346FB7110484FF40051002200F0AF
:106F8000BDF90020FFF7DCFFFB799BB20B481946E7
:106F9000FEF7EEFB00BF09488021FEF7F7FB034632
:106FA000002BF8D10A2000F0D9FA0120FFF7C8FF22
:106FB0000837BD4680BD00BF000C024000500140B4
:106FC00080B582B000AF0346FB7110484FF400510A
:106FD000012200F093F90020FFF7B2FFFB799BB28A
:106FE0000B481946FEF7C4FB00BF09488021FEF795
:106FF000CDFB0346002BF8D10A2000F0AFFA0120A8
:10700000FFF79EFF0837BD4680BD00BF000C024061
:107010000050014080B500AFCA20FFF7A7FFC32092
:10702000FFF7CEFF0820FFF7CBFF5020FFF7C8FF88
:10703000CF20FFF79BFF0020FFF7C2FFC120FFF723
:10704000BFFF3020FFF7BCFFED20FFF78FFF64206C
:10705000FFF7B6FF0320FFF7B3FF1220FFF7B0FFE3
:107060008120FFF7ADFFE820FFF780FF8520FFF7C5
:10707000A7FF0020FFF7A4FF7820FFF7A1FFCB2098
:10708000FFF774FF3920FFF79BFF2C20FFF798FFD5
:107090000020FFF795FF3420FFF792FF0220FFF753
:1070A0008FFFF720FFF762FF2020FFF789FFEA201C
:1070B000FFF75CFF0020FFF783FF0020FFF780FF52
:1070C000B120FFF753FF0020FFF77AFF1B20FFF7E7
:1070D00077FFB620FFF74AFF0A20FFF771FFA220D3
:1070E000FFF76EFFC020FFF741FF1020FFF768FF9A
:1070F000C120FFF73BFF1020FFF762FFC520FFF71D
:1071000035FF4520FFF75CFF1520FFF759FFC7202B
:10711000FFF72CFF9020FFF753FF3620FFF726FFE5
:10712000C820FFF74DFFF220FFF720FF0020FFF7F8
:1071300047FFB020FFF71AFFC220FFF741FFB6203C
:10714000FFF714FF0A20FFF73BFFA720FFF738FFE8
:107150002720FFF735FF0420FFF732FF2A20FFF733
:1071600005FF0020FFF72CFF0020FFF729FF00207C
:10717000FFF726FFEF20FFF723FF2B20FFF7F6FE98
:107180000020FFF71DFF0020FFF71AFF0120FFF787
:1071900017FF3F20FFF714FFF620FFF7E7FE01205F
:1071A000FFF70EFF0020FFF70BFF0620FFF708FF99
:1071B0002C20FFF7DBFEC82000F0D0F92620FFF7D7
:1071C000D5FE0120FFF7FCFEE020FFF7CFFE0F20E9
:1071D000FFF7F6FE2920FFF7F3FE2420FFF7F0FE6D
:1071E0000C20FFF7EDFE0E20FFF7EAFE0920FFF767
:1071F000E7FE4E20FFF7E4FE7820FFF7E1FE3C209B
:10720000FFF7DEFE0920FFF7DBFE1320FFF7D8FEB5
:107210000520FFF7D5FE1720FFF7D2FE1120FFF75C
:10722000CFFE0020FFF7CCFEE120FFF79FFE0020FD
:10723000FFF7C6FE1620FFF7C3FE1B20FFF7C0FEB8
:107240000420FFF7BDFE1120FFF7BAFE0720FFF76D
:10725000B7FE3120FFF7B4FE3320FFF7B1FE422026
:10726000FFF7AEFE0520FFF7ABFE0C20FFF7A8FEF0
:107270000A20FFF7A5FE2820FFF7A2FE2F20FFF728
:107280009FFE0F20FFF79CFE1120FFF76FFEC82026
:1072900000F064F92920FFF769FE2C20FFF766FE55
:1072A00080BD00BF80B500AF2920FFF75FFE80BD25
:1072B00080B500AF2820FFF759FE80BD80B582B0B1
:1072C00000AF04200121FBF7D7FB04233B6002231E
:1072D0007B7101233B710023BB710023FB713B4693
:1072E00005481946FCF74AFF03480421012200F033
:1072F00005F80837BD4680BD0008024080B582B061
:1073000000AF786013460A467A807B707A887B7873
:10731000786811461A46FCF7DBFF0837BD4680BD8A
:1073200080B588B000AF20200121FBF7A5FB4FF40A
:1073300080100121FBF7FAFB80237B6002237B7224
:1073400002233B720023BB720023FB723B1D2348C8
:107350001946FCF713FF4FF480737B603B1D1F48F9
:107360001946FCF70BFF4FF400737B603B1D1B4875
:107370001946FCF703FF194807210522FCF7C0FF57
:10738000164808210522FCF7BBFF144809210522F5
:10739000FCF7B6FF1248FEF71BF90023BB814FF440
:1073A0008273FB8100233B8200237B820023BB820C
:1073B0004FF40073FB8208233B8300237B83072366
:1073C000BB8307F10C0306481946FEF76DF9044824
:1073D0000121FEF7ADF92037BD4680BD0014024003
:1073E0000050014080B582B000AF6F200121FBF753
:1073F00043FB544803210E22FCF782FF514804212D
:107400000E22FCF77DFF4F4806210E22FCF778FF85
:107410004C480B210E22FCF773FF4A480C210E2228
:10742000FCF76EFF41F658033B6002237B71022399
:107430003B710023BB710023FB713B464148194659
:10744000FCF79CFE404800210922FCF759FF3E480A
:1074500001210922FCF754FF3B4808210E22FCF7CA
:107460004FFF394809210E22FCF74AFF36480A210E
:107470000E22FCF745FF34480B210E22FCF740FF9B
:1074800040F603733B603B462F481946FCF776FEF7
:107490002E4806210E22FCF733FF2C4807210E222E
:1074A000FCF72EFF29480A210E22FCF729FF4FF492
:1074B00098633B603B4625481946FCF75FFE24482D
:1074C00003210E22FCF71CFF214806210E22FCF7A7
:1074D00017FF48233B603B461D481946FCF74EFE0C
:1074E0001C480A210E22FCF70BFF4FF480633B601F
:1074F0003B4618481946FCF741FE174806210E2264
:10750000FCF7FEFE144807210E22FCF7F9FE124894
:107510000A210922FCF7F4FE0F480B210E22FCF78A
:10752000EFFE0D480C210922FCF7EAFE4FF4E6536A
:107530003B603B4608481946FCF720FE0837BD462D
:1075400080BD00BF0000024000040240000802406D
:10755000000C0240001402400018024080B485B0C4
:1075600000AF78600023FB607B68FB6002E0FB6893
:10757000013BFB60FB68002BF9D11437BD465DF879
:10758000047B704780B58AB000AF78600023FB6150
:10759000FCF70CF9494B1B68002B18D1484B494AA2
:1075A0001A60474B00225A60474B4FF4A0425A6082
:1075B000454B00221A60434B7B617B694FF4A0422C
:1075C0005A607B69404A1A603C4B01221A607B6812
:1075D000002B0DD010237A6813447B607B6803F086
:1075E0000703002B04D07B6823F0070308337B607C
:1075F0007B68002B56D07B68B3F5A04F52D2304B3E
:107600003B622F4B1B687B6204E07B6A3B627B6AB8
:107610001B687B627B6A5A687B689A4203D27B6AEA
:107620001B68002BF1D17A6A274B9A423AD03B6A09
:107630001A6810231344FB617B6A1A683B6A1A605C
:107640007B6A5A687B68D21A10235B009A4222D95F
:107650007A6A7B6813443B617B6A5A687B68D21AFA
:107660003B695A607B6A7A685A603B695B68FB6079
:10767000134BBB6102E0BB691B68BB61BB691B6844
:107680005A68FB689A42F6D3BB691A683B691A606C
:10769000BB693A691A600D4B1A687B6A5B68D21A3B
:1076A0000A4B1A60FCF790F8FB69002B01D1FBF73D
:1076B000A1F8FB6918462837BD4680BDA05C0020B4
:1076C000905C0020900C0020985C0020500000206E
:1076D00080B586B000AF78607B683B617B68002B2B
:1076E00027D010235B423A6913443B613B69FB603E
:1076F000FCF75CF8FB685B68BB600F4B7B6102E0EA
:107700007B691B687B617B691B685A68BB689A420E
:10771000F6D37B691A68FB681A607B69FA681A609D
:10772000FB685A68054B1B681A44044B1A60FCF747
:107730004BF81837BD4680BD905C002050000020FB
:1077400080B500AF044B1B68002B04D1FCF7F2FBA3
:107750000246014B1A6080BDA85C002080B400AFD7
:10776000134B1B68591C124A1160B3F57A7F1BDD5D
:107770000F4B00221A600F4B1B68B3F57A7F03D9B9
:107780000C4B4FF47A721A600A4B1B68642202FB9E
:1077900003F2094BA3FB02139B09C3F16402074BDD
:1077A0001A60044B00221A60BD465DF8047B7047E6
:1077B000BC5C0020B85C0020D34D6210AC5C0020A3
:1077C00080B500AFFCF7B6FB0246054B1B689A423A
:1077D00004D1FCF773F80246024B1A6080BD00BF6B
:1077E000A85C0020B05C002080B500AFFCF7A2FBD5
:1077F00002460A4B1B689A420ED1FCF75FF802461C
:10780000074B1B68D21A074B1A60074B1A68054BC7
:107810001B681A44044B1A6080BD00BFA85C00209E
:10782000B05C0020B45C0020B85C002080B582B061
:1078300000AF78607A685F4B9A4208D1012001213D
:10784000FBF7B0F901200021FBF7ACF9AFE07B6852
:10785000B3F1804F08D101200121FBF785F9012008
:107860000021FBF781F9A2E07A68534B9A4208D1D4
:1078700002200121FBF778F902200021FBF774F9BF
:1078800095E07A684D4B9A4208D104200121FBF71C
:107890006BF904200021FBF767F988E07A68484B10
:1078A0009A4208D108200121FBF75EF90820002147
:1078B000FBF75AF97BE07A68424B9A4208D11020D4
:1078C0000121FBF751F910200021FBF74DF96EE083
:1078D0007A683D4B9A4208D120200121FBF744F9F8
:1078E00020200021FBF740F961E07A68374B9A428B
:1078F00008D102200121FBF755F902200021FBF7F6
:1079000051F954E07A68324B9A420AD14FF48030F0
:107910000121FBF747F94FF480300021FBF742F9D2
:1079200045E07A682B4B9A420AD14FF4003001218E
:10793000FBF738F94FF400300021FBF733F936E05C
:107940007A68254B9A420AD14FF480200121FBF737
:1079500029F94FF480200021FBF724F927E07A6809
:107960001E4B9A4208D140200121FBF7FDF8402030
:107970000021FBF7F9F81AE07A68194B9A4208D10E
:1079800080200121FBF7F0F880200021FBF7ECF8C4
:107990000DE07A68134B9A4209D14FF480700121AF
:1079A000FBF7E2F84FF480700021FBF7DDF80837B1
:1079B000BD4680BD000001400004004000080040BA
:1079C000000C004000100040001400400004014082
:1079D00000400140004401400048014000180040C0
:1079E000001C00400020004080B483B000AF7860ED
:1079F00013460A467A803B807B687A881A857B68C2
:107A00003A889A820C37BD465DF8047B704700BF08
:107A100080B483B000AF78600B46FB70FB78002B1E
:107A200008D07B681B889BB243F001039AB27B6845
:107A30001A8007E07B681B889BB223F001039AB28F
:107A40007B681A800C37BD465DF8047B704700BF29
:107A500080B582B000AF786039603B681B88002B2E
:107A60000FD13B6859883B689A883B681B897868C6
:107A700000F030F93B68DB887868194600F048F878
:107A800036E03B681B88042B0FD13B6859883B6864
:107A90009A883B681B89786800F058F93B68DB8856
:107AA0007868194600F050F822E03B681B88082BE4
:107AB0000FD13B6859883B689A883B681B89786876
:107AC00000F08AF93B68DB887868194600F05AF8BC
:107AD0000EE03B6859883B689A883B681B89786848
:107AE00000F0BCF93B68DB887868194600F066F85E
:107AF0000837BD4680BD00BF80B483B000AF78605A
:107B00007B681B6C18460C37BD465DF8047B7047DC
:107B100080B483B000AF78600B467B807B681B8BA2
:107B20009BB223F00C039AB27B681A837B681B8B91
:107B30009AB27B8813439AB27B681A830C37BD468E
:107B40005DF8047B704700BF80B483B000AF7860FD
:107B50000B467B807B681B8B9BB223F440639AB2FD
:107B60007B681A837B681B8B9AB27B881B029BB253
:107B700013439AB27B681A830C37BD465DF8047BC9
:107B8000704700BF80B483B000AF78600B467B8045
:107B90007B689B8B9BB223F00C039AB27B689A8321
:107BA0007B689B8B9AB27B8813439AB27B689A83DB
:107BB0000C37BD465DF8047B704700BF80B483B0CE
:107BC00000AF78600B467B807B689B8B9BB223F475
:107BD00040639AB27B689A837B689B8B9AB27B885E
:107BE0001B029BB213439AB27B689A830C37BD4643
:107BF0005DF8047B704700BF80B483B000AF78604D
:107C000013460A467A807B707B78002B08D07B680D
:107C10009B899AB27B8813439AB27B689A8109E068
:107C20007B689B899AB27B88DB439BB213409AB2F4
:107C30007B689A810C37BD465DF8047B704700BFB6
:107C400080B485B000AF78600B467B800023FB7367
:107C50000023BB8100237B817B681B8A9AB27B88CF
:107C60001340BB817B689B899AB27B8813407B81E0
:107C7000BB89002B05D07B89002B02D00123FB732D
:107C800001E00023FB73FB7B18461437BD465DF80B
:107C9000047B704780B483B000AF78600B467B8074
:107CA0007B88DB439AB27B681A820C37BD465DF84D
:107CB000047B704780B483B000AF78600B467B8054
:107CC0007B687A88A3F850200C37BD465DF8047BAA
:107CD000704700BF80B487B000AFF86079813A8107
:107CE000FB800023FB820023BB82FB681B8C9BB2C2
:107CF00023F001039AB2FB681A84FB681B8BFB829A
:107D0000FB681B8CBB82FB8A23F0F303FB82FB889E
:107D10001B019AB23B8913439AB2FB8A1343FB823D
:107D2000BB8A23F00A03BB827A89BB8A13439BB2C6
:107D300043F00103BB82FB68FA8A1A83FB68BA8AA4
:107D40001A841C37BD465DF8047B704780B487B049
:107D500000AFF86079813A81FB800023FB82002329
:107D6000BB8200237B82FB681B8C9BB223F0100339
:107D70009AB2FB681A84FB681B8BFB82FB681B8C26
:107D8000BB827B891B017B82FB8A23F440731B052A
:107D90001B0DFB82FB881B039AB2FB8A1343FB82F9
:107DA0003B891B029AB2FB8A1343FB82BB8A23F0F6
:107DB000A003BB827A8ABB8A13439BB243F01003B1
:107DC000BB82FB68FA8A1A83FB68BA8A1A841C375A
:107DD000BD465DF8047B704780B487B000AFF860A3
:107DE00079813A81FB800023FB820023BB82002340
:107DF0007B82FB681B8C9BB223F480739AB2FB6876
:107E00001A84FB689B8BFB82FB681B8CBB827B8983
:107E10001B027B82FB8A23F0F303FB82FB881B019E
:107E20009AB23B8913439AB2FB8A1343FB82BB8A03
:107E300023F42063BB827A8ABB8A13439BB243F448
:107E40008073BB82FB68FA8A9A83FB68BA8A1A84B9
:107E50001C37BD465DF8047B704700BF80B487B017
:107E600000AFF86079813A81FB800023FB82002318
:107E7000BB8200237B82FB681B8C9BB223F4805364
:107E80009AB2FB681A84FB689B8BFB82FB681B8C95
:107E9000BB827B891B037B82FB8A23F440731B0517
:107EA0001B0DFB823B891B029AB2FB8A1343FB82A8
:107EB000FB881B039AB2FB8A1343FB82BB8A23F421
:107EC00000535B045B0CBB827A8ABB8A13439BB270
:107ED00043F48053BB82FB68FA8A9A83FB68BA8AB0
:107EE0001A841C37BD465DF8047B704730B50446E4
:107EF00083B00D4608B903B030BD0CF069F82046D8
:107F00000FF00EFC836B0190AB4203D085632046DB
:107F100004F0E6FD01A80FF015FC0CF04FF8EAE7BD
:107F200030B5044683B00D4618B90125284603B084
:107F300030BD0CF04DF820460FF0F2FB436C009082
:107F4000684601930FF0FEFB294601A80AF088FE5F
:107F5000D0F1010538BF002515B10CF02FF8E5E789
:107F600020460FF0DDFB0199426C00908A4218BF59
:107F7000416468460FF0E6FB204604F0B1FDECE7F3
:107F800030B5044683B00D4608B903B030BD0CF0DF
:107F90001FF820460FF0C4FB436B0190AB4203D0A7
:107FA0004563204604F09CFD01A80FF0CBFB0CF0CC
:107FB00005F8EAE730B5456885B00446014628462D
:107FC00010F082FEB8B123680C2B16D00F2B20D0F6
:107FD0000B2B0DD128460FF0A3FB04AD014645F84D
:107FE0000C1D00F144000FF0C1FC28460FF0AAFB65
:107FF000204605F005FA05B030BDE268002A3BD006
:10800000117A00290CBF02210121284602F094FCBC
:10801000EEE728460FF084FB0090806B0AF02AFD03
:108020000098406B0CF012F9284602F0E7F9E0B135
:10803000009B596CA9B102200CF0D8F802A803F0FB
:108040006FFA0098406C0FF06BFB009B0190B3F946
:10805000482093F8403002A90DF02AFB01A80FF048
:1080600071FB68460FF06EFBC5E7009AD06B0AF013
:10807000F7FC0DF091FFDBE70321C6E72DE9F043A4
:1080800087B08146884617461E46129D0BF0A0FF1A
:108090000E9C0F9813990094224C40F0010201F1BC
:1080A0002003019202940393484641463A463346E0
:1080B00004F01AFD044618B33DB1284617F092F9B2
:1080C00001300FF059FD804600BB4FF0000805AFAE
:1080D00020460FF025FB144D11990590002210F059
:1080E000E9FD95E80F00059E06F1340585E80F00CF
:1080F0001098C6F84480A6F8480038460FF022FBD6
:108100000BF05CFF204607B0BDE8F0830FF008FBE2
:1081100006AF294647F8040D17F006F938460FF068
:1081200011FBD5E7B57F00085400002010B586B0DC
:10813000089C0094099C01940A9C02940B9C039453
:108140000C9C049400240594FFF798FF06B010BD22
:108150002DE9F04F2DED028B85B00D460FF0E0FAC2
:10816000009000690CF072F8009BD8680CF0B6F82B
:1081700002200CF03BF8009CA08C10F001070AD103
:10818000E269002A68D168460FF0DCFA05B0BDEC60
:10819000028BBDE8F08FE269002AF4D0A0680FF0EE
:1081A000BFFA0190C16A60690B6803EB000802F036
:1081B00087FFA26908EB0001002A40F0AC80B5F906
:1081C0000430994200F3A38002A9A06802F0C4FF22
:1081D000019F3D6EBF6D0CF08DFABDF90E60019AE6
:1081E000216AD2F88030BDF80AE0761B751AED18C6
:1081F000AE4203DDE1696D18AE42FCDC07FA8EF792
:10820000AF4200F384804FF0020990FBF9F903E0DC
:10821000E269AD1AAF427ADCAE42F9DBA0690BF03D
:10822000F5FF019A206AD2F88020731B191A88186A
:1082300000EE900AD4ED0A1AB8EEE01AC9EB050177
:1082400021EE218A40460CF019FA18EE100A94F833
:108250002C100BF023FCDBE7A0680FF061FA019013
:10826000C16AD1F800800CF045FA63690646C8EB94
:10827000030902F037FFB5F90220E98848443618AF
:10828000964244DB0BB2984241DCA06802A902F09E
:1082900063FF019DBDF90CB0EA6DB5F87810D5F813
:1082A00054A0BDF90860206AC2EB0B0BCA07564404
:1082B00058BFD5F88C703318DD19AE4225DAE26963
:1082C00051426D18AE42FCDB1FE0AE421BDAA069E2
:1082D0000BF09CFF206A2B1ACAEB0302C8EB0201C9
:1082E000C81B08EE100AD4ED0A7AB8EEC80A49464F
:1082F00020EE278A28460CF0C1F918EE100A94F8EF
:108300002C100BF0CBFBE369ED18AB45DDDA01A8CF
:108310000FF018FA37E7012A7FF456AFB5F90000DD
:108320008142F4DB50E700BF2DE9F04782B082467E
:10833000894690461F460BF04BFE30200FF01CFC88
:108340000546D8B10FF0ECF902AE0F4B46F8040D1C
:10835000044693E8030004F10C0282E803000B4991
:10836000C4F814A04FF07E50A062C4F81890A4F88E
:108370002480E761216030460FF0E4F90BF01EFE27
:10838000284602B0BDE8F087640000205181000853
:1083900030B5044683B00D4610B9204603B030BD59
:1083A0000BF016FE20460FF0BBF9046A0190AC42B8
:1083B00003D00562806804F093FB01A80FF0C2F9B6
:1083C0000BF0FCFDE9E700BF30B5044683B00D4675
:1083D00010B9204603B030BD0BF0FAFD20460FF077
:1083E0009FF9C4680190AC4203D0C560806804F076
:1083F00077FB01A80FF0A6F90BF0E0FDE9E700BF5D
:1084000010B52DED028B044682B008EE901A38B9F3
:108410009FED108A18EE100A02B0BDEC028B10BD61
:108420000BF0D6FD20460FF07BF990ED0A8AB4EEF2
:10843000688AF1EE10FA019005D101A80FF082F9D7
:108440000BF0BCFDE6E7C0ED0A8A806804F048FB4B
:10845000F3E700BF0000000030B5044683B00D46CE
:1084600010B9204603B030BD0BF0B2FD20460FF02E
:1084700057F9C46A0190AC4203D0C562806804F029
:108480002FFB01A80FF05EF90BF098FDE9E700BFA4
:1084900010B582B004460FF043F90190406A20B154
:1084A0000FF03EFA019B00225A6201A80FF04AF930
:1084B00020460FF035FA02B010BD00BF2DE9F04F95
:1084C0008BB00FF02DF90790406A28B907A80FF07C
:1084D00039F90BB0BDE8F08F0FF022F9079B05903A
:1084E000064698680FF01CF9079AD0F85490014698
:1084F0000691D1F85C8090688F6D0D6E08A902F02E
:108500002BFE069BBDF82010079CD3F88C20D3F8D7
:1085100080A0BDF8243094F82800D4F820B0494455
:10852000BDF82690C8EB030CC5EB0905BDF8223059
:108530001FFA85F92569ADF8269089B2FF181FFA50
:108540008CF80128ADF82010ADF82270ADF8248029
:10855000C2EB05052CD00FFA88F2501B471C09B25C
:108560008F421FDB002D16DDA0690BF0B7FE4FF028
:10857000FF3201238DE80C00079A0FFA89F992F86F
:108580002900CBEB090B0290294630463A460BEB0B
:108590000A030CF0A1FD06A80FF0D4F805A80FF00F
:1085A000D1F893E7CB1B06EB4306ED1A0F46D9E74C
:1085B0000FB2D7E770B590F82830012B84B004468D
:1085C00004D0806800F042FD04B070BD02A980684C
:1085D00002F0C2FDA0680FF0A3F8466D856D016E34
:1085E0000190BDF80800226933189A1890B2BDF8BE
:1085F0000A30BDF80E20ED18511A431E821E01A844
:10860000ADF80E10ADF80A50ADF80820ADF80C30FA
:108610000FF098F8A06802A904F09EF9D4E700BF13
:108620002DE9F04782B007460D4690461E460BF0F6
:10863000CFFC2C200FF0A0FA044628B90BF0BEFCAA
:10864000204602B0BDE8F08768000FF095FA824638
:1086500018B1B8F1000F00D0AEB90DF104092046F1
:108660000FF05EF80F4B019002460F49D3600F4B9D
:10867000C2F824A0484697615561166111605360A5
:108680000FF060F8DAE70FF04BF80DF108094146FA
:1086900049F8040D7200F8F755FA48460FF052F801
:1086A000DDE700BFB5850008BD840008918400089F
:1086B00010B584B00446ADF806100BF089FC2046D6
:1086C0000FF02EF8029070B1406A0FF029F80346BF
:1086D0000146039302980DF10602022300F0E6FC26
:1086E00003A80FF02FF802A80FF02CF80BF066FC8F
:1086F00004B010BD30B5044683B00D4608B903B0D0
:1087000030BD0BF065FC20460FF00AF8036A0190BB
:10871000AB4203D00562806804F0E2F901A80FF0D3
:1087200011F80BF04BFCEAE7F0B58BB002A9064656
:1087300002F012FD30460EF0F3FFBDF90E50BDF908
:108740000A40B0F878200346806D196E01932F1B04
:1087500002F004043D1AA0B2DF6D5C6D6D1A0028B2
:108760003CD0BDF90800BDF90CE0596FC3F8845046
:1087700002F00202C0EB0E052C1B90B2D967E51B7C
:1087800040B9196FA9423046D4BF0021012101F040
:108790006FFE019B196FC3F8905003F17C00C3F882
:1087A000881002F0E7FE0198883002F0E3FE019C99
:1087B00004F17C0207CA07AD883485E8070094E815
:1087C000070004AC84E8070001A80EF0BBFF3046A8
:1087D0002946224610F04CFB0BB0F0BD596FA94260
:1087E0003046D4BF0021012101F062FE019BB3F8A5
:1087F0007820B6E72DE9F04F90E81800B3F5407FF8
:108800009DB0054600F07D822046294610F05CFAB6
:108810000646002E00F044822B68591F212900F2E1
:108820006C82DFE811F077026A026A026A026A0269
:108830006A027E026A026A026A0222006A026A020E
:108840006A026A026A026A026A026A026A026A02C8
:108850006A026A026A026A026A026A026A026A02B8
:108860006A026A026A026A0240022046ED680EF05D
:1088700057FF1190C76A436DC26D816DD0F860B02B
:108880003868069316AE089016A8099204960791C8
:1088900002F046FE119816A910F09EFB049E079A5E
:1088A000089B96E8030018AF87E80300BDF8621044
:1088B00003975618BDF86070099A9BB2D91903EB5B
:1088C0000B009F189B19BDF86660069AADF86230E0
:1088D000301ABDF86460ADF86600F71B8918ADF872
:1088E0006470039FADF8601097E803001AAB83E84B
:1088F00003001846059301F047FD1198406B0BF0FB
:10890000E1FC0DF049FB119ED6F894201AB12046E7
:1089100000219047119E96F86C10002940F0D882F3
:1089200016A9089A18A80AF0D9F918A801F02CFD80
:10893000119E96F83B30FF2B00F0A180069939B9C3
:10894000079828B9099A1AB9BBF1000F00F097806F
:10895000F76A14A92046D7F8008002F0FDFB02F068
:10896000AFFB089002F0BEFB0699BDF95030BDF98F
:108970005420BDF95290BDF956A05B180B93099B8A
:108980000799D21A0746B06B0A9289440BF09AFCF9
:10899000F06B0BF0A3FC069ECBEB0A0AE6B1B5F92F
:1089A0000000089B711E01EB0802C61AB24213DBDD
:1089B000BDF95610079EBDF95000CBEB0103013302
:1089C00008EB06010DF0B2FA0B9A09F1FF31501EC7
:1089D0000AF101020BF0FCFE0798B0B1B5F90210E4
:1089E000431E4344CE1BB3420FDBBDF95000BDF91B
:1089F0005210BDF954200DF099FA0B9A0A9B511EA2
:108A000009F1FF305A1C0CF039FB0998D8B1BDF9B7
:108A10005420B5F90460089B111A481CF61AB0429C
:108A200011DCBDF95610079ECBEB0103013308EBB7
:108A300006010DF07BFA0A9A09F1FF31501C0AF188
:108A400001020BF0C5FEBBF1000F17D0BDF9563087
:108A5000B5F90600CBEB03010131C71BB9420DDCB0
:108A6000BDF95000BDF954200DF060FA0B9F0A9B30
:108A70000AF10100791E5A1C0CF000FB119ED6F879
:108A8000942012B12046012190471AA801F07CFCE5
:108A90001198406E10F0A2FF8046002874D0119EFD
:108AA000002100F1FF37706E11F024F80EF038FE4F
:108AB00007F00107129078B1066830460EF030FEDC
:108AC000139030B1036829463046984713A80EF03A
:108AD00039FE12A80EF036FE0126464554D0DFB10D
:108AE000119A3146506E11F005F80EF019FE1290F1
:108AF00078B1076838460EF013FE139030B1036862
:108B000029463846984713A80EF01CFE12A80EF00E
:108B100019FE0136464537D031461198406E4F1C3C
:108B200010F0E8FF0EF0FCFD129080B106683046B0
:108B30000EF0F6FD024629463046139222B1136824
:108B4000984713A80EF0FEFD12A80EF0FBFD119839
:108B50003946406E10F0CEFF0EF0E2FD129080B16B
:108B6000066830460EF0DCFD024629463046139278
:108B700022B11368984713A80EF0E4FD12A80EF076
:108B8000E1FD791C4145C8D118A801F0FDFB119900
:108B9000886E10F023FF8046002874D0119E0021BB
:108BA00000F1FF37B06E10F0A5FF0EF0B9FD07F031
:108BB0000107129078B1066830460EF0B1FD1390AF
:108BC00030B1026829463046904713A80EF0BAFD2E
:108BD00012A80EF0B7FD0126464554D0DFB111981A
:108BE0003146806E10F086FF0EF09AFD129078B13B
:108BF000076838460EF094FD139030B1036829469B
:108C00003846984713A80EF09DFD12A80EF09AFD65
:108C10000136464537D03146119A906E4F1C10F000
:108C200069FF0EF07DFD129080B1066830460EF0AF
:108C300077FD034629463046139323B11A689047BF
:108C400013A80EF07FFD12A80EF07CFD1198394696
:108C5000806E10F04FFF0EF063FD129080B1066839
:108C600030460EF05DFD034629463046139323B18E
:108C70001A68904713A80EF065FD12A80EF062FD69
:108C8000791C4145C8D1002001F07EFB1199D1F833
:108C9000943013B120460221984711A80EF052FDDE
:108CA0001DB0BDE8F08FE868052826D12046AE68E3
:108CB00002F0EAF9864205D02046AC6802F0D6F907
:108CC00084421AD16E68AC6830460EF029FD1390CC
:108CD000204610F021FA0746204602F0B1FA139A16
:108CE000FE2808BFC2F88070304618BFC2F88C70EA
:108CF00003F0F6FE13A80EF025FD284604F080FBD5
:108D0000CEE7204629460FF0DFFF06462046FFF754
:108D10000BFD7EE52046FFF707FD284604F070FBBB
:108D2000BEE720460EF0FCFC1190406E10F056FE9F
:108D3000061E6FDD119C0021606E10F0DBFE0EF050
:108D4000EFFC751E05F00105129070B10468204615
:108D50000EF0E6FC139028B142682046904713A815
:108D60000EF0F0FC12A80EF0EDFC0124A64251D04A
:108D7000D5B111982146406E10F0BCFE0EF0D0FC2B
:108D8000129070B1056828460EF0CAFC139028B105
:108D900041682846884713A80EF0D4FC12A80EF0AC
:108DA000D1FC0134A64235D02146119B586E4C1C93
:108DB00010F0A0FE0EF0B4FC129078B105682846C1
:108DC0000EF0AEFC02461392284622B15168884745
:108DD00013A80EF0B7FC12A80EF0B4FC11982146AF
:108DE000406E10F087FE0EF09BFC129078B1056883
:108DF00028460EF095FC03461393284623B15A6883
:108E0000904713A80EF09EFC12A80EF09BFC611C6C
:108E10008E42CAD1119EB06E10F0E0FD061E49DDF3
:108E2000119C0021A06E10F065FE0EF079FC751EFD
:108E300005F00105139028B100680EF071FD13A82C
:108E40000EF080FC0124A64234D08DB11198214649
:108E5000806E10F04FFE0EF063FC139028B1006896
:108E60000EF05EFD13A80EF06DFC0134A64221D079
:108E70002146119B986E4C1C10F03CFE0EF050FCED
:108E8000139028B100680EF04BFD13A80EF05AFCA9
:108E9000119A2146906E10F02DFE0EF041FC1390B9
:108EA00028B100680EF03CFD13A80EF04BFC611CCD
:108EB0008E42DED111991CAC486E10F0EBFD54F8D7
:108EC0002C0D806E10F0E6FD20460EF03BFCE7E630
:108ED00014A9204602F040F9F76ABDF856203B6815
:108EE000BDF85210306C0D930A920C91D6F8449054
:108EF000D6F84880BDF854A0BDF850700BF0EEF9DC
:108F00000BF0EAFB0B90B9F1000F55D0B6F87820C2
:108F1000F06CD10758BFD6F88C1009EB000348BF9E
:108F200000215B18994503DCC9EB03039945FBDD80
:108F30000998069A811838B20FFA8AF2121AC1F10A
:108F4000010101EB020C96F87A000193CDF808C0FC
:108F50000BF06CF9019BDDF808C063452CDA0D9F1E
:108F600006980E9507EB000A03EB0A07CDF83C8044
:108F7000CAF1000A0D94079DE04606E00CF054F893
:108F80004F440AEB0702904513DDBDF95640BDF989
:108F900052E096F87AC0CBEB040438463A460EEB22
:108FA00005012346BCF1000FE8D122460BF010FC6E
:108FB000E6E70DAB93E83001B8F1000F42D0376D12
:108FC000D6F8800008EB07010F1AB84503DCC8EBA0
:108FD0000707B845FBDD079A0A9B0C980BEB0209C3
:108FE00019B202B2C9F1010E8B1A0EEB030996F801
:108FF0007B000BF01BF9B94524DD0C950A94069D06
:10900000DDF824A005E060460CF00EF84744B945B1
:1090100016DDBDF95610BDF950C0BDF9544096F8A3
:109020007BE0CBEB0100C11B08460B46AC44CAEB0E
:109030000402BEF1000FE6D161460CF01FF8E5E72F
:109040000A9C0C9D0B980BF0F1F869E42DE9F041B6
:1090500084B004460EF064FB034604A8D3F85480A1
:1090600040F80C3D9F6DDE6D1D6E0EF06BFB2046D3
:1090700002A902F071F8BDF80800BDF80A10BDF8A9
:109080000C20BDF80E3080447F18961B5D1B2046D7
:1090900002A9ADF80880ADF80A70ADF80C60ADF823
:1090A0000E5003F059FC04B0BDE8F0812DE9F04109
:1090B000856886B004460E4617467DB10069626930
:1090C00090420ED0411C216100FB03601A463946D4
:1090D00016F05AF8E368ABB12046984706B0BDE8F1
:1090E000F081451E05FB03F2C9183046019316F0C6
:1090F0004BF820693946019F451E3A4605FB07603B
:1091000016F042F8A46820460EF00AFB024606A8B4
:10911000D2F8548040F80C2D976DD66D156E0EF078
:1091200011FB204604A902F017F8BDF81010BDF895
:109130001400BDF81230BDF816208844861BFF18B5
:10914000551B204604A9ADF81080ADF81270ADF89B
:109150001460ADF8165003F0FFFBBFE72DE9F041B6
:1091600086B0804616461D460F460AF031FF0C9C1D
:109170001C4B00940D9C02936C200390324601948A
:10918000404639462B4603F0AFFC064618B310F0B4
:10919000D3FC054610F0D0FC074630460EF0C0FA6E
:1091A0004566114D87660F99059000220FF082FDEC
:1091B00006AF0FCD57F804ED0EF134040FC40FCDF8
:1091C0000FC495E80F000E9D84E80F00AEF87850AC
:1091D00038460EF0B7FA0AF0F1FE304606B0BDE8A8
:1091E000F08100BFF58700086C00002030B585B025
:1091F00004460191F8B10AF0EBFE20460EF090FA19
:10920000024604A8556E40F8042D0EF09BFA019812
:109210000EF086FA014604A88C6040F8081D0EF096
:1092200091FA01A90422284610F0E8FB204603F039
:1092300057FC0AF0C3FE05B030BD00BF30B585B0A5
:1092400004460191F8B10AF0C3FE20460EF068FA18
:10925000024604A8956E40F8082D0EF073FA0198A6
:109260000EF05EFA014604A88C6040F8041D0EF072
:1092700069FA01A90422284610F0C0FB204603F039
:109280002FFC0AF09BFE05B030BD00BF70B5044650
:1092900082B00E4618B90546284602B070BD0AF0E5
:1092A00097FE20460EF03CFA90F86C500190B542C3
:1092B00004D080F86C60204603F012FC01A80EF088
:1092C00041FA0AF07BFEE7E770B5044682B00E462D
:1092D00018B90546284602B070BD0AF079FE20464E
:1092E0000EF01EFA856C0190B54203D086642046CC
:1092F00003F0F6FB01A80EF025FA0AF05FFEE9E79D
:109300002DE9F043044685B00E4620B905462846AF
:1093100005B0BDE8F0830AF05BFE20460EF000FACF
:10932000056D0090B5422BD0066520460EF0F8F989
:10933000034604A8D3F8549040F80C3DD3F8588065
:10934000DF6D1E6E0EF0FEF9204602A901F004FF4B
:10935000BDF80800BDF80A10BDF80C20BDF80E30AD
:1093600081448844D71B9E1B204602A9ADF8089073
:10937000ADF80A80ADF80C70ADF80E6003F0ECFAB1
:1093800068460EF0DFF90AF019FEC0E72DE9F0415A
:10939000044682B00E4617469846C0B10AF018FE41
:1093A00020460EF0BDF902AD089B45F8040D03669A
:1093B00046658765C0F85C8028460EF0C3F92046F4
:1093C000FFF7B2F9204603F08BFB0AF0F7FD02B07D
:1093D000BDE8F08130B5044683B00D4688B10AF08F
:1093E000F7FD20460EF09CF902ABC0F8945043F80C
:1093F000040D18460EF0A6F9204603F071FB0AF0A2
:10940000DDFD03B030BD00BF70B5044682B00E462E
:1094100018B90546284602B070BD0AF0D9FD2046AD
:109420000EF07EF990F87B500190B54204D080F8A0
:109430007B60204603F054FB01A80EF083F90AF08C
:10944000BDFDE7E770B5044682B00E4618B9054683
:10945000284602B070BD0AF0BBFD20460EF060F950
:1094600090F87A500190B54204D080F87A60204696
:1094700003F036FB01A80EF065F90AF09FFDE7E75F
:109480002DE9F041044692B00068944D00F0DAFAFC
:10949000934A6368002818BF15461C2B00F2D88039
:1094A000DFE813F0DA00D600D600D600D600EE00D2
:1094B000D600D600D600D600D6001D00D600D600B5
:1094C0000601D600D600D6002001D600D6005A01EB
:1094D0005C015E016001D600D600D60062012668FC
:1094E0001C27304609960A970EF01AF9016D05906F
:1094F00009A88847064605A80EF024F9012E40F376
:1095000053812B68206900936A68A1690192AF6852
:1095100062690297334609F0B7FC2069A16906EB3E
:1095200000088F1B28680AF0D9FE41463A46606958
:109530000BF0A4FD68680AF0D1FE63694146581C2F
:109540003A460BF09BFD6B6A022B00F320812A6ADE
:10955000964217DA616920698F1C012E40F352810F
:1095600006EB010812183946013A801943460BF000
:10957000E5F8A1698A1BE8690B1A581C394643466D
:109580000BF0DCF8012ECCBF63696669E7692868D7
:10959000CCBFF6180236013F0AF0A0FE3A46206919
:1095A00031460BF015F93A463146A0690BF010F937
:1095B000E16968688F1E0AF091FE2069314601302A
:1095C0003A460BF005F9A2693146501E3A460BF0B7
:1095D000FFF8EB69022B02DC296A022921DDA86A67
:1095E000E7690228C8BFC0EB0707A868D8BF023FD9
:1095F0000AF074FEEA69022A07DD2369D218981C72
:109600003146013A3B460BF099F8296A022908DDF8
:10961000A269E869131A581C3146023A3B460BF01E
:109620008DF828680AF05AFE2169A269E0690BF0FA
:1096300025FD68680AF052FEE6692169A269701E7C
:109640000131013A0BF01AFDAE6A022E00F38E8052
:10965000002012B0BDE8F08120680EF061F812AB76
:10966000B0F85A1043F8340D41F00C02A0F85A201B
:1096700018460EF067F8206800F098FE0020E8E732
:10968000EF68208A0097A78A268B2A69A48BADF8F9
:109690001C00019200B239B232B223B2ADF81E7092
:1096A000ADF82060ADF822400BF058FE0020D0E766
:1096B00004F1140090E80E002669A868ADF81E10A9
:1096C000ADF82020ADF82230ADF81C600AF006FE9F
:1096D00007A80BF027F80020BBE700BFC800002058
:1096E0009C0000202B8B2169A5696669E2692068CE
:1096F000ADF81E605918EB1AADF81C10ADF820300B
:10970000ADF822200EF00CF80590006FF8B10220A1
:109710000AF06CFD0599B1F87C20C2F3C0030E334A
:1097200001EB830080680AF0D9FD0599486B0AF0C7
:109730008DFD059A106F0DF0F3FF059B069007A9AC
:10974000B3F95A200CF0B4F906A80DF0FBFF05A8F8
:109750000DF0F8FF00207CE7A86A7AE7E86978E76F
:10976000286A76E7686A74E7686972E7E7692369D7
:10977000A469A868023C9D1C0AF0B0FDB91B2846EC
:1097800001312246BB1E0AF0D9FF002061E7A8681C
:109790000AF0A4FD61696A6A8B18404602313A46B4
:1097A000013B0AF0CBFFEDE628680AF097FD21693E
:1097B000EA6960698B185A1E0BF060FCA269EF69B8
:1097C0006069D11B01310BF059FC62692069571C9B
:1097D00039460BF027F83946A0690BF023F8686882
:1097E0000AF07CFD2069394601300BF01BF8A369B3
:1097F0003946581E0BF016F82169A26901F10208DA
:10980000971E8FE613185A1E394602303B460AF05F
:1098100095FFA169B8468A1EADE600BF70B58AB053
:1098200005460C460DF07CFF0AAB066D43F8280D8B
:1098300068460DF087FF0195032C05D8DFE804F09A
:109840000E0B08021720029001A8B0470AB070BDA5
:1098500015210291F8E716220292F5E718230293E8
:10986000F2E700BF30B58BB005460DF059FF0AABEB
:10987000C26D43F8280D684694680DF063FF0AA88E
:10988000002140F8245D0291636898470BB030BD19
:109890002DE9F04F8FB005460DF042FFC26D416BD0
:1098A000D2F8088001910490046D00F081F9074618
:1098B0000EA850F8286DB6F858A00DF043FF2846C2
:1098C00001F080FA8146284601F09AFAD8F8003073
:1098D0000090012128469847D8F800200321064629
:1098E00028469047D8F800308346002128469847FC
:1098F00080460020059503F037FA002849D00099EA
:10990000474407FA8AF0CBEB090B4A1E0BF1FF3CE8
:10991000431E3946781E00922A4609F1FF3A47460F
:10992000029303904FF00009654693468846009BDA
:10993000CDF828900B200C930690CDF82490CDF80C
:109940002CA005A8A047029909960E220C91069218
:10995000CDF828800B9505A8A047039B0996052004
:109960000C9306900A970B9505A8A04709A90BAA86
:10997000584600F02DF902200AF038FC01980AF050
:1099800065FC1221069105A8A04703F0CBF9002839
:10999000CDD10FB0BDE8F08F40F2F403C2F2000366
:1099A00010B440F20812586093E80300C2F20002BB
:1099B00040F23013D4691832C2F2000382E8030087
:1099C00040F2FC00C2F200001860204610BC704754
:1099D0002DE9F041044684B00E460AF0F9FA002C55
:1099E0002AD020460DF09CFEC16D03908D6800F0DA
:1099F000DFF8804604A850F8042D56630DF0A2FE4F
:109A00002E6801212046B0472B68074603212046D7
:109A10009847002106462D682046A847054620465F
:109A200000F05EFB2046009541463A46334610F072
:109A300087F8204603F054F80AF0C0FA04B0BDE8F5
:109A4000F08100BF10B5044682B080B10AF0C0FAC0
:109A500020460DF065FE02ABB0F87C4043F8040DE3
:109A60001846C4F3C0040DF06DFE0AF0A7FA2046B4
:109A700002B010BD70B58AB005460C460DF050FE20
:109A80000AABC26D43F8280D684696680DF05AFE81
:109A90000195032C05D8DFE804F00F0C090217200C
:109AA0000290716801A888470AB070BD1521029123
:109AB000F7E716230293F4E718220292F1E700BFBA
:109AC0002DE9F047466886B00446304601F0EAFAD0
:109AD00080460DF025FE06AD034645F8140D476E91
:109AE000D3F84890D3F880A028460DF02BFE2068CC
:109AF0000E38142815D8DFE800F00B3414141414B1
:109B00001C1C141C141414141414202C14143100D0
:109B1000E3685868002804DD1968092935D00A2946
:109B200042D037B1C4F804802046B84706B0BDE83B
:109B3000F087204603F064FCF8E7E1680029F5D0DF
:109B4000BAF1000F21D0B2451FD0504600F058FDA9
:109B5000ECE7404621460FF0B7F8E7E7C4F80C9071
:109B6000E4E76FF07042914504D0484608F078FF72
:109B70000CF012FA002FD9D094E80F0002AC84E860
:109B80000F0003962046B847D0E7304600F0E8FCC7
:109B9000044640460DF0C4FD02462846C2F8804007
:109BA00001920DF0CFFDC1E7304600F0A1FCEFE7D8
:109BB00008B50346408E00F0200188B210B1B3F919
:109BC000540000B108BD586B0AF068FD023008BDB2
:109BD0002DE9F04784B00446924689460DF0A0FD79
:109BE000034603C8DA6D0093956804AE06E90300E6
:109BF00068460DF0A7FD00212B68204698470646D1
:109C0000204601F03BFB044680B3BDF90880BDF956
:109C10000A7007E001A80DF095FD204601F074FAE6
:109C2000044618B320460DF07BFDB0F902500190B8
:109C3000ED1BB54201888288ECD1806A0BB212B26A
:109C4000C8EB03010306C8EB020207D5DAF80020CF
:109C50009142DFDC0139CAF80010DBE7D9F80000D7
:109C60008242D7DB531CC9F80030D3E704B0BDE80B
:109C7000F08700BF2DE9F04F89B005460C460DF086
:109C80004FFDC36D05909E680121326828469047BC
:109C90003768032180462846B84733680221814649
:109CA000284698470021366807462846B0470646AA
:109CB000059801F077F88246059801F07BF8059B3E
:109CC0008446588E00F020018AB2D2B1B3F8540015
:109CD000B3F85810002851D082B21FFA82FB0BEB68
:109CE000010081B2D86E88B101910392CDF808C00D
:109CF00001F086F880B203460199039ADDF808C0A6
:109D000005E093461146D86E0028EDD103461FFAB0
:109D100086FE0AF1FF3A71440CF1FF3CC9EB0A09D7
:109D20000EF1FF3E5B18DE44C7EB0C011FFA89F908
:109D30001FFA88F822806080E3806181A4F812E035
:109D4000A4F80480A4F80890A4F80C80A4F810905B
:109D5000E68105A80DF0F6FCB4F90C20B4F910303A
:109D60000692284606A907AA0793FFF731FF06982F
:109D70000799A081218209B0BDE8F08F586B01914D
:109D8000CDF808C00AF08AFC0199DDF808C0831CF0
:109D90009AB25018059B934681B2B4E72DE9F0477B
:109DA00046688CB0054630460DF0BAFCC26D019095
:109DB000D0F88840D0F88070D0F86880B0F87C90F7
:109DC000002A6DD0D2F800A001A80DF0BBFC14B998
:109DD00009E024683CB16368284698470028F8D019
:109DE0000CB0BDE8F08728680B381F284ED8DFE894
:109DF00010F05900D900C7004D00C1004D00AF0060
:109E00004D004D00A5004D004D00A2004D004D003D
:109E10004D004D004D004D0082004D0020004D00D2
:109E20004D004D004D004D0074004D004D004D00A3
:109E30006600EC6854B36068314600F093FA00287D
:109E400040F0DF8030460DF06BFCB0F87C100290E3
:109E500001F0080293B233B121F00801A0F87C10A0
:109E6000304602F03DFE02A80DF06CFC2068314641
:109E700000F068FA50B130460DF052FC22680290B2
:109E8000034602A8C3F880200DF05CFC304629464A
:109E90000EF01AFF0028A3D0284603F0B1FA9FE77E
:109EA000924691E730460DF03BFC034600F170000E
:109EB00001930DF05BFD01A80DF044FCE6E7304690
:109EC0000DF02EFCE9680190002900F0EB80C0F84D
:109ED000841001A80DF036FC82E7EB68022B7FF4BA
:109EE0007FAF0CA9272041F8240DA868059606939A
:109EF00000F00AFA74E7EC68012C00F09580002E5F
:109F00003FF46EAF0AF064F830460DF009FCB0F88B
:109F10007C30029003F0080291B231B123F00803C3
:109F2000A0F87C30304602F0DBFD02A80DF00AFC00
:109F30000AF044F854E7C5F80C8051E7304607A909
:109F4000FFF798FE08AB03CBEA681060516047E763
:109F50003046EC680DF0E4FB02902189012905D11F
:109F6000B0F87C3043F48072A0F87C2002A80DF099
:109F7000E9FB8BE7BAF1000F88D03046D04785E780
:109F800009F0080081B2002980D1EB68DA68002A64
:109F90003FF47CAF107A00283FF478AF304600F0F1
:109FA0002FFB73E73046D5F80C800DF0B9FB0CACF5
:109FB000B0F87C7044F8280D20460DF0C3FBE9682A
:109FC00000293FF40DAF98F80830002B58D007F067
:109FD000080083B2002B61D0304601F0DDFA07F4AF
:109FE0008872B2F5887F7FF4FBAE07F080018BB2F8
:109FF000002B7FF4F5AE30464146052200F078FB99
:10A00000EEE630460DF08CFBB0F87C10029001F0CB
:10A0100008039AB2002AA9D141F00801A0F87C10E7
:10A02000304602F05DFDA1E7384600F05FFE0028F3
:10A030003CD0384600F0E4FA384600F093FEC0B950
:10A0400026B9002F7FF4CCAEEF60C9E609F0C0FF5F
:10A0500030460DF065FBB0F87C10029001F008036B
:10A060009AB2002A33D002A80DF06CFB09F0A6FFCB
:10A07000E7E7384621460EF0E3FD002EE1D0E5E7A4
:10A0800030460DF04DFBB0F87C20029022F4807138
:10A09000A0F87C1020460DF055FBA1E6304600F0FC
:10A0A000AFFA99E7D0F88420EA6012E7404600F062
:10A0B00057FA074630460DF033FB024601A8C2F8B6
:10A0C000807001920DF03EFB002EBAD0BEE741F049
:10A0D0000801A0F87C10304602F002FDC3E700BF83
:10A0E00070B586B006460DF01BFB034606A89C6EB5
:10A0F00040F8183D6846DD6E0DF024FB84B96DB163
:10A10000304601A9FFF7B6FDBDF90A20BDF90630BA
:10A11000BDF908102846D21A00F018FC06B070BD30
:10A1200001A93046FFF7A6FD2046BDF90810BDF98C
:10A130000A2000F00BFCBDF90C00BDF90810BDF9B8
:10A140000E20BDF90A30411AD21A204601310132DF
:10A1500000F064F9002DE1D0D6E700BF2DE9F0470B
:10A160008CB0814616461D46DDF854800F4609F036
:10A170002FFF149C484800941A9C029048F4805386
:10A180006034019332460394484639462B4602F028
:10A19000ABFC064628B909F011FF30460CB0BDE80B
:10A1A000F0870DF0BDFA0DF13009179904903022B7
:10A1B0000EF080FD394D59F8207D1999DFF8E4A0A3
:10A1C00079660FCD07F134040FC40FCD0FC495E8A5
:10A1D0000300DAF80030169AFB65002584E80300D6
:10A1E000A7F87C20C7F88050FD66C7F8885048461D
:10A1F0000DF0A8FA304607A9FFF73CFDBDF9221083
:10A20000BDF92440BDF92630BDF920000096221A80
:10A210005C1A631C41F282740194214C0395013253
:10A22000029402F061FCDAF8001004464B683046F4
:10A23000984730460DF074FA0246484694660492F8
:10A240000DF080FA42F2040008EA000191B109F031
:10A25000BFFE30460DF064FA036F059005A8069323
:10A260000DF070FA06A8189908F0FAFC30B909F058
:10A27000A5FE90E7304600F025FDE8E730460DF0FA
:10A280004FFA069A0590026705A80DF05BFA304672
:10A2900002F026FCEBE700BF9D9D000808010020AE
:10A2A000C19A00083001002010B588B00A9C0094C3
:10A2B0000B9C01940C9C02940D9C03940E9C0494A2
:10A2C0000F9C059400240694FFF748FF08B010BDCA
:10A2D00030B5044683B00D4608B903B030BD09F06F
:10A2E00077FE20460DF01CFAB0F95A300190AB42CF
:10A2F00004D0A0F85A50204602F0F2FB01A80DF05D
:10A3000021FA09F05BFEE8E770B50D4C2368132BCA
:10A3100006460D4600DD70BD0DF0F8F901696E606E
:10A3200041B122682846531C236088472068411E9B
:10A33000216070BD2846BDE8704003F061B800BFE1
:10A34000C05C002010B50C4600B119B9002010BD4A
:10A350000028FBD00DF0DAF98069A042F8D1012085
:10A3600010BD00BF884210B50C4608D048B109B9ED
:10A3700007E030B10DF0CAF980698442F9D10120BB
:10A3800010BD002010BD00BF38B5054609F020FE05
:10A3900040F26413C2F200031868446C456401F093
:10A3A000ABFD09F00BFE204638BD00BF10B50446DA
:10A3B00082B009F00DFE1CB909F000FE02B010BD1C
:10A3C00020460DF0ADF9836A0190DB0703D501A8A3
:10A3D0000DF0B8F9F0E720460FF046FE019A064B63
:10A3E000906A196840F001000131906220461960BE
:10A3F00002F076FBEBE700BF0080022010B50446B8
:10A4000009F0E6FD2CB120460DF080F9846A04F0D5
:10A41000010409F0D3FD204610BD00BFF0B504468D
:10A4200083B00D46164600B309F0D2FD20460DF06C
:10A4300077F9034602A8B3F904E0B3F90020B3F9B1
:10A440000210B3F9067040F8043DC2EB0E027B1A0D
:10A45000D143DA434D1996190DF074F92046294677
:10A46000324600F0E3F909F0A9FD03B0F0BD00BFEA
:10A4700070B505460E4609F0ABFD2846FF2101F0F8
:10A4800011F8044636B168B109F098FD201C18BFD8
:10A49000012070BD0028F7D000F044FC204602F0F7
:10A4A000B1FEF1E7284621460EF04CFEECE700BF76
:10A4B00070B505460E4609F08BFD2846FE2100F0DA
:10A4C000F1FF044636B168B109F078FD201C18BFD1
:10A4D000012070BD0028F7D000F024FC204602F0D7
:10A4E00091FEF1E7284608210EF02CFEECE700BFB4
:10A4F00038B5054608B9284638BD09F069FD284633
:10A500000FF096FD054628BB28460FF083FD8542D7
:10A5100014BF054600252C46204600F0F3FBB8B9D1
:10A520002046ACB10FF060FD10B920460FF072FD6F
:10A53000844214BF04460024A542EDD1284600F011
:10A540005FF8002818BF002509F038FD284638BDFF
:10A550002546F3E70FF048FD0028D8D1D4E700BF27
:10A5600070B5064610B90546284670BD09F030FDA5
:10A5700030460FF05DFD0446002834D130460DF022
:10A58000C5F8C569AC4208BF00252C46204600F03E
:10A59000B9FB00282DD1204674B10DF0B7F8036A3D
:10A5A0001BB930460DF0B2F8C3699C4214BF1C467B
:10A5B0000024A542EAD125B9002509F0FFFC284670
:10A5C00070BD0E4C2846266802F08AFB0130F4D09C
:10A5D000284602F085FB2060284600F011F826602E
:10A5E0000028E9D1E9E70DF091F8056A002DC9D1FD
:10A5F000C4E72546002DDFD0E3E700BFDC7F022063
:10A600002DE9F04186B00025044602950395049596
:10A61000059509F0DDFC002C3CD0244EDFF890803D
:10A62000336858F82300A04234D01E2105958DE8E8
:10A630001100029102AD002833D1012220462946A3
:10A640000592FFF761FE059F2FBB3068202648F872
:10A65000204004E000AA02960592FFF755FE20462E
:10A6600000F020FD294604460028F3D1009C204636
:10A6700000F03CFB78B1202604E000AB0296059385
:10A68000FFF742FE204600F00DFD29460446002853
:10A69000F3D100E0012709F091FC384606B0BDE88F
:10A6A000F0812946FFF730FEC7E700BFDC7F0220BC
:10A6B000CC7F022010B50B4B19684B7C012B024656
:10A6C00088BF6FF0704401D9204610BD0648074985
:10A6D00050F8230051F8234041F8232002F000FAFB
:10A6E000F2E700BF64010020C07F0220E87F022063
:10A6F0002DE9F04385B005460C4616461F4600F08E
:10A7000041FB00283FD0254A2068B2F90010B2F979
:10A7100002306268C1EB0008C3EB0209002E2AD1A7
:10A72000002F22D0284669466C4600F0A1FBBDF8F8
:10A730000200411ECF19ADF80670284600F0B2FCA9
:10A7400002A900F095FB684641464A4609F03AFFE7
:10A7500002A80146324608F0C1FA684602A909F08B
:10A7600049FE10B905B0BDE8F083284641464A4687
:10A7700000F098FAF6E7284669466C4600F078FB48
:10A78000002FDAD0D3E70121284600F009F894E839
:10A790000600024B19805A80E4E700BFC45C002029
:10A7A000F0B5104E104C85B005460F4609F010FC70
:10A7B000316854F82100A84200D038B90B4844F859
:10A7C0002150077009F0FAFB05B0F0BD04A9182369
:10A7D00041F8103D6946FFF797FD3168002244F8C3
:10A7E0002120EBE7DC7F0220F87F0220E07F0220BF
:10A7F00030B50C4D0C4C85B009F0EAFB2B6854F8D1
:10A80000230050B104A9182241F8102D6946FFF722
:10A810007BFD2868002344F8203009F0CFFB05B009
:10A8200030BD00BFDC7F0220F87F02202DE9F0411F
:10A8300052EA01038CB00C46054600D010B90CB0AA
:10A84000BDE8F081039209F0C3FB28460CF068FFD5
:10A85000064603C80DF1200806AF88E803000596F8
:10A8600087E80300039A4CB1B36A03F42070802890
:10A870005CD0BDF81C106418ADF81C4052B1B16A30
:10A8800001F4A064B4F5807F4AD0BDF81E30D21820
:10A89000ADF81E20B46AE2033CD497E80300A30796
:10A8A00086E803000BD50AA841463A4609F09CFE0B
:10A8B000059E0AA8B169326A02F020F8059EBDF92A
:10A8C0001EC0BDF92640BDF91AE0BDF91C00BDF956
:10A8D0001870BDF92010BDF92220BDF92430C4EB59
:10A8E0000C0400940CACC31AC2EB0E023046791A69
:10A8F0000FF0CEFA54F81C0D0146083008F0A4FA07
:10A900002846052102F00EF820460CF01BFF09F046
:10A9100055FB94E7284601F019FC059EB46ABCE794
:10A92000BDF81A00811AADF81A10B3E7BDF8183057
:10A93000181BADF81800A1E700B585B026230391D8
:10A94000694600930FF082FF05B000BDF0B50446E4
:10A9500083B00D46164608B903B0F0BD09F038FBC8
:10A96000204600F09FFB10B909F028FBF4E70CF03B
:10A97000D7FE009020460CF0D3FE02ABB0F9027077
:10A9800053F8082DB0F90010B2F900E0B2F9023026
:10A990000190C1EB0E01DA1B68464D1996190CF0B7
:10A9A000D1FE01A80CF0CEFE20462946324600F02A
:10A9B00023F9D9E72DE9F04FB5B0002306908A4678
:10A9C00014461C931D931E931F93002800F01181C1
:10A9D0008B4606980CF0A4FE594622460A9009F0D0
:10A9E000F1FD0A9822465946083009F0EBFD0A9815
:10A9F000C169036A05910AA807930CF0A3FE0598A4
:10AA000000222092219222922392002800F0E080DE
:10AA100005980CF085FE594622460B9009F0D2FDB0
:10AA20000B9859460830224609F0CCFD0B99CB69AA
:10AA30000A6A04930BA808920CF084FE0499002083
:10AA40002490259026902790002900F0B0805D4644
:10AA500004980CF065FE294622460C9009F0B2FDE0
:10AA60000C9829460830224609F0ACFD0C9B186A68
:10AA7000DA6909900CA802920CF064FE029B002196
:10AA8000289129912A912B91002B7FD00DF16808F4
:10AA900002980CF045FE294622460D9009F092FDE1
:10AAA0000D9829460830224609F08CFD0D9A106A4F
:10AAB000D2F81C9003900DA80CF044FE00212C91BC
:10AAC0002D912E912F91B9F1000F50D003274846B8
:10AAD0000CF026FE294622460E9009F073FD0E98D2
:10AAE00029460830224609F06DFD0E9B1A6ADE6980
:10AAF00001920EA80CF026FE00203090319032908A
:10AB0000339036B330460CF00BFE294622460F90A8
:10AB100009F058FD0F9822462946083009F052FDE9
:10AB20000F99D1F81CB0D1F820A00FA80CF00AFEA4
:10AB3000584629462246FFF73DFF304630A9564683
:10AB40003097CDF8CC801A951B94FFF7DDFB002ED3
:10AB5000D8D14846DDF804902C9718AB2CA92F9338
:10AB600018951994FFF7D0FBB9F1000FAFD1039AF4
:10AB700002980292032316AA28A928932B921695CD
:10AB80001794FFF7C1FB0298002881D1099B049814
:10AB9000049324A9032214AB2492279314951594AB
:10ABA000FFF7B2FB049900297FF452AFAB46089A35
:10ABB00005980592032312AA20A920932392CDF889
:10ABC00048B01394FFF7A0FB059800287FF420AF4E
:10ABD000079B069806931CA9032210AB1C921F9397
:10ABE000CDF840B01194FFF78FFB069900297FF450
:10ABF000F0AE35B0BDE8F08F2DE9F0438BB0002307
:10AC000005460C46164606930793089309930028B9
:10AC10003AD009B9002A37D028460CF081FD074602
:10AC200003C80DF1080888E803003246384621467B
:10AC3000019709F0C7FC01980AAF21460830324657
:10AC400009F0C0FC57F8240DD0F81C9038460CF0E1
:10AC500079FD324648462146FFF7ACFE28460CF007
:10AC60005FFD826A0190920701D5816979B9384602
:10AC70000CF068FD032204AB284606A9069209934E
:10AC800004940596FFF740FB0BB0BDE8F083026A21
:10AC900001F004FD019B404699691A6A01F0FEFC2F
:10ACA000E5E700BF70B506460D46144609F090F979
:10ACB000304629462246FFF79FFFBDE8704009F065
:10ACC0007DB900BF10B5044600B910BD09F080F988
:10ACD00020460CF01BFD836A23F4005121F004028E
:10ACE0008262BDE8104009F069B900BF10B50446A2
:10ACF00009F06EF9204601F013FA044609F05EF9F6
:10AD0000204610BD00B585B008B905B000BD04A946
:10AD10001F2241F8102D00236946039301F0F2FD34
:10AD20000398F2E710B5044682B008B902B010BD2E
:10AD300009F04EF920460CF0F3FC826A019091076D
:10AD400005D401A80CF0FEFC09F038F9EEE722F07A
:10AD500002018162026A816901F0D0FD01A80CF054
:10AD6000F1FCF1E747F6DC72C2F2020247F6CC735F
:10AD7000C2F20203116853F82120131A58425841B5
:10AD8000704700BF47F6DC72C2F2020247F6F87362
:10AD9000C2F20203116853F82120131A5842584195
:10ADA000704700BFB0F90420B0F90030D01A01306C
:10ADB000704700BFB0F90620B0F90230D01A013058
:10ADC000704700BF10B5044682B009F001F914B90C
:10ADD00001F0A0FF044620460CF0A2FC02ABB0F943
:10ADE0000020B0F9041043F8040D881A441C1846DA
:10ADF0000CF0A8FC09F0E2F8204602B010BD00BF3C
:10AE000010B5044682B009F0E3F814B901F082FFEE
:10AE1000044620460CF084FC02ABB0F90220B0F9E5
:10AE2000061043F8040D881A441C18460CF08AFCDE
:10AE300009F0C4F8204602B010BD00BF10B50446AA
:10AE400009F0C6F844B1084B186848B10CF05EFC34
:10AE5000024603CA20606160BDE8104009F0AEB848
:10AE600002480168886CF1E7BC7F02206401002081
:10AE700038B505460C4668B161B109F0A9F8284615
:10AE80000CF044FC034603CB20606160BDE8384011
:10AE900009F094B838BD00BF2DE9F0470D460CF01D
:10AEA00035FCD0F81C90B9F1000F31D048460CF0B9
:10AEB0002DFCC46924B90AE00CF028FC046A34B102
:10AEC000204600F0BDF985422046F5D121E04846F4
:10AED0000CF01CFCD0F81CA0BAF1000F10D05046AA
:10AEE0000CF014FCC46924B916E00CF00FFC046AE1
:10AEF00094B1204600F0A4F985422046F5D144B92A
:10AF000048460CF003FCD0F82090B9F1000FCDD1E9
:10AF100000242046BDE8F08750460CF0F7FBD0F83F
:10AF20001C80B8F1000F11D040460CF0EFFBC46953
:10AF300024B914E00CF0EAFB046A84B1204600F066
:10AF40007FF985422046F5D1002CE2D150460CF025
:10AF5000DDFBD0F820A0BAF1000FC0D1D0E7404609
:10AF60000CF0D4FBC7698FB138460CF0CFFBC46935
:10AF700024B914E00CF0CAFB046A84B1204600F046
:10AF80005FF985422046F5D1002CC2D140460CF035
:10AF9000BDFBD0F82080B8F1000FC5D1D6E7384608
:10AFA0000CF0B4FBC6698EB130460CF0AFFBC4693F
:10AFB00024B912E00CF0AAFB046A74B1204600F038
:10AFC0003FF985422046F5D1002CA2D138460CF03D
:10AFD0009DFB076A002FC7D1D8E730462946FFF707
:10AFE0005BFF0446002894D130460CF08FFB066AC4
:10AFF000002ED9D1EAE700BF70B506460D460CF029
:10B0000085FBC46924B90BE00CF080FB046A3CB1F9
:10B01000204600F015F9A8422046F5D1204670BD23
:10B0200030460CF073FBC669EEB130460CF06EFB97
:10B03000C46924B90AE00CF069FB046A34B1204603
:10B0400000F0FEF885422046F5D1E7E73046294674
:10B05000FFF722FF04460028E0D130460CF056FBF3
:10B06000066A002EE1D10024204670BD10B50446CA
:10B0700040B108F0ADFF2046FF21FFF7BDFF0446B9
:10B0800008F09CFF204610BD10B5044640B108F002
:10B090009FFF2046FE21FFF7AFFF044608F08EFF1A
:10B0A000204610BD10B5044638B108F091FF204687
:10B0B0000CF02CFB846908F081FF204610BD00BF16
:10B0C000074B186810B5846C44B108F081FF204626
:10B0D0000CF01CFBB0F9004008F070FF204610BDDA
:10B0E00064010020074B186810B5846C44B108F067
:10B0F0006FFF20460CF00AFBB0F9024008F05EFF3B
:10B10000204610BD6401002010B5044608F060FF21
:10B110001CB120460CF0FAFA046A08F04FFF2046F2
:10B1200010BD00BF38B504460D4608B9204638BDED
:10B1300008F04EFF20460CF0E9FA846A14F020046F
:10B1400005D000F1080303CB01242860696008F0F2
:10B1500035FF204638BD00BFF0B50C4687B0054628
:10B16000B8B1B1B1FF2100F09DF9FE210646284695
:10B1700000F098F904A907462846FFF779FE28460B
:10B18000694600F03FF837B906BB6A4603CA20603B
:10B19000616007B0F0BD384602A9FFF769FEBDF94E
:10B1A0001010BDF912204942524202A809F00AFAD1
:10B1B000384600F055F800F082008228E4D1BDF84E
:10B1C0000830591EADF80410002EDED0304602A91A
:10B1D000FFF74EFEBDF91000BDF912204142524268
:10B1E00002A809F0EFF9304600F03AF800F4817354
:10B1F000B3F5817FC9D1BDF80A10481EADF806002D
:10B20000C3E700BF00B585B004AB142203916946C3
:10B2100043F8102D01F076FB05B000BD00B540F2FB
:10B220006413C2F2000385B004A91A6803901423C2
:10B2300041F8103D906C694601F064FB05B000BD1B
:10B2400000B585B004A91523002241F8103D6946D8
:10B2500001920292039201F055FB039805B000BDE4
:10B2600010B5044638B108F0B3FE20460CF04EFA93
:10B27000048D08F0A3FE204610BD00BF10B50446A3
:10B2800038B108F0A5FE20460CF040FAC46908F079
:10B2900095FE204610BD00BF2DE9F04F8DB00C4645
:10B2A0000CF03EFA0CABC26943F8240D184600922C
:10B2B0000CF048FA0098002800F0E9800098FFF7A9
:10B2C000BFFFA04200F0A18000980CF029FA0146CF
:10B2D00004A8D1F81C8004910CF034FAB8F1000FE6
:10B2E00000F0CD804046FFF7ABFF844200F08B803A
:10B2F00040460CF015FA034605A8D3F81C900593B8
:10B300000CF020FAB9F1000F00F0B0804846FFF7CA
:10B3100097FF844276D048460CF002FA024606A80F
:10B32000D2F81CA006920CF00DFABAF1000F00F052
:10B3300094805046FFF784FF844262D050460CF060
:10B34000EFF9014607A8D1F81CB007910CF0FAF903
:10B35000BBF1000F78D05846FFF772FF84424FD000
:10B3600058460CF0DDF9034608A8DA690893019203
:10B370000CF0E8F9019800285ED00198FFF760FF13
:10B38000844200F08D8001980CF0CAF9014609A8AA
:10B39000CE6909910CF0D6F9002E46D03046FFF761
:10B3A0004FFF84427AD030460CF0BAF903460AA81F
:10B3B000DD690A930CF0C6F9002D30D02846FFF75E
:10B3C0003FFF844268D028460CF0AAF902460BA839
:10B3D000D7690B920CF0B6F967B91AE021463846E6
:10B3E000FFF75AFF01463846002953D10CF08EF979
:10B3F000076A77B13846FFF723FF8442EED1BB4698
:10B40000DA46D146C846CDF8008000980DB0BDE8B8
:10B41000F08F28460CF07AF9056A002DCED130461F
:10B420000CF074F9066A002EB8D101980CF06EF990
:10B43000006A01900028A0D158460CF067F9D0F8B6
:10B4400020B0BBF1000F86D150460CF05FF9D0F868
:10B4500020A0BAF1000F7FF46CAF48460CF056F90B
:10B46000D0F82090B9F1000F7FF450AF40460CF0B7
:10B470004DF9D0F82080B8F1000F7FF433AF009879
:10B480000CF044F9036A0093002B7FF417AF0022FD
:10B490000092BAE70F46B2E72F46B0E73746AEE76D
:10B4A000019FACE738B504460D4640B108F090FD69
:10B4B00020462946FFF7F0FE044608F07FFD2046AF
:10B4C00038BD00BF40F26412C2F2000247F6C073FA
:10B4D0001068C2F20203417C53F82100704700BF9C
:10B4E00000B585B004A9172341F8103D0022694634
:10B4F000039201F007FA039805B000BD30B50C4681
:10B5000083B058B151B10CF00BF902AD214645F8AA
:10B51000040D01F013FA28460CF014F903B030BD05
:10B5200030B583B0054608F053FD104B1C685CB97C
:10B530000F4801688C6C08F04BFD3CB908F03EFDEB
:10B5400008F03CFD03B030BD08F042FD002DF5D001
:10B5500020460CF0E5F802AC294644F8040D01F051
:10B56000EDF920460CF0EEF8E8E700BFBC7F0220C2
:10B5700064010020826801684368891A002B21EA6F
:10B58000E17203DB9342C8BF42607047002343600F
:10B59000704700BF01F0A4BA30B5044683B008F08C
:10B5A00017FD1CB908F00AFD03B030BD20460CF0B1
:10B5B000B7F801460090006A38B38A6A120710D4BF
:10B5C0000CF0AEF8836A01901B0706D568460CF0B4
:10B5D000B9F801A80CF0B6F8E4E701A80CF0B2F84D
:10B5E00000998D6968460CF0ADF8204600F076FDB4
:10B5F0002946204600F008FD204601F071FA204659
:10B60000044900220FF01EFBCCE768460CF09AF8C4
:10B61000C8E700BF95B500082DE9F00145F6D04C0C
:10B6200045F6F04847F6F07747F6CC7147F6F872E2
:10B6300048F2000647F6BC7547F6E47447F6F47026
:10B64000C2F20201C2F20202C2F20008C2F2000C0F
:10B65000C2F20207C2F20206C2F20205C2F20204FC
:10B66000C2F20200002388F80030CCF800303B60C2
:10B670000B6013604B60536033602B60236003608A
:10B68000BDE8F001704700BF2DE9F043284D2B685D
:10B6900083B00446986C0CF043F8009020460CF000
:10B6A0003FF8014601900098083008F0A3FE0646D6
:10B6B00048B968460CF046F801A80CF043F830464B
:10B6C00003B0BDE8F08302AE2968019856F8082D52
:10B6D000D1F84C90D1F85080164F0146083208300E
:10B6E00007F07CFB68460CF02DF802A82B6850F898
:10B6F000042D3C60B2F90010B2F90220D9641A6539
:10B700000CF020F820460CF001F8806A0A490B4B37
:10B7100010F4803F08BF0B46204698472868002257
:10B72000C0F84C90C0F850803A600120C8E700BFD4
:10B7300064010020BC7F022029CF000825D7000823
:10B74000F0B585B006460BF0EBFF836A01909B07CE
:10B7500023D5C46901AD2CB91FE01C6A68460BF003
:10B76000F1FFACB120460BF0DBFF826A009002F0E3
:10B77000030103290346F0D10199083108F03AFE8C
:10B7800068B9009B1C6A68460BF0DCFF002CE9D10D
:10B7900028460BF0D7FF05B0F0BD01ADF8E70198E2
:10B7A000083003C802AF87E8030028460BF0CAFF41
:10B7B00068460BF0C7FF2046FFF766FF78B93046B2
:10B7C0000BF0AEFF019020460BF0AAFF019C009009
:10B7D000034697E80300083484E80300BDE72046E9
:10B7E0000BF094FF00902046FFF7AAFF20460BF0D5
:10B7F0008DFF009030460BF089FF0190DFE700BF1E
:10B80000F0B5044685B00E461746002834D02046D1
:10B810000BF086FF846A0090A107034626D5002F0F
:10B8200042D002AD284619463A4607F0D7FA3046CC
:10B83000294608F0DFFD00282ED0E207009B1DD42A
:10B84000002F45D0B7F90220B3F902109142B8BFDA
:10B850001146B6F9020081422BDDBDF80A40B6F967
:10B86000060022B2904201DB611EF1801C6A68462C
:10B870000BF068FF002CCAD105B0F0BDDC69002CCC
:10B88000F4D0204631462A46FFF7BAFF20460BF097
:10B890003DFF046A002CF4D1009B1C6A68460BF043
:10B8A00051FF002CB3D1E7E703C802AD85E80300E0
:10B8B000BDE7BDF80E40B6F9062021B28A42D5DDBB
:10B8C000F4801C6A68460BF03DFF002C9FD1D3E743
:10B8D000B3F90210BDE700BF2DE9F041044684B082
:10B8E0000F469046002847D000260CE0E00700995C
:10B8F0002FD4BDF80C20501C388001260C6A6846F5
:10B900000BF020FFE4B120460BF00AFF846A0090A0
:10B91000A3070146F2D5B8F1000F15D002AD2846B5
:10B92000424607F05BFA3846294608F063FD0028D6
:10B93000DCD100990C6A68460BF004FF002CE2D1C0
:10B94000304604B0BDE8F08103C802AD85E80300CD
:10B95000E9E7CC69002CD1D0204639462A46FFF7CA
:10B96000BBFF002818BF012620460BF0CFFE046A5B
:10B97000002CF1D10099DDE70646E1E7F0B5044679
:10B9800085B00E46174660B926E0E20700992AD432
:10B99000BDF80820501EB0800C6A68460BF0D2FE3D
:10B9A000D4B120460BF0BCFE846A00900146A0078B
:10B9B000F2D59FB102AD28463A4607F00FFA30465D
:10B9C000294608F017FD0028DFD100990C6A684667
:10B9D0000BF0B8FE002CE4D105B0F0BD03C902ADF8
:10B9E00085E80300EBE7CC69002CD5D02046314632
:10B9F0002A46FFF7C3FF20460BF088FE046A002C9E
:10BA0000F4D10099E2E700BFF0B5044685B00F46D7
:10BA1000002835D0002502AE20460BF081FE846A56
:10BA20000090A30708D503C886E8030038463146CE
:10BA300008F0E0FC48B90098046A68460BF082FE02
:10BA4000002CE9D1284605B0F0BDE407009805D4E4
:10BA5000BDF80C30591C39800125EDE7C469002C74
:10BA6000EAD0204639463246FFF736FF002818BF95
:10BA7000012520460BF04AFE046A002CF1D1DAE7DA
:10BA80000546DFE770B5044684B00E46B0B102AD9E
:10BA900020460BF045FE846A0190A10708D503C833
:10BAA00085E803003046294608F0A4FC40B9019817
:10BAB000046A01A80BF046FE002CE9D104B070BD69
:10BAC000E207019818D4B6F90230B0F902209A4280
:10BAD00009DDBDF80A40B6F9061022B29142E7DB53
:10BAE000631EF380E4E7BDF80E40B6F9061023B2FA
:10BAF0009942DDDDF480DBE7C469002CD8D0204614
:10BB000031462A46FFF77CFE20460BF0FFFD046A13
:10BB1000002CF4D1CBE700BFF0B585B005460C464C
:10BB200016460BF0F3FD836A0190980736D5B4F9F9
:10BB30000010B4F90420914230DCB4F90200B4F9E9
:10BB4000061088422ADC40F601021A40012A25D05C
:10BB500028460BF0E5FD02AD0346214628461A466D
:10BB6000019307F03BF9BDF90800BDF90C108842BC
:10BB700011DCBDF90A20BDF90E309A420BDC019AA6
:10BB8000946A44F22000204050B102F108000146BE
:10BB90002A4608F029FD01A80BF0D4FD05B0F0BD40
:10BBA000074B95E803001F8802F10805344301376D
:10BBB00085E8030094621F8007F052FEEBE700BFA8
:10BBC000D47F02202DE9F0438D4E06F1080797E857
:10BBD000030087B0336902AD85E8030063B93068BC
:10BBE00073880290B6F90610854C1BB299421EDA92
:10BBF000002007B0BDE8F083B289B6F9040073896C
:10BC0000511C8CB222B29042ADF80A30ADF8084017
:10BC1000E8DAF4893188631C9BB2ADF80810B6F9F4
:10BC20000610ADF80A301BB29942754CE0DBDFF824
:10BC3000D481D8F80020906C0BF072FDBDF808108C
:10BC4000024620880192814200F0C180D8F80000AD
:10BC5000ADF80C10806C10B913E0A06988B10BF03E
:10BC600055FD29460446006AFFF7CEFE0028F4D0B1
:10BC7000D8F80000BDF80810806CADF80C10002852
:10BC8000EDD1019B2946D869FFF7BEFE0028EFD110
:10BC9000B188BDF90820ADF80C1008B2824200F35B
:10BCA0008E80D8F80040A06C00282FD00DF110082D
:10BCB0000BF02CFD046A81466CB923E0E207009882
:10BCC0005DD4BDF81030591EADF80C10046A6846FA
:10BCD0000BF038FDB4B120460BF022FD846A0090D1
:10BCE000A107F3D503C888E803002846414608F0B9
:10BCF00081FB0028E2D10098046A68460BF022FD1F
:10BD0000002CE8D1D9F818000028D1D1019AD469C3
:10BD100034B30DF110080CE0E40700983FD4BDF8EF
:10BD20001030591EADF80C10046A68460BF00AFD7D
:10BD3000B4B120460BF0F4FC846A0090A307F3D55D
:10BD400003C888E803002846414608F053FB002852
:10BD5000E2D10098046A68460BF0F4FC002CE8D1AC
:10BD600001A80BF0EFFC306944F6206290423FF7E7
:10BD70003FAF95E8030087E80300012039E7C46975
:10BD8000002CA3D0204629464246FFF7F7FD204667
:10BD90000BF0BCFC046A002CF4D10098ACE7C46939
:10BDA000002CC1D0204629464246FFF7E7FD204639
:10BDB0000BF0ACFC046A002CF4D10098CAE795E8BB
:10BDC000030087E8030001A80BF0BCFC21E7D8F8CA
:10BDD00000106468886C039450B10BF097FC044623
:10BDE0002946006AFFF74EFEA0690028F5D1019AA6
:10BDF0002946D069FFF746FEBDF8081026E700BFC8
:10BE0000D45C002064010020F0B5374F3B6885B05A
:10BE10000546986C0BF084FC00F1080304463A6870
:10BE2000009493E80300083202AE86E8030092E82B
:10BE3000030083E8030068460BF084FC2C6820466E
:10BE40000BF06EFC836A019040F601011940012954
:10BE50000ED001A80BF076FC20460BF057FC806A50
:10BE60002249234A10F4803F08BF114620468847E4
:10BE7000204B186880B93968886C0BF051FC034678
:10BE800096E8030003F1080282E803006846009385
:10BE90000BF058FC05B0F0BD2046FFF751FC2046E2
:10BEA0000BF034FC8569046A002DE4D084B120468F
:10BEB0000BF02CFC806A00F00301032910D020460F
:10BEC000FFF73EFC20460BF021FC046A002CEED16B
:10BED00028460BF01BFC8569046A002DE6D1CAE7F1
:10BEE0002046FFF7D1FBEAE76401002025D70008D0
:10BEF00029CF000800800220F0B5404E336893F847
:10BF0000542087B0002A4BD1986C3D4F0BF008FCB1
:10BF1000044603C802AD85E80300684600940BF0B0
:10BF200011FC3C68002C2CD13468616C00295DD078
:10BF300008683A68496804AB03C3002A2ED010464B
:10BF40000BF0EEFB06ACB0F90220B0F9001044F89B
:10BF5000140D04A808F036FB20460BF0F3FB04A8F0
:10BF6000294606F071FF04A804F076FC07B0F0BD86
:10BF700006F06AFF0198846901A8002C33D00BF009
:10BF8000E1FB20460BF0CCFB836A01909B07014646
:10BF90002846EDD401A80BF0D5FBC5E7A26CCEE78F
:10BFA000596C39B3164C08682468496804AA03C25E
:10BFB000BCB120460BF0B4FB06ACB0F90220B0F9DE
:10BFC000001044F8140D04A808F0FCFA20460BF009
:10BFD000B9FB04A80B4906F037FF04A804F03CFCA9
:10BFE000C4E79C6CE5E70BF0ADFB9DE7284604F049
:10BFF00033FCBBE7034804F02FFCB7E764010020E3
:10C00000BC7F0220DC5C002070B50C4684B0054685
:10C0100009B904B070BD0BF083FB002203468461B4
:10C020000262204601930BF07BFB0199C4690290E8
:10C030008E6A44B320460BF073FB3307039038D469
:10C04000806A010727D402A80BF07CFB03A80BF041
:10C0500079FB20460BF05AFB046A03902CB9056269
:10C060000DE0046A0390002CF9D020460BF04EFB43
:10C07000826A1207F5D50399019B0D621C6201A823
:10C080000BF060FBC5E7C56101A80BF05BFB02A8E4
:10C090000BF058FBBDE70198029A0462D56101A834
:10C0A0000BF050FB02A80BF04DFB03A80BF04AFB72
:10C0B000AFE702A80BF046FB03A80BF043FB2046BA
:10C0C0000BF024FB036A0390002BC8D018460BF03A
:10C0D0001DFB036A0390002BF8D1C0E770B504463E
:10C0E0000BF014FB0546806900B970BD0BF00EFB28
:10C0F000C369A34206460CD013B910E0002BF4D05C
:10C1000018460BF003FB036AA342F7D1296A0162C8
:10C1100070BD18460BF0FAFA006AF06170BD70BD90
:10C12000094B196810B5044651B1814202D109E0AA
:10C130008C4207D008460BF0E9FA41690029F7D193
:10C14000002010BD012010BDD87F02202DE9F04F46
:10C1500004468BB010B90BB0BDE8F08F0BF0E0FADD
:10C16000826A0290910740F1D980406A002840F02D
:10C17000FD802046FFF782F88346002800F0CE803D
:10C1800058460BF0CDFA816A03908A0740F1BA80D5
:10C19000406A20B102F0D0FF039800224262584664
:10C1A000FFF76CF88246002800F0AC804FF00009E1
:10C1B00050460BF0B5FA836A04909B0740F19680D5
:10C1C000406A002840F0CC805046FFF757F8804680
:10C1D000002800F08B8040460BF0A2FA826A05909E
:10C1E000910777D5406A002840F0B4804046FFF7B9
:10C1F00045F8019000286DD001980BF091FA836A00
:10C2000006909A075CD5406A002840F09D8001980E
:10C21000FFF734F80646002852D030460BF080FA7B
:10C22000816A07908B0742D5406A002840F08680DB
:10C230003046FFF723F80546002838D028460BF093
:10C240006FFA826A0890910728D5406A00286FD15A
:10C250002846FFF713F8044600B320460BF060FAB7
:10C26000836A09909A0710D5406A00285AD120465F
:10C27000FFF704F8074640B13846FFF767FF384636
:10C280000BF044FA076A002FF6D109A80BF05AFA0E
:10C2900020460BF03BFA046A002CDED108A80BF014
:10C2A00051FA28460BF032FA056A002DC6D107A8CC
:10C2B0000BF048FA30460BF029FA066A002EACD192
:10C2C00006A80BF03FFA01980BF020FA006A0190E3
:10C2D000002891D105A80BF035FA40460BF016FA6C
:10C2E000D0F82080B8F1000F7FF475AF04A80BF0F0
:10C2F00029FA50460BF00AFAD0F820A0BAF1000F44
:10C300007FF456AF03A80BF01DFA58460BF0FEF968
:10C31000D0F820B0BBF1000F7FF432AF02A80BF0D1
:10C3200011FA18E702F008FF099FC7F824909EE76A
:10C3300002F002FF089CC4F8249089E702F0FCFE9A
:10C34000079DC5F8249073E702F0F6FE069EC6F836
:10C3500024905CE702F0F0FE0598C0F8249045E7D1
:10C3600002F0EAFE0499C1F824902DE702F0E4FE01
:10C37000029B00205862FCE62DE9F0470D4692B082
:10C380009246044610B912B0BDE8F0870BF0C8F928
:10C39000836A00909907024640F1D88006A8294692
:10C3A00006F01CFD002800F0D18068460BF0CAF9A9
:10C3B000204606A95246FFF7AFFB2046FEF75EFF78
:10C3C00005460028DFD028460BF0AAF90246019066
:10C3D000806A830740F1BE8008A806A906F0FEFC2B
:10C3E000002800F0B78001A80BF0ACF9284608A996
:10C3F0005246FFF791FB2846FEF740FF064600280D
:10C4000000F09C8030460BF08BF9816A0290024666
:10C41000880740F1AA800AA808A906F0DFFC0028D6
:10C4200000F0A38002A80BF08DF930460AA952460D
:10C43000FFF772FB3046FEF721FF0746002876D053
:10C4400038460BF06DF9836A03909907024640F174
:10C4500097800CA80AA906F0C1FC002800F0908083
:10C4600003A80BF06FF938460CA95246FFF754FBAE
:10C470003846FEF703FF8046002852D040460BF0B6
:10C480004FF902460490806A830740F184800EA829
:10C490000CA906F0A3FC00287DD004A80BF052F9EB
:10C4A00040460EA95246FFF737FB4046FEF7E6FE30
:10C4B000814600282DD048460BF032F9816A05905C
:10C4C0000246880774D510A80EA906F087FC00283C
:10C4D0006ED005A80BF036F9484610A95246FFF772
:10C4E0001BFB4846FEF7CAFE044650B1204610A981
:10C4F0005246FFF741FF20460BF008F9046A002C72
:10C50000F4D148460BF002F9D0F82090B9F1000FB1
:10C51000D1D140460BF0FAF8D0F82080B8F1000FE6
:10C52000ACD138460BF0F2F8076A002F88D13046BC
:10C530000BF0ECF8066A002E7FF464AF28460BF08F
:10C54000E5F8056A002D7FF43EAF1CE768460BF066
:10C55000F9F818E701A80BF0F5F828460BF0D6F823
:10C56000056A002D7FF42FAF0DE702A80BF0EAF863
:10C5700030460BF0CBF8066A002E7FF443AFDDE7C0
:10C5800003A80BF0DFF838460BF0C0F8076A002F5D
:10C590007FF456AFCBE704A80BF0D4F840460BF07D
:10C5A000B5F8D0F82080B8F1000F7FF467AFB8E796
:10C5B00005A80BF0C7F848460BF0A8F8D0F8209073
:10C5C000B9F1000F7FF477AFA3E700BF2DE9F04189
:10C5D0000C4686B0054617461E4611B906B0BDE8A2
:10C5E000F08108460BF09CF8D0F82880009018F0F5
:10C5F000020F024642D002A8294606F0EFFB0028AF
:10C600003CD040F6010308EA030001283ED0204652
:10C6100002A93246FFF780FA0099CC69002C2DD090
:10C62000BC422BD020460BF07BF8836A0190024677
:10C63000980727D504A802A906F0D0FB10B301A8DB
:10C640000BF080F8204604A93246FFF765FA204631
:10C65000FEF714FE054650B1284604A93246FFF7FE
:10C660008BFE28460BF052F8056A002DF4D12046C7
:10C670000BF04CF8046A0CB1A742D3D168460BF01A
:10C6800061F8ABE701A80BF05DF8F0E7009A02A8AB
:10C690009169126A3346FFF799FFBDE770B5064608
:10C6A00008460C4615460BF031F8836A13F4803FB8
:10C6B000304621462A460CBF20234FF48043BDE874
:10C6C0007040FFF783BF00BF2DE9F043804D87B076
:10C6D000044607F07DFC286830B9ABE00BF016F893
:10C6E0004069002800F0A6808442F7D1274600E088
:10C6F0001F4638460BF00AF88369002BF8D1754EB7
:10C700003268974200F0E1807068874214BF4FF0B2
:10C71000FF37012706A90B2341F8103D204603945B
:10C72000FDF7F2FD20460DF0D1FF20460AF0F8FF9C
:10C730000090406A002840F0A2806749674A0B6871
:10C7400067480021016052F82300844208BF42F884
:10C750002310644A52F823108C4200F09380624BFD
:10C760001868002130B14268944208BF41600068F7
:10C770000028F8D120460721FEF7DEF8DDF800801A
:10C78000D8F81C0000285AD120460AF0C9FF816958
:10C790000190002965D101A80AF0D4FF286858B19A
:10C7A0000AF0B4FF804640698442F8D120460AF07E
:10C7B000ADFF4269C8F814200098836ADA0703D5F0
:10C7C0004A4A1168481E10609B0645D468460AF024
:10C7D000B9FF474BDFF820811A882046541E1C8081
:10C7E0000BF09EF856F8277007F0F2FBD8F800001F
:10C7F00007B92F6887643C4600E00C4620460AF0E3
:10C8000085FF81690029F8D133689C4257D0314AAD
:10C810005068844257D006F00DF838460AF076FF8B
:10C82000D8F80030B0F90010B0F90220D9641A65C8
:10C8300007F0C4FB07F0C2FB07B0BDE8F083FFF7C9
:10C8400043FFD8F81C0000289ED0FFF73DFFD8F822
:10C850001C000028F3D197E7264B1A88511E198037
:10C86000B4E7026A2023FFF7B1FE20460AF04EFF2C
:10C870008046806950B9019B002199618BE702F0E5
:10C880005BFC5AE7002042F8230068E70AF03EFF0D
:10C89000C1698C4281460BD00029ECD008460AF0D1
:10C8A00035FF016A8C42F7D1D8F820200262E2E716
:10C8B00020460AF02BFF006AC9F81C00DBE7084697
:10C8C00007F02EFDA7E70120FAE71F4622E700BF89
:10C8D000D87F0220C07F0220DC7F0220CC7F022094
:10C8E000EC5C0020F87F0220F07F02200080022014
:10C8F000B87F0220D47F0220640100202023FFF7AC
:10C9000065BE00BF38B504460D4600B938BD07F016
:10C910005FFB20462946FDF7F7FCBDE8384007F0ED
:10C920004DBB00BF00B585B004AB019043F8101DAE
:10C930006946FDF7E9FC05B000BD00BF00234B8050
:10C940000B8030B402888588C4884088AA1A231ACC
:10C950008A80CB8030BC70472DE9F041074686B015
:10C960000C4610B906B0BDE8F08107F031FB38463F
:10C970000AF0D6FED0F82880009018F0020F2ED0D2
:10C9800003C804AE18F4803F86E803002DD17CB1C3
:10C9900020686168009C02AB03C3B4F90220B4F9BB
:10C9A000001002A807F00EFE304602A906F04CFA6D
:10C9B0003D4608E006F048FA0198846901A8C4B130
:10C9C0000AF0C0FE254628460AF0AAFE826A0190B7
:10C9D000930701463046EDD401A80AF0B3FE68463D
:10C9E0000AF0B0FE07F0EAFABCE73846FFF7AEFB04
:10C9F000CDE70AF0A7FE0D490B689D4202D04A68B8
:10CA00009542ECD140F6010008EA0001012905D069
:10CA1000384631462022FFF77FF8E0E7009B30469A
:10CA200099691A6A2023FFF7D1FDD8E7C07F022059
:10CA300003680E2B10B5044633D00F2B19D00E3BD4
:10CA40006068E1681A2B11D8DFE803F03410101089
:10CA500010100E10103910101010101010101010AF
:10CA60003B10101010103F00FEF748FD0022E2605E
:10CA700010BD194A436811688B422BD0506883421D
:10CA800014BF4FF0FF330123144A52F823006FF014
:10CA900070418842EAD007F015FC09F07DFA23685E
:10CAA000CDE7C1684B68012BE2D10868BDE81040B2
:10CAB00007F05EBD2146BDE810400DF0C7BEE06046
:10CAC00010BD6FF07040E06010BD0021BDE8104067
:10CAD000FFF742BF0023D7E7C07F0220E87F022094
:10CAE0000021FFF739BF00BF2DE9F04F87B09A460C
:10CAF00006460F469146109D07F06AFA724BD3F82E
:10CB0000008025B16A1C00F0DC802C4619E06F48DB
:10CB1000018861B913982C300BF02EF804460028D8
:10CB200036D107F04BFA204607B0BDE8F08F684ACF
:10CB3000684813685C7C50F82440611CEAD0002CE3
:10CB4000E8D020460AF0ECFDB0F90050B0F9021030
:10CB5000019076197F18B9F1000F05D1B0F9049052
:10CB6000C5EB090202F10109BAF1000F05D1B0F9D4
:10CB700006A0C1EB0A0303F1010A01A80AF0E2FDD5
:10CB800013982C300AF0F8FF254604460028C8D038
:10CB90004E490A88531C0B800AF0C2FD1199826A23
:10CBA00043F69F7341EA0808C0F2070308EA03034B
:10CBB00042EA030106EB090C129A81620DF1180B8F
:10CBC000BA440CF1FF390AF1FF3A4BF8180DA0F8FE
:10CBD000049006804780A0F806A0026168460AF02B
:10CBE000B1FD3D4B186800285BD11C6020462946EA
:10CBF000FFF70AFA18F0200F2FD118F0010F0ED10D
:10CC000018F0400F12D118F0020F15D106A901201B
:10CC100041F8100D20460394FDF776FB81E72F487D
:10CC20000368591C18F0400F0160ECD020460EF04C
:10CC30003DF818F0020FE9D020460AF071FD0346D6
:10CC400068469A6A009342F0020199620AF07AFDFE
:10CC500020460021FFF780FED8E71D4E07F0B8F907
:10CC600030682546846400E01D4628460AF04EFDE3
:10CC70008369002BF8D1174A11688D421BD0506888
:10CC800085421CD005F0D6FD20460AF03FFD3368F2
:10CC9000B0F90010B0F90220D9641A6507F08EF9D6
:10CCA000ABE70AF033FD064620460AF02FFD716916
:10CCB000416174619AE7184607F032FBE2E7012010
:10CCC000FAE7002526E700BFE47F0220B87F0220B4
:10CCD00064010020C07F0220D87F02200080022053
:10CCE00010B5044600E01C4620460AF00FFD83699B
:10CCF000002BF8D1064A11688C4206D05068844255
:10CD000014BF4FF0FF30012010BD184610BD00BF0A
:10CD1000C07F022040F26413C2F200031868806CE6
:10CD2000704700BF10B50E4B186890F8540050B112
:10CD30000C4C6169012907DD481E6061002010BDAF
:10CD4000FFF7DAF8012010BD2269531C2361FEF7BA
:10CD500039FF0028F4D161694A1E626110BD00BF2D
:10CD600064010020D45C00202DE9F043DFF8B48199
:10CD7000D8F8002092F8543089B004464BB1654D84
:10CD80006869411C0129696107DD012009B0BDE81E
:10CD9000F083FFF7B1F80120F8E7906C5E4E0AF0DF
:10CDA000BFFC337801904FF0FF322A61002B60D036
:10CDB000083003C804AE86E803001CB130462146A3
:10CDC00006F042F8D8F80070796C002900F09080E5
:10CDD000524F0868019C49683A68029406AB03C345
:10CDE0000DF10809002A68D1B4F90220B4F9001045
:10CDF00006A807F0E7FB304606A906F025F84846E6
:10CE00000AF0A0FC3F680DF10C0947BBD8F8007090
:10CE1000BF6C09E006F018F8039CA4694846002C92
:10CE200030D00AF08FFC274638460AF079FC826A37
:10CE30000390930701463046ECD448460AF082FC42
:10CE40006A69531E6B610020A0E705F0FDFF039C9B
:10CE5000A4694846002C39D00AF074FC27463846AD
:10CE60000AF05EFC826A0390920701463046ECD4D9
:10CE7000E3E7816A11F0020632D003C804AE86E807
:10CE800003009AE70AF05EFC254801688F4202D051
:10CE900043689F42D4D1D8F800201E4C92F85430F9
:10CEA00096E8030085E80300002BCCD060690128D8
:10CEB00023DD01386061002068E748460AF042FC43
:10CEC00038680AF02DFC044602908DE70AF03AFC1F
:10CED000134801688F4299D043689F42B0D195E7CB
:10CEE0006B6901A85A1E6A610AF02CFC30464DE7B6
:10CEF00001A80AF027FC094F84E721694A1C226136
:10CF0000FEF760FE00287FF444AF6369591E61613B
:10CF10003CE700BFD45C0020E17F0220BC7F022000
:10CF2000C07F0220640100202DE9F04F89B0054642
:10CF30000AF0F6FB00F10802034692E803001F69BD
:10CF4000019302AC84E8030001A89E6A0AF0FAFB90
:10CF50000FB1B10702D409B0BDE8F08F294F2E21DF
:10CF600028460DF087FC3878411C16F4805939703A
:10CF70002AD12046FFF7F8FEF0B1234EDFF88CB03F
:10CF80004FF00F0A0595CDF810A0079407F07AF935
:10CF90003368DFF87880C3F84490284604A9FDF789
:10CFA000B3F9326892F8540030B1DBF81420012A4A
:10CFB00019DD501EC8F81400397828464B1E2F2161
:10CFC0003B700DF057FCC6E70F21049105950794BF
:10CFD00007F058F90C4B18680022426404A928464F
:10CFE000FDF792F9E8E7DBF810104B1CCBF8103096
:10CFF000FEF7E8FD10B9D8F81420DAE7FEF77CFF59
:10D00000C0E700BFE17F022064010020D45C002063
:10D010002DE9F04788B006AE03900AF081FB00F1DD
:10D020000802034692E803009F6A049386E803001F
:10D0300004A8D3F818801C690AF084FB44F220008D
:10D040003840002832D0C4B1039D09E005F0FCFE51
:10D0500005998C6905A8002C2AD00AF073FB254697
:10D0600028460AF05DFB846A0590A4070146304615
:10D07000ECD405A80AF066FB002403980AF050FBE4
:10D08000836A049023F4804121F020029B0448BF6E
:10D0900042F00402826204A80AF054FB514803885B
:10D0A000591E0180204608B0BDE8F0870446F9E724
:10D0B000DFF838910AF046FBD9F800309D4203D0E2
:10D0C000D9F804209542D7D1039DDFF834A106F0AA
:10D0D0007FFFDAF800000DB9434D2D6885642C46BA
:10D0E00000E00C4620460AF011FB81690029F8D1C6
:10D0F000D9F800309C4272D03C4A506884426AD0D1
:10D1000005F098FB28460AF001FBDAF80040B0F978
:10D110000010B0F90230E164236506F04FFF7A0792
:10D1200011D5B8F1000F0CD007F0010282F0010018
:10D1300000902F49304603AA002300F067FB00242B
:10D140009BE70120F4E7039C20460AF0E9FA826A93
:10D15000059040F60101114001290ED005A80AF002
:10D16000F1FA20460AF0D2FA806A224B224910F4E2
:10D17000803F08BF0B4620469847204A106808B9F0
:10D1800001247AE72046FEF7DBFA20460AF0BEFAD1
:10D190008569046A002DF3D084B120460AF0B6FAFE
:10D1A000836A03F00301032911D02046FEF7C8FA71
:10D1B00020460AF0ABFA046A002CEED128460AF0A9
:10D1C000A5FA8569046A002DE6D1012455E72046B9
:10D1D000FEF75AFAE9E7012007F0A2F890E70846BF
:10D1E000FAE700BFD47F0220D87F0220C07F022050
:10D1F00009BE000825D7000829CF000800800220BA
:10D200006401002008B50AF081FA826A45F6D0432D
:10D21000C2F2000342F4004181620120186008BD9F
:10D220002DE9F04F604EDFF89091DFF890815F4D6F
:10D23000DFF88CB1A3B006F0CBFE3068002300937A
:10D240009A46002848D1D9F8001001B18847D8F88B
:10D25000002012B19047002839D12B6893F8540070
:10D2600000BB002606F0AAFEDFF840B1DFF84481DB
:10D27000DFF850912B6893F8540018B1B8F80010FB
:10D2800000294AD106F0A4FE36B1494A10680028A8
:10D2900000F081804368984706F090FE009823B024
:10D2A000BDE8F08F07F06CF988B9404E316891F80D
:10D2B0005420002AD5D03F4B18880028D1D03C4EAE
:10D2C000316800296AD00A6890470126CAE73068A9
:10D2D000012100910028B6D006F07AFEDBF800406C
:10D2E00094B120460AF01CFA826A039012F4004FAF
:10D2F000034603A80DD05F690AF024FA20463C4695
:10D30000FFF7E2F9002CECD1C6F800A006F056FEBB
:10D3100099E75C690AF016FAE2E706F059FED9F8D7
:10D32000007004A877BB47F6D877C2F202073F68BF
:10D3300007F04AF8DBF80030586BD3F830A00190C2
:10D34000AFB95046C9F8007006F0C8FF019806F062
:10D35000B9FF04A807F042F806F030FEB8F8001054
:10D3600000298FD00120009084E7002CE9D13846B5
:10D37000FFF74EFE044638460AF0C8F94769002F09
:10D38000F3D1DEE707F020F8DBF80040626BD4F859
:10D3900030A00192EBE705F017FD7DE7012005F0D5
:10D3A00013FD01265EE700BFD05C00206401002071
:10D3B000F47F0220D47F0220C87F02203080022028
:10D3C000D87F0220EC5C002040F26413C2F200031C
:10D3D0000122186880F85420704700BF08B540F259
:10D3E0006413C2F200030022186880F8542006F08B
:10D3F000EFFD05F01FFABDE8084006F0DFBD00BFF5
:10D4000010B5036804460E3B4068E1681A2B11D83A
:10D41000DFE803F01810101010100E10101D10107F
:10D4200010101010101010101F10101010101300FA
:10D43000FEF764F80021E16010BD0021BDE8104056
:10D44000FFF78ABA2146BDE810400DF0FFB9E06051
:10D4500010BD6FF07040E06010BD00BF2DE9F043DB
:10D46000DFF8788198F8004085B0002C40F08D807E
:10D470004B4EDFF86C9133684A494B4A4B4D5C6424
:10D480002046C9F800400C6014802C8008F0E8FBAE
:10D4900000287DD04648039440F6FF724FF0FF33DA
:10D4A000022721468DE88800029013462046FFF7A8
:10D4B0001BFB404F404B386021466FF070441C60AE
:10D4C000FFF74AFA012008F0CBFBB8B14FF0FF3369
:10D4D00002258DE82800364D002440F6FF721346E1
:10D4E0002146029503942046FFF7FEFA324B7860FE
:10D4F0006FF0704221465A60FFF72EFA2F480DF068
:10D50000B1FB2F480DF0AEFB2E480DF0ABFB2E48C3
:10D510000DF0A8FB2D480DF0A5FB2D480DF0A2FB4A
:10D520003D6806F055FD31680DB9D9F800508D649D
:10D530002C4600E0044620460AF0E8F880690028FE
:10D54000F8D13A68944225D01A4B59688C4224D0BD
:10D5500005F070F928460AF0D9F83368B0F90010E0
:10D56000B0F90200D964186506F028FD3168194B3E
:10D57000012281F85420184988F8002018461960C3
:10D5800005B0BDE8F04308F019BD05B0BDE8F08373
:10D59000084F97E706F0C4FEDAE70120FAE700BF7C
:10D5A00064010020EC5C0020D47F0220B87F0220C0
:10D5B00031CA0008C07F0220E87F022010810220CB
:10D5C00000810220F08002201881022008810220C0
:10D5D000F8800220C85C002019B60008F05C00202A
:10D5E000D87F02202DE9F04F87B082460AF098F8E4
:10D5F00006ADB0F9006045F8040DB0F90480B0F94B
:10D600000690B0F90270446A28460AF09BF8C6EB0F
:10D61000080000F10108C7EB0901B8F1000F01F1A2
:10D62000010940DDB9F1000F3DDD002C40D1FDF7CF
:10D6300049FF82455CD0384B384801934FF0010BCD
:10D64000394642464B460290CDF800B0304601F0D4
:10D65000C7FC044650460AF063F805904462002C6B
:10D660003FD0826A42F48031816228460AF06AF82B
:10D67000204601F0CDFD0546584606F03BFE20460B
:10D6800000F0B0F8264B09FB08F21978920005F07B
:10D69000FBF95046FFF748FC002006F02BFE284619
:10D6A00001F0B6FD00E00024204607B0BDE8F08F91
:10D6B00020460AF035F8014606A8B1F9045040F8B2
:10D6C000081DB1F806800AF03DF8B54203D10FFA03
:10D6D00088F8B845E8D0204631463A4600F02CF8A4
:10D6E000E2E728460AF02EF85046FFF71DFCDBE77C
:10D6F00004F076F8044604F087F8A0450ADC81457A
:10D7000099DD8145A8BF8146414650464A46FCF70F
:10D7100085FE90E7A046F4E7E42D0208806A02083F
:10D720003401002008B5FFF75DFF00B908BDBDE872
:10D7300008400EF061B900BF70B5044682B00D46D6
:10D74000164628B9174B1868046E0CB902B070BDA4
:10D7500006F03EFC204609F0E3FFB6B2ADB2C6804B
:10D760008580009005F066F80099486928B96846F8
:10D7700009F0E8FF06F022FCE8E709F0D1FF009A83
:10D780000190138951898380C18013B109B105804B
:10D79000468001A809F0D6FF684609F0D3FF06F0DD
:10D7A0000DFCD3E76401002010B5044682B006F0FA
:10D7B0000FFC7CB1204609F0B3FF02A9B0F90A4082
:10D7C00041F8040D084609F0BDFF06F0F7FB2046BE
:10D7D00002B010BD024B1868046E002CF5D0E9E7CA
:10D7E0006401002010B5044682B006F0F1FB20462B
:10D7F00009F096FF044602A840F8044D09F0A2FF84
:10D8000006F0DCFB04F1180002B010BD2DE9F04F6A
:10D81000044687B0894692461D46002800F0858060
:10D82000494E05A904A806F03FFF3768B4F9001077
:10D83000B4F90220787CB4F9047021EAE17322EA99
:10D84000E2710393029103F069FF3268049EB4F918
:10D8500006408019461E507C03F06EFF059B039A1C
:10D86000BE42A8BF3E46C118B01A029E01F1FF3861
:10D87000A045D4BFC6EB0806C6EB0406334603F149
:10D880000108461C0DB9C8F10005002E3DDDB8F1B8
:10D89000000F3ADD109903980091324602992B4609
:10D8A00001F074FC064600283BD0FFF77DFF0746D9
:10D8B000304601F0ADFCC7F1000B4546002411E0F5
:10D8C0005D44C4B95046C84745F6F443C2F200036C
:10D8D000E4191968002001B18847304601F052FD73
:10D8E000A04516DDAF42EBDD294630460EF022FAA8
:10D8F0005D44002CE6D0029A03993046A218FFF747
:10D900001BFF30460EF036FADCE7002007B0BDE81A
:10D91000F08F304601F010FC002001F079FC00206F
:10D92000F4E75046C8470120F0E7074F3B68587CB2
:10D9300003F0F4FE064638680294407C03F0FCFED7
:10D94000029C804603949DE76401002042F6E45067
:10D95000C0F60200012918BF002070474BF699005D
:10D96000C0F60100162918BF0020704708290CBF17
:10D9700020200020704700BF006808B5C3681B6AFC
:10D98000984708BD70B582B080680C4609F0C8FEA3
:10D99000034602A89988DA881D895E8940F8043D0B
:10D9A0004D199319013D013B21806280A580E380E0
:10D9B00009F0C8FE02B070BD2DE9F04F40F26415C9
:10D9C000C2F200059DB02C68269FDDF8ACA008933C
:10D9D0000546206E91460C4609F0A2FE199040695A
:10D9E000002840F034821CAE1A9056F80C3DD968DD
:10D9F0000F963046099109F0A5FE2A9A1A98A418A4
:10DA00000A94002800F0A98640F26416C2F20006CB
:10DA10003368197C01F00202D6B2002E00F0B98200
:10DA2000186E09F07DFE03461CA8B3F90620D968DC
:10DA3000B3F9046040F8043DC2EB0902183301FB5E
:10DA400002330A998E1B03EB860609F07BFE2798AA
:10DA5000172844DD002F3ADD0899DDF8A4A00695CB
:10DA60008A004F440B9204971A9828B185680A9946
:10DA70006C68089B4A46A047069B1869C168002944
:10DA800040F0F580089F3546D346D8467A1E58F8B0
:10DA9000043B1B0E02F0010000F0BC80DBF800002C
:10DAA000010EFF2905D0CA43D2B2296805F02AFC2D
:10DAB0002860013F0435C346002FE6D1049D289815
:10DAC000099B09F10109A94582441E44CCD11A9948
:10DAD00011B11AA809F036FE1DB0BDE8F08F10286C
:10DAE00000F07C830828054600F03F86984BBAF189
:10DAF000000F14BFD3469B46002FE8DD2A9D2A9ACB
:10DB0000CDF810906800C5F10404C5F10201299D0B
:10DB100014909300681C04364F44E4B2C9B21593C4
:10DB20000E900B9612971694179117E0042B00F0A5
:10DB30001181012B00F0A18004982999289E0E9B49
:10DB4000421C8D19049298190B9A29950999049BE6
:10DB5000129D0E905618AB420B96B8D00B9A279B8D
:10DB6000141F022BE2D140F26410C2F200000E9D9D
:10DB7000016815F8016C0B7C149ADDF86880169D1D
:10DB800003F0030006FA02F60128F6B200F036852B
:10DB900080F06081DDF8A4C0089FBD42C8BFFDB21F
:10DBA000B20923465BF82210681EB60043F8041B36
:10DBB00000F0010110F0FF00C5EB0707F2B21ED024
:10DBC00051B1960901385BF82610920010F0FF0061
:10DBD00043F8041BD2B212D0960919465BF82660AE
:10DBE0009200D2B241F8046B960902385BF82660C5
:10DBF00092005E600B1D10F0FF00D2B2ECD1013D2F
:10DC0000EBB2591C04EB8104002F95D01CF8016F76
:10DC10000425C2E70124BC4208F1040315D030B149
:10DC200013F8011CF9B902240433BC420DD01A4682
:10DC300013F8013CBBB952F8040B0134030E02F196
:10DC4000040310D10134BC42F1D14FEA84082846C4
:10DC5000594642463F1BF2F775FF4544C344002F27
:10DC60007FF413AF2AE7002C3FF418AFEDE73046FE
:10DC700051460B9AF2F766FF20E740F26417C2F2B2
:10DC8000000740F264163D68C2F20006286E09F0F3
:10DC900047FD31680E9A0B7C12F8017C2A99199085
:10DCA00046F6DC05C0F6020503F00302ED5DDDF883
:10DCB00068C0DDF82090022AC1F1080645FA01F596
:10DCC00000F0E383032A00F08A83012A00F08783AF
:10DCD000299FA4464C4605F00100B44234BFA64635
:10DCE000B6465BF8203062460EF1FF3642F8043B40
:10DCF0003146CEEB040406F001006B08CEB140B112
:10DD000003F00106AB085BF82650013942F8045BCA
:10DD10000FD003F0010610465BF82660C3F3400500
:10DD200040F8046B5BF825609B085660021D0239C1
:10DD3000EFD10CEB8E0C002C00F0858046F6DC0257
:10DD400017F8013FC0F602020826D55CC3E700BF02
:10DD5000A42D020840F26412C2F200020E9E156861
:10DD600016F8010C2B7C1599DDF868A003F003026E
:10DD700000FA01F0012A5FFA80F900F09C8480F03B
:10DD800011812A9B002B40F0DA82089D299E012DEB
:10DD90004EDD4FEA191722465BF8271009F00F09EC
:10DDA00042F8081B5BF82900334642F8040C4FEA9E
:10DDB000650C13F8019F06EB0C07F643F1190832C6
:10DDC000BB4205F0010501F001002FD080B14FEA00
:10DDD000191609F00F095BF8261042F8081C5BF8C9
:10DDE000290042F8040C13F8019F0832BB421DD0F1
:10DDF0004FEA191609F00F095BF8261042F8081CC3
:10DE00005BF8290042F8040C13F8016F310906F0A1
:10DE10000F065BF8210042F8080B5BF8260042F879
:10DE2000040C13F8019F0832BB42E1D104EBCC048F
:10DE3000002D3FF481AE4FEA19195BF829202260CA
:10DE40007AE6DDF840B00F9809F07CFC74E609F042
:10DE500067FCC8E502287FF46FAE299F08990A9BEA
:10DE600010970C93059147460D940B469D42C4BFF5
:10DE7000DDB2059B5C1B0594002F00F06C820D9AAF
:10DE800005F1FF3A16F0C00F02F104080AF0010A8A
:10DE90000AD0B009B9685BF820400B68049A48F8CA
:10DEA000044C38460C999847B2000C9E05F1FF3996
:10DEB000013619F0FF09D4B208F1040853D0BAF1C1
:10DEC000000F17D014F0C00F0AD0A009B9685BF892
:10DED00020200B6848F8042C38463146049A9847AD
:10DEE00009F1FF3CA40001361CF0FF09E4B208F17F
:10DEF000040838D013955D46CB46DDF810903146C6
:10DF0000A30914F0C00F01F1010608F1040A384614
:10DF10004A4608D055F82330D7F808E048F8043CC2
:10DF2000DEF800309847A000C4B20BF1FF3B14F0BC
:10DF3000C00F5FFA8BF80AD0A109BA6855F8210022
:10DF400013684AF8040C314638464A46984708F1A7
:10DF5000FF3CA400711C1CF0FF0BE4B20AF10408A2
:10DF6000CED1AB46139D013DE8B20C9B0D9A411CEE
:10DF700002EB81055E1C05990D9530180C90002967
:10DF80003FF4DAAD109C059B14F8016F0425109442
:10DF90006CE7089B00970A994A460DF095FE8E485B
:10DFA00003683DE5022A7FF4C7AD2A9F002F00F0E9
:10DFB000348510F0F00F0ED04FEA19185BF8285096
:10DFC0002560BAF1000F06D0DAF808400A992368F4
:10DFD000049A50469847299A0A9808990B9C92F8F7
:10DFE000019000F101084F1E012F40F3DE80BAF1CD
:10DFF000000F00F01885023F7D086B0003EB08005E
:10E00000821CC8EB000119F0F00F10970C950D93CE
:10E0100004F1080C0592C1F3400710D04FEA19151E
:10E02000DAF808305BF82500049A1D684CF8080CF3
:10E030004146CDF80CC05046A847DDF80CC019F099
:10E040000F090FD0DAF808205BF8291013684CF894
:10E05000041C5046CDF80CC008F10101049A984701
:10E06000DDF80CC0059816F8019F08F102058542FD
:10E070000CF1080C00F08C806FB319F0F00F10D089
:10E080004FEA1917DAF808105BF827200B684CF8EC
:10E09000082C5046CDF80CC02946049A9847DDF864
:10E0A0000CC019F00F090ED05BF82900DAF80870DF
:10E0B000049A4CF8040C3B68CDF80CC05046691C1F
:10E0C0009847DDF80CC0059916F8019F02358D427E
:10E0D0000CF1080C5CD0049F1194CDF84C803446B0
:10E0E000E046CC461CF0F00F4FEA1C1305F1020984
:10E0F00008F10806294650463A460CD05BF8233012
:10E10000DAF808E048F8083CDEF80030CDF80CC03A
:10E110009847DDF80CC01CF00F0C05F101015046CA
:10E120003A4607D05BF82C50DAF8083048F8045C1F
:10E130001D68A84714F8018F18F0F00F0CD04FEAB3
:10E140001812DAF808005BF82210036846F8081C79
:10E15000504649463A46984718F00F0309F1020520
:10E1600006F10808504609F101013A4607D05BF86C
:10E17000233046F8043CDAF8086033689847059A7B
:10E1800014F801CF9542ADD1119CDDF84C80E146E9
:10E190000C9F0D9D109E0C9B781C08F1020104EB56
:10E1A000C00401EB0508A6EB4307002F3FF4C4AC05
:10E1B0005FEA19193FF4C0AC5BF829202260BAF17C
:10E1C000000F3FF4B9ACDAF80810049A0E68504614
:10E1D0004146B047B0E400BF64010020002F7FF744
:10E1E00076AC299C0796A11C1A9C04914F44069773
:10E1F000002C70D0A768089B7E680A994A46204682
:10E20000B0472A690498516830F8020C8847A3681F
:10E21000079EDDF820B046F8040B4A4620461B68EE
:10E220000A990BF1FF3798470A9A0498BA4607F003
:10E23000010B00F10208571CBAF1000F3AD0BBF1F4
:10E24000000F12D0296938F8020C4B689847A26871
:10E2500046F8040B3946136820464A46984701376A
:10E26000BAF1010A08F1020824D0296938F8020C31
:10E270004A689047B346A3684BF8040B39461B68BD
:10E280004A4620469847296938F8020B4A68904761
:10E29000A36870607E1C31461F6820464A460AF11A
:10E2A000FF3AB847771CBAF1010A0BF1040608F1EE
:10E2B0000208DAD10798049B289E099942189819F8
:10E2C000069E079209F10109B14504903FF4FFABA6
:10E2D0001A9C002C8ED12B69049E5A6836F8020CC9
:10E2E0009047089C611E079C44F8040B04988A46DA
:10E2F00001F00103871C0029DCD053B12E6937F8E7
:10E30000020C726890470237BAF1010A44F8040B14
:10E31000D0D0296937F8020C4B68984726462A69FD
:10E3200046F8040B516837F8020B88470AF1FF33AF
:10E3300060600237341DB3F1010AEAD1BAE74FEA4F
:10E34000191C089D5BF82C002060299C013D94F865
:10E3500001900B9C1BE50D9A691E101D16F0C00F55
:10E3600001F0010104D0B3095BF8234040F8044CEC
:10E370006A1EB600041D12F0FF02F6B23FF4F3ADC0
:10E3800079B116F0C00F04D0B0095BF8201044F842
:10E39000041C531EB600043413F0FF02F6B23FF41F
:10E3A000E2ADB000C3B2B009013A16F0C00F1CBF15
:10E3B0005BF8200044F8040C13F0C00FD2B204F153
:10E3C000040104D09C095BF8246041F8046C9800B7
:10E3D000531E0C1D13F0FF02C6B2E2D1C3E507685D
:10E3E000396988688047299F86464846B04238BFC9
:10E3F0000646731E221D03F0010CEB07C6EB00005E
:10E4000005D552F8041C81EA0E0342F8043C6B085F
:10E410000432711E2BD0BCF1000F0BD0DD0705D5E7
:10E4200052F8045C85EA0E0542F8045C5B0804328D
:10E4300001391CD013F0010F4FEA530C01F1FF31E9
:10E4400002F1040505D052F8043C83EA0E0342F8B9
:10E45000043C1CF0010F05D055F8042C82EA0E0391
:10E4600045F8043C2A1D01394FEA5C03E2D104EB74
:10E47000860400283FF4E7AC46F6DC0317F8015F9A
:10E48000C0F6020308265D5DB0E7DBF8047029984A
:10E490000597B14538BF4E46E2460C900A9FCDF82D
:10E4A00040B0C6EB0909BAF1000F57D0002D00F0BB
:10E4B0009680F10704F104080AD4E90700F193807B
:10E4C0000137013E6D08444608F1040800F08780DA
:10E4D000D346CDF8349012E00137013E4446B946A8
:10E4E00016B36D0878D015F0010F544606F1FF36CB
:10E4F0000AF1040862D16D0809F101076CD015F02A
:10E50000010F08F1040AE7D0DBF80840049A2368F9
:10E5100039465846984705990137013E48F8041C8A
:10E520004446B946002EDCD1DDF83490DA46B9F124
:10E53000000F3FF486AC0C9E16F8011F46F6DC0C6B
:10E540000C96C0F6020C0826B14538BF4E461CF8A2
:10E550000150C6EB0909BAF1000FA7D1002D00F058
:10E56000F980231DF2070BD4EA0748BF05981C4623
:10E5700048BF43F8040C013E04336D0800F0EA8004
:10E5800005990FE06D0800F0E58015F0010F18BF48
:10E5900042F8041C6D08144606F1FF3602F104032C
:10E5A00000F0D88015F0010F18BF43F8041C013E9D
:10E5B00003F104021C46002EE4D1B8E7DBF80800A2
:10E5C000049A394607685846B847059B6D084AF8CB
:10E5D000043C09F1010792D1DDF83490DA4604EBEE
:10E5E0008604BF19A3E7DAF80840049A2368504666
:10E5F00039469847059848F8040C61E7299F089820
:10E600008542C8BFC5B205F1FF3C221D16F0C00F00
:10E61000C5EB00000CF0010C05D052F8043C83F06F
:10E62000FF0142F8041C691EB600043211F0FF011C
:10E63000F3B234D0BCF1000F0FD013F0C00F05D0EF
:10E6400052F8046C86F0FF0642F8046C01399B0016
:10E65000043211F0FF01DBB221D04E1E4FEA830CD1
:10E6600013F0C00FF1B25FFA8CFC02F1040605D082
:10E6700052F8043C83F0FF0342F8043C1CF0C00F46
:10E6800005D056F8042C82F0FF0346F8043C4FEA0C
:10E690008C020139D3B2321D11F0FF01DDD1013DF1
:10E6A000EEB2731C04EB830400283FF445AA17F86C
:10E6B000016F0425A4E7179A299D08988242C8BFD4
:10E6C000C2B2571E231D19F0C00FC2EB000007F0A5
:10E6D000010705D053F8041C81F0FF0643F8046CD1
:10E6E000561E4FEA0911043316F0FF06C9B225D0B1
:10E6F0007FB111F0C00F05D053F8047C87F0FF07FD
:10E7000043F8047C013E0901043316F0FF06C9B248
:10E7100014D09046721ED6B21F1D013E11F0C00FDC
:10E720004FF0000105D053F8042C82F0FF0C43F8A1
:10E7300004CC3B1D16F0FF06ECD14246511ECBB275
:10E740005E1C04EB860400283FF4F6A915F8019F2F
:10E750000222B3E704EB8604E9E640F2641EC2F24B
:10E76000000EDEF80030FFF75BB9002F40F3F381B5
:10E77000299C0898DDF868800A9A4F4404EB000E43
:10E7800006F1040B0697A61A45467446574640F212
:10E790006411C2F20001ABF104000B681A7C002F77
:10E7A00000F09C8012F0030339D1299B1A1B13F847
:10E7B000011B57F82110D2439C42016002F0010076
:10E7C0005A4619D040B113F8011B5A4657F8210098
:10E7D0009C4242F8040B0FD01846114610F801CBAA
:10E7E00057F82CC041F804CB5B7857F823305360BE
:10E7F000431C0A1D9C42EFD1299A2899099B501865
:10E80000069A299009F1010991450C449B440E4454
:10E81000BDD14546002D7FF45CA9FFF75DB9022B01
:10E82000EAD1002D64D00A990898735C421E02F068
:10E830000101049153B157F82300AB680A994BF8D2
:10E84000040C1B6828464A46984708980A9A531CA5
:10E85000B0F1010A0BF104083DD00499A1B1F05CBC
:10E8600060B157F82010AA6848F8041CD2F800C01C
:10E870000393194628464A46E047039B0133BAF101
:10E88000010A08F1040826D004945C1C1946F35CC4
:10E8900028464A4643B157F82330D5F808E048F8EF
:10E8A000043CDEF800309847305D0AF1FF3A08F189
:10E8B000040848B157F82010AA6848F8041C1368E7
:10E8C000284621464A469847631CBAF1010A08F1D6
:10E8D0000408DAD1049C1A9DA8468DE712F00301C2
:10E8E00034D12999089AF2F72DF91A9DA84683E7A1
:10E8F000299BD84313F8012B011901F001001AB12B
:10E9000057F822204BF8042CA3420BF10402E3D069
:10E9100048B113F8011B19B157F8210042F8040C53
:10E920000432A342D8D013F8010B111D18B157F8C7
:10E93000200042F8040C13F8012B1AB157F82200FA
:10E9400041F8040C0A1DA342EDD1C5E702297FF46A
:10E9500053AF002D00F0D7800A9A0898B35C00F1FD
:10E96000FF3A0AF00101049143B1AA680A994BF8F1
:10E97000043C284613684A4698470A9A0898B0F11A
:10E98000010C02F101080BF1040AA4D00499A9B109
:10E9900016F808305BB1AA684AF8043C28461368A8
:10E9A000CDF80CC041464A469847DDF80CC0BCF192
:10E9B000010C08F101080AF1040A8CD043460494C2
:10E9C000B04618F803605C1C194628464A4646B112
:10E9D000AB684AF8046C1E68CDF80CC0B047DDF88F
:10E9E0000CC018F804000CF1FF3C0AF1040A58B1FD
:10E9F000A9684AF8040C0B68CDF80CC028462146DB
:10EA00004A469847DDF80CC0631CBCF1010C0AF1C2
:10EA1000040AD6D1049C46465DE7089F299EDDF88E
:10EA20002880FFF7E1BAA7F1020C721C4FEA5C07DD
:10EA3000F043D519421919F0F00F04F1080302F060
:10EA4000010059D119F00F0918BF5BF82920314690
:10EA500018BF43F8042C11F8019F0833A94240D095
:10EA6000A0B119F0F00F05D04FEA19165BF8262077
:10EA700043F8082C19F00F001CBF5BF8202043F866
:10EA8000042C11F8019F0833A9422AD008464FEA06
:10EA9000191119F0F00F1CBF5BF8211043F8081C86
:10EAA00019F00F091CBF5BF8291043F8041C10F87B
:10EAB000016F16F0F00F03F1080204D033095BF880
:10EAC000231042F8081C16F00F0601461CBF5BF825
:10EAD000260042F8040C11F8019FA94202F1080334
:10EAE000D4D17D1C08F1020000EB470804EBC504FB
:10EAF000ACEB4707FFF759BB4FEA19115BF8212030
:10EB000043F8082C9EE7299B181B13F8012BC143DF
:10EB100001F001000AB14BF8042C9C420BF10402F5
:10EB20003FF4DAAE40B113F8011B09B142F8041CFE
:10EB300004329C423FF4D0AE13F8010B111D08B112
:10EB400042F8040C13F8012B0AB141F8042C0A1DF9
:10EB50009C42F1D1C0E61A9D002D7EF4BAAFFEF7BB
:10EB6000BBBF00BF2DE9F0411E4C236882B0186E78
:10EB70001746884608F0D4FD21680090086E08F01A
:10EB8000CFFD02ACB0F9065044F8040DC268B0F9EC
:10EB9000046000F11803791B204602FB013508F0E0
:10EBA000D1FD009802681369C6EB0806996888478A
:10EBB00055F82620009B504045F82600586950B172
:10EBC00008F0AEFD01908268414613683A469847C6
:10EBD000204608F0B7FD684608F0B4FD02B0BDE875
:10EBE000F08100BF6401002070B540F26413C2F2EE
:10EBF000000382B01868006E0C46164608F090FDBF
:10EC000002ABB0F90610B0F90420C56843F8040D52
:10EC1000761A183005FB0605A41A184608F092FD6E
:10EC200055F8240002B070BD2DE9F0431A4C20685D
:10EC300083B0006E0E4615461F4608F071FD23682E
:10EC40000090186E08F06CFD02ACB0F90680C16847
:10EC5000B0F9049044F8040DC8EB0502183001FB2C
:10EC60000208C9EB0609204608F06CFD48F8297037
:10EC70000098406950B108F053FD01908268314618
:10EC800013682A469847204608F05CFD684608F05D
:10EC900059FD03B0BDE8F083640100202DE9F04781
:10ECA000694F386884B0006E0E461446994608F0E5
:10ECB00037FD01904069002859D13B680290186ED9
:10ECC00008F02EFD024604A8B2F906E0D168B2F9B8
:10ECD000045040F8042DCEEB040302F1180201FBAE
:10ECE0000321751B01EB850508F02CFD3F68019899
:10ECF0003B7CFA6BC768D2F80080D9073AD40298F7
:10ED0000002800F08780C4EB0902D30718D5836878
:10ED100022461B68314601349847A145C5F800805A
:10ED20003D4419DB02980BE00298816822460B688B
:10ED300031469847029845F8078001340AEB0705E9
:10ED400083682246314601341B689847A14505EB8C
:10ED5000070AC5F80080E7DA01A808F0F3FC029B77
:10ED600013B102A808F0EEFC04B0BDE8F08708F08B
:10ED7000D7FCA2E707683869826890478046029806
:10ED8000C4EB090101F0010720B1836831461B681B
:10ED900022469847019A2868D168013480EA08031E
:10EDA0004C452B600D44D7DC87B1029820B18268B6
:10EDB000314613682246984701992868CA68013489
:10EDC00080EA08034C452B601544C5DC029B2246B3
:10EDD000314618461BB19F683B689847029B0198D3
:10EDE0002A68C76882EA080201342A601846314658
:10EDF000EF19224613B19D682B689847019839682E
:10EE0000C268013481EA08054C453D6007EB020504
:10EE1000DCDDA1E7C4EB09042146C5F8008004F05D
:10EE20000104ED19002997D024B10139C5F80080FB
:10EE30003D4491D00239C5F8008045F8078005EBC4
:10EE40004705F7D188E700BF640100202DE9F04FA6
:10EE5000DFF83C81D8F8000087B0006EDDF8409004
:10EE60008B4615461F4608F05BFCD8F8003004902E
:10EE7000186E08F055FC0DF1180CB0F90610C268B8
:10EE8000B0F904604CF8040D6C1A183002FB04034E
:10EE9000C6EB0B01604603EB8106CDF80CC008F011
:10EEA00051FC049AD8F800405069E36BD2F80CA0EA
:10EEB0001C68CBEB070701370297002855D14D4559
:10EEC0001FDCD8F80000037CD80720D4029F002F55
:10EED00013DD31467A1E104602F0010341F8044B5F
:10EEE0005AB11BB1501E41F8044B06D00A4642F8F5
:10EEF000044B4C60111D0238F8D10135A945564428
:10EF0000DFDA04A808F01EFC07B0BDE8F08F049F0C
:10EF100039680B6998688047029F3268791E3346CA
:10EF200082EA000E0A4643F804EB01F00101002AD0
:10EF3000E3D031B11968013A81EA000143F8041BBA
:10EF4000DBD01F68194687EA000C41F804CBD3F8E0
:10EF500004E00B46023A8EEA000143F8041BF0D1AC
:10EF60000135A9455644ACDACBE708F0D9FBC5EB2F
:10EF700009014A1C009259462A46029B05900CF052
:10EF8000A3FEDDF80CC0604608F0DCFB97E700BF8D
:10EF90006401002000B583B00092FFF757FF03B073
:10EFA00000BD00BF2DE9F04182B00E4690460746F5
:10EFB00008F0B6FB056802ACEB6844F8040D5A6A29
:10EFC0000020162190470546204608F0BBFB1DB1E6
:10EFD000384631464246A84702B0BDE8F08100BF3E
:10EFE0002DE9F04F454F87B03C6882468B46164668
:10EFF0001D461198637C1299002206F049FE0446D2
:10F00000002831D003699868804702F073FC06FB42
:10F0100000F808F1070181464FEAD10808F0F4FB37
:10F02000109A12F0010C05D10028B8BF03308310EC
:10F0300003EB4300002D40DDBCF1000F47D0002161
:10F040000391002D56DD08FB05F01830BCF1000FD0
:10F050000FD008F04DFB024682B92046029206F01E
:10F0600015FE039C002C40D10021084607B0BDE8E6
:10F07000F08F08F081FD0246002AEED01046029281
:10F0800008F04EFB034606A85D81039D40F8043D51
:10F090005D61A3F804A0A3F806B01C601E81C3F84C
:10F0A0000C80C3F8109008F04DFB0299129D38684F
:10F0B0002561A160427CA261D7E718386D42B0FBA0
:10F0C000F8F0A842B8BF0546BCF1000FB7D1CDF8A3
:10F0D00000C05046594632462B46CDF808C00CF0C9
:10F0E000A7FDDDF808C00390ABE7204608F018FC48
:10F0F0000299BAE7204606F0C9FDB5E76401002091
:10F1000030B5044683B098B104F062FF204608F0A1
:10F1100007FB02AD036845F8040D1869816888474C
:10F1200002F0E8FB0446284608F00CFB04F046FF1A
:10F13000204603B030BD00BF10B5044682B008B908
:10F1400002B010BD04F044FF0F4B1868016EA142DD
:10F1500016D0204608F0E4FA426901905AB90068D6
:10F1600006F094FD01A808F0EDFA204608F0D8FB5F
:10F1700004F024FFE4E710460CF08CFD0198EEE764
:10F1800005F014F9E5E700BF640100202DE9F04F18
:10F1900085B0804689469B4692460E9F04F018FF34
:10F1A000184B19491868407C51F8204002E0246847
:10F1B000002C22D0E5682E68042EF8D1EA6A204699
:10F1C00001219047054690B12469A3689847013012
:10F1D00008BF0E4C019508BF47F001070097029445
:10F1E0004046494652465B46FFF7FAFE054604F0A4
:10F1F000E5FE284605B0BDE8F08F06F031FD044677
:10F20000C568DBE76401002028800220806A0208CC
:10F2100070B5194E82B0044604F0DAFE33681D6EF4
:10F22000002C25D00DBBFEF7D9F8204608F078FA5F
:10F2300033680190196E024679B11C66106806F0B9
:10F2400063FD01A808F07EFA01F0F2FA03F0F2FA89
:10F2500004F0B4FE284602B070BD03F1080003C8F4
:10F2600003F1640686E80300E7E705F09FF8DAE7B4
:10F2700005F09CF8ECE700BF640100202DE9F047A1
:10F28000044684B00D46164610B904B0BDE8F087B8
:10F2900004F09EFE002004F0E9FF394F3B688146F0
:10F2A0002046D3F8608008F03BFA0090006880693F
:10F2B00005F036F8009B4FF20101CFF6FF718D4249
:10F2C0001A8904BFB3F90450B3F90660ADF80850C9
:10F2D00082465889ADF80A60511E431E98194A1992
:10F2E000ADF80C20ADF80E00FEF76EF8684608F099
:10F2F00029FA02A8FDF738FD40BB504605F010F88A
:10F3000004F066FE39680B6EB8F1000F34D083BB91
:10F31000FEF764F8404608F003FA3B6801900246A5
:10F32000186EE8B1C3F86080106806F0EDFC01A823
:10F3300008F008FA01F07CFA03F07CFA04F03EFED3
:10F34000484604F093FF04F039FE9EE72046294624
:10F3500032460BF0F7FCFDF7E5FC0028F6D1CCE7D0
:10F3600003F1080494E8030003F1640484E8030053
:10F37000D8E705F01BF8CBE705F018F8DEE700BF8B
:10F38000640100204FF20101CFF6FF710A46FFF73A
:10F3900075BF00BF836858699A6901380023013A34
:10F3A0000B804B808880CA80704700BF2DE9F04FEA
:10F3B000774C83B0D4F800C084680D4617469CF89B
:10F3C00010100C9AD4F81CA05B1BC7EB02085E1C43
:10F3D000CA0708F1010900F1A3802068DCF83C109D
:10F3E0000AFB07550F2E00EB850B0A6872D9B9F19D
:10F3F000000F00F0CB804FEA8A0CCCF1000708F137
:10F40000804501970CFB05B44F46A6F11000054658
:10F410000F2D22606260A260E26022616261A261DF
:10F42000E26122626262A262E26222636263A263BA
:10F43000E263C0F3001004F1400138D998B1103DE7
:10F440000A604A608A60CA600A614A618A61CA6168
:10F450000A624A628A62CA620A634A638A63CA6348
:10F4600040310F2D23D9203D0A604A608A60CA606E
:10F470000A614A618A61CA610A624A628A62CA6230
:10F480000A634A638A63CA630A644A648A64CA6410
:10F490000A654A658A65CA650A664A668A66CA66F0
:10F4A0000A674A678A67CA6780310F2DDBD8013F38
:10F4B000CCEB0404A9D10F3B1809411C09F180438E
:10F4C000581E8B0101990CFB003008FB01039B4483
:10F4D00006F00F060EB3B9F1000F1ED04FEA8A0AEC
:10F4E00008F180480AFB08BB701E5B46014643F8E2
:10F4F000042B00F0010059B118B1013943F8042B75
:10F5000006D0184640F8042B5A60031D0239F8D182
:10F51000B9F10109CAEB0B0BE6D103B0BDE8F08FDE
:10F52000036999688847E269002EF6D0B9F1000FA7
:10F53000F3D002FB0755CAEB8A7E08FB0A574FEA55
:10F540008E0CBF002368FA58711E82EA00050A4635
:10F55000FD5001F001013B1D9AB131B125685959A7
:10F56000414059510433013A0BD025685959414063
:10F570005951043321685D5845405D500433023AC7
:10F58000F3D1B9F101096744DCD1C6E7CB469FE767
:10F590006401002010B48068C469006804FB021292
:10F5A00040F8223010BC70478368D8691B6800FBA4
:10F5B000021253F822007047F8B58368DF690D46E0
:10F5C00001690446164618688B6807FB025250F81A
:10F5D00022709847A168CA690B6802FB06557840FB
:10F5E00043F82500F8BD00BF70B5846882B0246B75
:10F5F000069E05464CB1084800960668A869F56B5A
:10F600002D680195A04702B070BD069602B0BDE816
:10F610007040FFF7CBBE00BF640100202DE9F04F22
:10F6200093B005461D981C9EDDF87C900B93013825
:10F63000AF681F283BD8DFE810F08900C5013A0009
:10F640002F013A003A003A0020003A003A003A000E
:10F650003A003A003A003A003A003A003A003A00DA
:10F660003A003A003A003A003A003A003A003A00CA
:10F670003A003A003A003A003D00FF6B002F00F0DC
:10F68000398283480368187C00F00203D8B200284E
:10F6900040F03082219C002C00F02C82A8690B9D48
:10F6A00003948DE860001E9E4B460296B84713B047
:10F6B000BDE8F08F002EFADD0B9BDDF878A009F194
:10F6C000040902EB060801EB030C9B46BBF1000F9B
:10F6D00037DDAC6859F8040CE7692668CB4303EBC7
:10F6E0000C0407FB02174B1C634546F8270004F087
:10F6F000010409F1040024D064B1AE6850F8044C50
:10F70000F769366807FB023701330430634546F872
:10F71000274016D0AC6850F8047CE669246806FBE4
:10F720000236013344F82670AC6850F8047BE66971
:10F73000246806FB023601330430634544F8267022
:10F74000E8D101324245D144C0D1B0E7D7F838C042
:10F75000BCF1000F05D04E480368187CC30740F188
:10F760003F85002EA3DD209C0B9BDFF828B1DDF840
:10F7700084C00919924658189219C4F108060D91CF
:10F780000C920E960F90A84640F26415C2F2000546
:10F79000DCF800002C68DCF80430217C01F0030266
:10F7A000022A00F09384032A00F01484012A00F056
:10F7B000118499F80050FE691BF8052039680B9DEB
:10F7C000209F0D9C42FA07F76A1E02F0010517F010
:10F7D000010F11950E9D0CBF02461A4606FB0A4604
:10F7E00001EB860410926A1E09944C4640F0BD84D9
:10F7F00099F801701BF8075009F101040822109FC5
:10F8000041F8267009990B9F0E1D06967E1E00F08A
:10F810007C821199002900F0B38415F0010F0CBF10
:10F8200007461F46013A109740F0A78465781BF8F9
:10F83000055008220134109F09994F60069F391D19
:10F84000013E069117D160E26D0815F0010F41F8F5
:10F85000047B0CBF07461F46013A06F1FF3640F015
:10F86000968365781BF8055008220134013E41F863
:10F87000047B00F04A8215F0010F0CBF07461F46BB
:10F88000013AE1D1627801341BF802500822DCE72A
:10F8900064010020DC680208002E7FF708AF944C5A
:10F8A00020982768219C0E97091896190D960F919C
:10F8B000F020002C7ED0AB680E9FD96997F810C05D
:10F8C0000F9F1E6899F8003001FB027806EB880A4A
:10F8D0001CF0030CCDF830A040F09E82209FC7F1B1
:10F8E00001018F00C7F1040A40FA0AF101EA030A94
:10F8F0002AFA07F70B9954F8277046F82870209ECB
:10F900000C9F01F1FF3A711C3E1D0229C8460AF006
:10F91000010A00F040840B9FB7F1010C4AD0BAF104
:10F92000000F18D0C1F1010B4FEA8B0ACAF104078E
:10F9300040FA07FB0BEA030B2BFA0AFA013154F8E1
:10F940002A70DDF830A004360229CAF8047029D0E4
:10F95000BCF1010C2ED0C1F10107BF00C7F1040AB0
:10F9600040FA0AFA0AEA030A2AFA07F7013154F8B8
:10F970002770022946F8047B0CF1FF3C00F0098354
:10F98000C1F10107BF00C7F1040A40FA0AFA0AEA06
:10F99000030A2AFA07F7013154F82770022946F8BA
:10F9A000047BD5D10021BCF1010C98F8013008F19D
:10F9B0000108D0D10D9F1E9E0132BA42B1447FF49E
:10F9C00078AF74E6002E7FF772AE494CB318209ED4
:10F9D0002068219C0E9089190D930F91C020002C56
:10F9E0007ED0AB680E9FD969DDF83CA097F810C0B7
:10F9F0001E6899F8003001FB02A806EB88071CF08E
:10FA0000030C0C9740F08C81209FC7F103014F003D
:10FA1000C7F1060A40FA0AF101EA030A2AFA07F7CF
:10FA20000B9954F8277046F82870209E0C9F01F11E
:10FA3000FF3A711C3E1D0429C8460AF0010A00F075
:10FA4000B7830B9FB7F1010C4AD0BAF1000F18D061
:10FA5000C1F1030B4FEA4B0ACAF1060740FA07FB54
:10FA60000BEA030B2BFA0AFA013154F82A70DDF87D
:10FA700030A004360429CAF8047029D0BCF1010C66
:10FA80002ED0C1F103077F00C7F1060A40FA0AFA37
:10FA90000AEA030A2AFA07F7013154F82770042901
:10FAA00046F8047B0CF1FF3C00F08E82C1F10307A5
:10FAB0007F00C7F1060A40FA0AFA0AEA030A2AFA9C
:10FAC00007F7013154F82770042946F8047BD5D193
:10FAD0000021BCF1010C98F8013008F10108D0D1E7
:10FAE0000D9F1E9E0132BA42B1447FF478AFDEE52D
:10FAF00064010020002E7FF7DAAD0B9FDFF8FC8653
:10FB0000083FFB08D8F800404FEAC30A581CA7EB8F
:10FB1000C3070AF1080C0D9406EB020B4301C60063
:10FB2000219C0E970F960C93CDF840C08A46002C6E
:10FB300000F0E480A9680D9FC8693E7C0B6816F050
:10FB4000030600FB02A103EB810740F0DF810B9B62
:10FB5000072B40F3428310994B4609EB01063946C7
:10FB6000187854F820000860587854F8200048604D
:10FB7000987854F820008860D87854F82000C8603D
:10FB8000187954F820000861587954F82000486129
:10FB9000987954F820008861D87954F82000083307
:10FBA000C8612031B342DBD10F9B0C9E0E9909EB4B
:10FBB000030CBF19032977DD9CF8000054F82030AE
:10FBC0003B609CF8016054F8260078609CF8023095
:10FBD00054F82360A1F10408BE609CF80300CDF83E
:10FBE0004480119E54F82030032EFB60C8F3800837
:10FBF0000CF1040007F110034DDDB8F1000F00F027
:10FC0000B98290F8008054F828601E6090F8018056
:10FC100054F828605E6090F8028054F828609E6076
:10FC200090F8038054F82860DE60119E043E043092
:10FC30001033032E1196C8BF09922CDD027854F8B8
:10FC400022201A6090F8018054F828205A6090F819
:10FC5000028054F828209A6090F8038054F82820F5
:10FC6000DA6090F8048054F828201A6190F8058032
:10FC700054F828205A6190F8068054F828209A6198
:10FC800090F8078054F82820083EDA6108302033C5
:10FC9000032ED3DC099A04398E08731CA1EB86016C
:10FCA0000CEB830C07EB031741B36346614413F875
:10FCB000010B6FEA0C0654F8200006EB010C8B4296
:10FCC00047F8040B0CF0010618D03EB113F8010BF5
:10FCD00054F820608B4247F8046B0FD01E4638461C
:10FCE00016F801CB54F82CC040F804CB5B7854F8DC
:10FCF00023307B60731C071D8B42EFD101321E9EA7
:10FD00005A45B1447FF413AFD1E40C9F1E9E0AF113
:10FD1000010ABA45B1443FF4CAACD8F8087033E5DB
:10FD2000BCF1020F7FF4DCAE2099C1F10306710033
:10FD3000C1F1060740FA07F80B9E0C9F08EA030C76
:10FD4000013E04373CFA01F1C84606F0010A03D02F
:10FD500054F8216047F8046C20990131042900F01F
:10FD600021820B9E0437B6F1010C3FF4B9AEBAF113
:10FD7000000F18D0C1F103067600C6F1060A40FA5A
:10FD80000AFA0AEA030A3AFA06F61CBF54F8266091
:10FD900047F8046C0131042900F010820437BCF1EB
:10FDA000010C3FF49DAE934619E0C1F103077F00BB
:10FDB000C7F1060A40FA0AFA0AEA030A3AFA07F70A
:10FDC00003D054F8277046F8047C0131042906F169
:10FDD000040700F0E480BCF1010C00F0E980C1F1FF
:10FDE00003067600C6F1060A40FA0AFA0AEA030A8E
:10FDF00001313AFA06FA1CBF54F82A2047F8042CBD
:10FE000004290CF1FF3C07F10406CED198F801302B
:10FE1000002108F10108C8E7BCF1020F7FF4CAAD68
:10FE20002099C1F10106B100C1F1040740FA07FAB7
:10FE30000B9E0C9F0AEA030C013E04373CFA01F1C9
:10FE4000C84606F0010A03D054F8216047F8046C54
:10FE500020990131022900F098810B9E0437B6F1F8
:10FE6000010C3FF4A7ADBAF1000F18D0C1F10106A3
:10FE7000B600C6F1040A40FA0AFA0AEA030A3AFA94
:10FE800006F61CBF54F8266047F8046C01310229BD
:10FE900000F09A810437BCF1010C3FF48BAD93461E
:10FEA00017E0C1F10107BF00C7F1040A40FA0AFADE
:10FEB0000AEA030A3AFA07F703D054F8277046F81B
:10FEC000047C0131022906F1040773D0BCF1010C56
:10FED00078D0C1F10106B600C6F1040A40FA0AFA68
:10FEE0000AEA030A01313AFA06FA1CBF54F82A203A
:10FEF00047F8042C02290CF1FF3C07F10406D0D18D
:10FF000098F80130002108F10108CAE7022E7FF4B9
:10FF1000F5AE0B9800287FF7F1AE4B4609EB0001D8
:10FF20006FEA090613F8010B7618043706F001068C
:10FF300018B154F8200047F8040C04378B423FF402
:10FF4000DDAE56B113F8016B1EB154F8260047F828
:10FF5000040C04378B423FF4D1AE13F8016B381D0B
:10FF60001EB154F8266047F8046C13F8017B1FB1EA
:10FF700054F8276040F8046C071D8B42EDD1013224
:10FF80001E9E5A45B1447FF4D2ADFFF790BB6D0879
:10FF90006CE498F80130002108F10108F0E4002138
:10FFA000BCF1010C98F8013008F101087FF417AF9B
:10FFB0005A4695E50021BCF1010C98F8013008F192
:10FFC000010886D15A46F5E498F80130002108F17D
:10FFD00001086BE5D8F810008368CDF828C0984771
:10FFE0000D9C209B99F800700F9ADDF828C08026A0
:10FFF000E1431E418D1837424C4605F001010BD0FC
:020000040801F1
:10000000D8F808700D9EFD693A6805FB0A6752F83A
:100010002730434042F82730209D0D9A6B1C0F9DDE
:100020000132082B04BF09F101040023AA423FF466
:100030006CAE002900F0A7808021257819410D427F
:100040000AD0D8F80870FE693D6806FB0A2755F803
:100050002710414045F8271001330132082B00F0EA
:10006000B9800F9EB2423FF450AE354616E080276D
:1000700026781F413E420AD0D8F80820D769166872
:1000800007FB0A1756F82720424046F8272001337D
:100090004A1C082B66D0AA423FF437AE802127784D
:1000A000194101330F4202F101010AD0D8F808606A
:1000B000F769366807FB0A2756F82720424046F8BA
:1000C0002720082BD3D101340023D0E7FE690D9DF2
:1000D000396899F8000006FB0A5701EB87021BF804
:1000E000004020990B9844FA01F4461E101DE707C2
:1000F000494606F0010601D540F8043C0E9D6A1EF3
:1001000036D199F801401BF8044009F10101082299
:100110000B9F04307D1E3FF4F8AD76B1E60701D5A4
:1001200040F8043C013A15D14E781BF806400822ED
:1001300001310430013D3FF4E8ADE60748BF40F827
:10014000043C013A08D06408013D0430E707E7D4D5
:10015000013AE9D06408ECE74C7808221BF8044027
:100160000131F1E70134002395E77D08FFF747BB34
:100170006408CDE70992119E60E56D08FFF75BBB4F
:100180000699FFF778BB0F9D88E799F8013009F1D0
:100190000108002161E699F8013009F10108614682
:1001A000FFF7B9BB99F8013009F101080021D8E542
:1001B00099F8013009F10108614642E498F80130EC
:1001C000002108F10108E9E598F80130002108F163
:1001D00001085FE60134002343E71946CC46E9E411
:1001E000A869209B0B9D0296219C1E9E0093019561
:1001F000039604944B46E047FFF759BA6401002088
:10020000013983680D290CD8DFE801F00E101214B3
:100210000B0B0B1607090907070700207047012081
:1002200070474FF0FF307047D868704718697047C3
:1002300058697047986970472020704742F6E4502B
:10024000C0F60200012918BF002070472DE9F00F09
:100250008468099FE0695B1A03F1010802FB001141
:100260004FEA800A4FEA810C4FEA8809256808F1B5
:10027000FF315CF805603B460846C7EB0C0501F012
:10028000010143F8046BC0B131B121685E19013836
:10029000715843F8041B10D0266803EB050B194670
:1002A0005BF8066041F8046B266801EB050B5BF810
:1002B00006605E600B1D0238EED101320898531EB5
:1002C00098424F44D444D1DCBDE8F00F704700BFE2
:1002D0000139242946D8DFE801F043413F3D453B41
:1002E00045453937353345312F4545452D2B292790
:1002F0004545234545454545451F1D1B17451300ED
:1003000003689868C06B704702689168086C704712
:10031000154870471548704703689868806B7047A8
:1003200002689168086B7047114870471148704720
:10033000114870471148704711487047114870477D
:10034000114870471148704711487047114870476D
:10035000114870471148704711487047114870475D
:100360001148704700207047AD0301085506010889
:1003700051070108E90301080104010819040108F3
:10038000310401083D04010825050108C1060108E2
:10039000190701081506010859050108A5070108F4
:1003A000D1050108950501084D02010870B582B01C
:1003B00085680023044601930E4645B102AAA06950
:1003C00042F8046D0E21F6F74BF902B070BD4420DF
:1003D00007F0CAF82946A060442202F055FBA06845
:1003E0000028F2D0EAE700BF00B583B08DE8060030
:1003F00080690D216A46F6F733F903B000BD00BFEE
:1004000000B583B002AA806942F8041D0C21F6F7FA
:1004100027F903B000BD00BF00B583B002AA806910
:1004200042F8041D0B21F6F71BF903B000BD00BF15
:10043000806906210022F6F713B900BF8069052103
:100440000022F6F70DB900BF2DE9F043044683B052
:10045000002380690093884691460193A56801F0C6
:1004600095F90646A06901F09FF90746A06901F0D9
:10047000A9F9800040EA47013143072911D8DFE894
:1004800001F0181B242D3A3F48042A69EB68A8693B
:100490006969801AC91AC9EB0002C8EB01038DE82B
:1004A0000C00A06903216A46F6F7DAF803B0BDE84C
:1004B000F0838DE80003F4E76A69EB68CDF80490F7
:1004C000D01AC8EB00010091EBE7AA692B69CDF8BF
:1004D0000080D01AC9EB00010191E2E7EA682B69BC
:1004E0006869A969801AC91AC8EB0002C9EB01033F
:1004F0008DE80C00D5E7CDF80090CDF80480D0E76A
:10050000AA692B69CDF80480D01AC9EB00010091CB
:10051000C7E76A69EB68CDF80090D01AC8EB000114
:100520000191BEE738B58468054654B10121002227
:10053000A869F6F795F8D4F1010438BF00242043E8
:1005400038BD442007F010F82146A860442202F08C
:100550009BFAAC68EAE700BF70B582B084680023FC
:10056000054601930E464CB102AAE66242F8046DBC
:10057000A8690921F6F774F802B070BD442006F0AE
:10058000F3FF2146A860442202F07EFAAC68002CFA
:10059000F2D0E9E770B582B0846800230546019384
:1005A0000E464CB102AAA66242F8046DA8690A215F
:1005B000F6F756F802B070BD442006F0D5FF21468C
:1005C000A860442202F060FAAC68002CF2D0E9E79F
:1005D000F0B583B084680023054600930F461646A5
:1005E000019354B127626662A869009708216A46A0
:1005F0000196F6F735F803B0F0BD442006F0B4FFDD
:100600002146A860442202F03FFAAC68002CF2D0E8
:10061000E8E700BF70B582B0846800230646019306
:100620000D4654B102AA2560656042F8045DB069C8
:100630000221F6F715F802B070BD442006F094FFD1
:100640002146B060442202F01FFAB468002CF2D0B8
:10065000E8E700BF2DE9F041846805460F461646DD
:100660000CB3B74217D0EB6808219A6A2846904726
:100670002269E168D4F804C0636B01FB02FE00FB51
:100680000EF0C20806FB02C83BB1A86939463246E3
:100690009847C4F80080BDE8F081404607FB02C1DE
:1006A000F0F750FAF5E7442006F05EFF2146A86017
:1006B000442202F0E9F9AC68002CD2D1BDE8F08107
:1006C000F0B583B084680023054600930F461646B4
:1006D0000193ACB1E06950B1E7602661A869009769
:1006E00007216A460196F5F7BBFF03B0F0BDA86984
:1006F00001F068F800280CBF39463146E161EBE7AC
:10070000442006F031FF2146A860442202F0BCF9E3
:10071000AC68002CE9D0DDE7F8B5846805460E46E4
:1007200017464CB1A86901F04DF86661A76108B998
:10073000E661F8BDE761F8BD442006F015FF2146EB
:10074000A860442202F0A0F9AC68002CEAD1F8BD00
:10075000F8B5846805460E461746B4B1A6F11901EE
:100760000C2909D8DFE801F00B0808080808080D73
:100770000F08070809002764F8BDE763F8BD276381
:10078000F8BDA763F8BD6763F8BD442006F0ECFE32
:100790002146A860442202F077F9AC68002CDDD134
:1007A000F8BD00BFF8B5846805460F46164624B16B
:1007B000236A3B60606A3060F8BD442006F0D4FED6
:1007C0002146A860442202F05FF9AC68002CEFD10A
:1007D000F8BD00BF70B5846882B0246B00920546F6
:1007E000164644B105480668A869F56B2D68019561
:1007F000A04702B070BDFEF7D9FDFAE76401002002
:1008000070B5846882B0246B009305460E464CB1E7
:10081000064B80691B68DB6B1B6801930B46A04786
:1008200002B070BD0B46FEF7C1FDF9E76401002080
:1008300010B540F26414C2F200042368186B02F091
:10084000CBF802F0EDF82068406B02F0C5F8BDE887
:10085000104002F0F5B800BF30B540F26414C2F2A7
:10086000000448F228032268C2F20203517C53F8C4
:100870002130DA6883B0054669461846136B9847FD
:100880002068294608306A4602F0A8FA03B030BD55
:1008900010B582B00C4605F0E3F9019060B1C36871
:1008A00009215A6A01A89047034628B101982146B8
:1008B0009847002002B010BD0120FBE730B583B09F
:1008C0000D46144605F0CCF9019068B1C3680A21C1
:1008D0005A6A01A89047034630B10198294622463A
:1008E0009847002003B030BD0120FBE730B583B04E
:1008F0000D46144605F0B4F9019068B1C3680B21A8
:100900005A6A01A89047034630B101982946224609
:100910009847002003B030BD0120FBE730B583B01D
:100920000D46144605F09CF9019068B1C368032197
:100930005A6A01A89047034630B1019829462246D9
:100940009847002003B030BD0120FBE730B583B0ED
:100950000D46144605F084F9019068B1C368102172
:100960005A6A01A89047034630B1019829462246A9
:100970009847002003B030BD0120FBE730B583B0BD
:100980000D46144605F06CF9019068B1C368042166
:100990005A6A01A89047034630B101982946224679
:1009A0009847002003B030BD0120FBE730B583B08D
:1009B0000D46144605F054F9019068B1C36816213C
:1009C0005A6A01A89047034630B101982946224649
:1009D0009847002003B030BD0120FBE781880388E1
:1009E000428810B4C48851181C19A21ACB1A8280EC
:1009F000C38010BC704700BF2DE9F04F93B00024B6
:100A000006460CA80F4608920A930C940D94DDF844
:100A100078B0B44CFAF712FA00F0E2FE00F0F4FEFF
:100A2000BDF93630B4F90620BDF93050B4F90010E4
:100A3000B4F902E001389842B8BF03B2BDF9320000
:100A4000C6EB030C6244C31AD3187D1900226D183B
:100A50000CA8C9180B910C920D92CEEB0505FAF774
:100A6000EDF900F0BDFE00F1FF3800F0CDFEBDF95C
:100A700034301C9AB4F800C06188B4F806A0BDF800
:100A8000324001389845BDF93630B8BFADF83480F2
:100A90009842B8BF03B2012ABDF8300000F00582C9
:100AA0000A9F002FCBF1080940F3D98040F2641669
:100AB000C2F200060027326803971D9CB2F9083085
:100AC0002819461EB342059000F3BB80B2F90C1002
:100AD000A942C0F2B680089F002F40F3B280219C4B
:100AE000002C00F013812098089B8246591E1AF8AA
:100AF000017B47FA09F007FA0BF410F0FF0FCDF86D
:100B000010A001F0010CCA46E4B206D1137C03F038
:100B10000201CFB2002F40F0F280219F0B9BD26BDD
:100B2000C1B257F821001C9917681060C1EB030887
:100B3000284632460B9BCDF804C008F1010101F0B4
:100B4000E9F840F26412C2F20002DDF804C0126853
:100B5000D06B43460760089901278F4271D0BCF1E2
:100B6000000F39D0BAF1000F40F0C680DDF810A0B8
:100B70001AF8014BCDF810A0CA4644FA09F111F059
:100B8000FF0F04FA0BF4E4B206D1107C00F002006F
:100B9000C0B2002840F0B780DDF88480D26BC8B2C4
:100BA00058F82010106811601C9A0990C2EB0308D5
:100BB000284608F10101324601F0ACF840F2641316
:100BC000C2F2000309981A68D16B43460860DDF849
:100BD00020C00137674534D05146AA460D46002D46
:100BE00000F08280CBEB050504FA0BF044FA09F41F
:100BF00014F0FF0F5FFA80F851D1117C01F0020070
:100C0000C1B200294BD01C9C01371B1B002D66D1A3
:100C1000049C14F8018B4D46049408FA0BF048FA32
:100C200009F818F0FF0FC4B21CD1117C01F00200CA
:100C3000C1B2B9B11C981B1ADDF820C00137674555
:100C4000CDD1039E209D1F9FDDF828C0741C6445F4
:100C500005EB070603942096059D7FF42EAF13B095
:100C6000BDE8F08F5FFA88F8DDF884E0D26B5EF8BB
:100C70002810106811601C9A0990C2EB03085046B6
:100C800008F10101324601F045F840F26413C2F266
:100C9000000309981A68D16B43460860CCE7E0B2BC
:100CA000DDF884E0D26B5EF820101C9814681160A7
:100CB000C0EB030C0CF1010132465046CDF804C0E4
:100CC00001F028F840F26413C2F20003DDF804C01A
:100CD0001A68D16B63460C600137002D98D0CBEBBE
:100CE00005059AE704800220DDF8108018F8014B12
:100CF0004D46CDF8108077E7CBEB0A0A3DE70B981D
:100D00001C9BC31A27E71C995B1A60E7209C2346AB
:100D100007F1FF3A13F8011B41FA09F001FA0BF74A
:100D200010F0FF0F04930AF0010ACC46FCB200F069
:100D3000D181DDF82CE01C9FD26BC7EB0E08C1B24D
:100D400017681160284608F1010132467346CDF854
:100D500004C000F0DFFF40F26410C2F20000DDF8D2
:100D600004C00268D16B43460F60089F4FF0010832
:100D7000B8453FF466AFBAF1000F1DD0BCF1000FCB
:100D800000F0B381CBEB0C0C44FA09F111F0FF0F2A
:100D900004FA0BF4E4B240F0B081107C00F00207DA
:100DA000F8B2002800F0A9811C995B1A089F08F18D
:100DB0000108B8453FF445AFAA466546002D37D136
:100DC000DDF810C01CF8014B4D46CDF810C004FAF8
:100DD0000BF044FA09F414F0FF0FC7B22BD1117CC9
:100DE00001F00200C1B231B31C9C08F101081B1BC9
:100DF000002D3DD1DDF810C01CF8017B4D46CDF82B
:100E000010C007FA0BF147FA09F717F0FF0FCCB241
:100E100031D1107C00F00201C8B260B31C9FDB1B13
:100E2000089808F1010880453FF40BAF002DC7D0AA
:100E3000CBEB0505CBE71C98D26BC0EB030EE1B200
:100E400050461468116032460EF10101CDF804E0FD
:100E500000F060FF40F26413C2F20003DDF804C04A
:100E60001A68D06B6346046008F10108002DC1D0F8
:100E7000CBEB0505C5E71C99D26BC1EB030EF8B2AD
:100E80000EF101011768106032465046CDF804E0BB
:100E900000F040FF40F26413C2F20003DDF804C02A
:100EA0001A68D16B63460F60BAE71D9A012A7FF476
:100EB000F7AD0A9ADFF82898D719013FD9F80080D2
:100EC00007FA80F00FFA8CFC00EB0C0709B2B8F9B6
:100ED0000C007F1AB84202DA391A521A0A92B8F98B
:100EE0000810A94209DD20981F9F4D1B07FB050232
:100EF0000A982092451B0A950D46089FB9194A1E6B
:100F0000981A24B200FA8AF1E31ACA18B8F90A004A
:100F10009444604503DDCCEB00043F1B0897B8F90F
:100F20000E10DDF82CC06145C0F201814FF0000CBD
:100F3000089CCDF814C0002C7FF791AE0A9E002EBD
:100F40007FF78DAEDDF814A00B9ACDF80CB0CAEB8C
:100F50000207AA463D1B681C5644069709960A904C
:100F6000209D0DE0042C00F05981012C00F0F88048
:100F7000099E1F9C0AF1010AB24525443FF46FAE59
:100F8000039C022CEED142F69457C0F6020797E874
:100F90000F00059EC6F1030467002E78D9F80040C3
:100FA000C7F1060B0DF1480E4FF0C0080EE90F0017
:100FB00048FA0BF3227C089C334023FA07F346F6E9
:100FC000CC070EEB830102F00300631EC0F602079C
:100FD00003F0010311F8102C57F820700699059CB6
:100FE000029350460195B8470699089A029BDDF88E
:100FF00004C00134501A042C049001F1FF3B00F0AE
:101000001F8200EB0B02002AB2D003B3C4F103012C
:101010004B00C3F1060048FA00F2324022FA03F313
:1010200012A901EB83025046594612F8102CCDF854
:1010300004C00134B847042C0BF1FF3BDDF804C0B9
:1010400000F02682049800EB0B03002B90D007954C
:101050005D46A34664461BE0CBF103025300C3F197
:10106000060E48FA0EF202EA060C2CFA03F312AA54
:1010700002EB83030BF1010B13F8102CB847BBF103
:10108000040F00F05F8104984119002900F0588195
:10109000CBF103014A00C2F1060048FA00F33340E5
:1010A00023FA02F112AA02EB8103504629460BF102
:1010B000010B13F8102CB84705F1FF3CBBF1040FEE
:1010C00050466146A5F10205C6D166784FF0000B87
:1010D0000134C1E7137C03F00201CFB2002F3FF4CB
:1010E00028AE0B981C9BC31A3FE6DDF810C01CF815
:1010F000014BCDF810C0CC4646E61C9FD26BDF1BDF
:10110000C8B2D2F800A01060791C32462846CDF84B
:1011100004C000F0FFFD40F26413C2F20003DDF8EA
:1011200004C01A68D16B3B46C1F800A03EE6089A9D
:10113000C1EB0C03D41ABBF1010F059308947FF4A3
:10114000FAAE209C1F4623F0070004EBE301C0EB3E
:101150000C0607F0070720910B960597089CEAE616
:10116000D9F8003021991A7C0F68D1F804B002F048
:101170000306012E00F0928180F0E980DDF81880EE
:101180000A98059CC0EB0801CA074646A84600F12C
:101190005D81049520E00A9B802040FA04FC013424
:1011A0009E4200F06682D9F8000098F80060437C07
:1011B00048F2280EC2F2020E16EA0C0F5EF8230067
:1011C000C3689E690CBF3B465B46B047082C00F0E5
:1011D0001382D9F800306E1E48F228005D7C98F822
:1011E0000020C2F20200802350F825002341D0F8ED
:1011F0000CE01A42514632460CBF3B465B4604F1B6
:101200000104DEF818C0E04706F1FF35082C51460E
:101210002A46C0D1002408F10108BCE7D9F80070C3
:10122000059B387C2E780195C3F101029400C4F12E
:10123000040100F003074FF0F008089848FA01F2A3
:1012400046F6CC0B431EC0F6020B324003F00103FE
:1012500022FA04F25BF827700699059C0293504627
:10126000D2B2B8470699089A029BDDF804C001344F
:10127000501A022C049001F1FF3B00F0DB8000EBE0
:101280000B02002A3FF474AEEBB1C4F101018B00F4
:10129000C3F1040048FA00F2324022FA03F2594640
:1012A000CDF804C05046D2B20134B847022C0BF13D
:1012B000FF3BDDF804C000F09981049901EB0B03BA
:1012C000002B3FF455AE07955D46A346644614E0F7
:1012D000CBF101039A00C2F1040E48FA0EF303EABF
:1012E000060C2CFA02F2D2B20BF1010BB847BBF19B
:1012F000020F20D00498411911B3CBF101008200F4
:10130000C2F1040148FA01F3334023FA02F22946FC
:1013100050460BF1010BD2B2B84705F1FF3CBBF1CF
:10132000020F50466146A5F10205D1D166784FF013
:10133000000B0134CCE766784FF0000B0134D9E79D
:10134000079D15E666784FF0000B01349BE6022EF0
:101350007FF40EAE0899069F059A2878DDF820C024
:101360007C1A01F1FF3880211141084204942E4675
:1013700008F0010804EB0C0240F0A4810598441C1D
:10138000082C00F09C8108994F1E3FF4F1ADB8F194
:10139000000F1FD080233078DDF810C023411842A1
:1013A0000CEB07020ED0D9F8001048F2280E487C4A
:1013B000C2F2020E51465EF82000C368D3F818C08E
:1013C0005B46E0470134082C01D101360024013F7F
:1013D0003FF4CEAD3A462F46049D12E0082C05EBB3
:1013E000080200F04381802330782341184240F006
:1013F0002D810134082C00F02681B8F1010200F0A3
:101400003A818021307821410134084202F1FF38CD
:101410002A44E3D0D9F8003048F2280E587CC2F2B2
:10142000020E5B465EF82000C168D1F818C0514634
:10143000E047D3E76E78049805F1010C00241EE71D
:101440006E78049805F1010C0024DAE548F2280EC4
:101450005B7C2E78C2F2020E80225EF823002241CD
:10146000C16816420CBF3B465B468E69069A5146E0
:10147000B0470134DDF818C0D9F800300495082CC5
:1014800008BF05F101080CF1FF3608BF0024A3E6F0
:101490009CF8016000240CF1010CD3E548F228010E
:1014A0005F7CC2F20201AB4651F8272010698468C4
:1014B000A04704900598089E2978069B8022024147
:1014C000771EC6EB030C114207F00107664440F09B
:1014D000D480441C089E082C04BF05F1010B002495
:1014E000B6F101083FF444AD002F34D080239BF8BF
:1014F0000010234119420CEB080722D0D9F8002034
:1015000048F2280E507CC2F2020E51465EF82000CE
:10151000C6683A467369CDF804C09847D9F80010F8
:10152000049B4E7C48F22802C2F20202434052F869
:101530002610CA680846966951463A46B047DDF813
:1015400004C00134082C04BF0BF1010B0024B8F1D6
:1015500001083FF40DAD674614E0082C04BF0BF101
:10156000010B00249BF8000080212141084247D153
:101570000134082C04BF0BF1010B0024B6F1010863
:101580003FF4F6AC80219BF80000214108F1FF36C2
:101590000134084207EB080307EB0608DDD0D9F851
:1015A000002048F2280E507CC2F2020E51465EF82E
:1015B0002000D0F80CC01A46DCF814C00293E047B3
:1015C000D9F80010DDF810C04B7C48F22802C2F2B6
:1015D000020280EA0C0E52F82310029ACB680846E9
:1015E000D3F818C051467346E047B6E79CF801604F
:1015F00000240CF1010C60E608F101080024E8E584
:10160000D9F8003048F2280E5A7CC2F2020E514638
:101610005EF82200C36842465B699847D9F800101B
:10162000DDF810E04A7C48F2280CC2F2020C80EA95
:101630000E035CF82220D1681046D1F818C042464B
:101640005146E04794E701360024D6E6D9F8001069
:1016500048F22803487CC2F2020353F82000C16814
:101660005B46D1F818C05146E047C2E60136002477
:10167000B9E6049D7CE43D467AE4D9F8000048F2DE
:101680002804417CC2F20204324654F82100C368A7
:1016900051465B69CDF804C09847D9F80020517CC9
:1016A00054F82110049CCA6880EA0403084694692F
:1016B00051463246A047DDF804C0059809E76E1C84
:1016C000002460E648F2280E5B7CC2F2020E51460E
:1016D0005EF82300C7685B46BC69A0474EE600BFC2
:1016E00064010020012808B501DD002008BD04F0D8
:1016F000B7FA20B1C2680121936A984708BD08BDB6
:10170000012808B501DD002008BD04F0A9FA20B1C8
:10171000C2680221936A984708BD08BD012808B530
:1017200001DD002008BD04F09BFA20B1C26803214E
:10173000936A984708BD08BD012808B501DD00205F
:1017400008BD04F08DFA20B1C2680421936A98475D
:1017500008BD08BD012808B501DD002008BD04F062
:101760007FFA20B1C2680821936A984708BD08BD76
:10177000012808B501DD002008BD04F071FA20B190
:10178000C2680921936A984708BD08BD012808B5B9
:1017900001DD002008BD04F063FA20B1C2680C210D
:1017A000936A984708BD08BD012808B501DD0020EF
:1017B00008BD04F055FA20B1C2680D21936A98471C
:1017C00008BD08BD012808B501DD002008BD04F0F2
:1017D00047FA20B1C2680E21936A984708BD08BD38
:1017E00008B5084B1868407C012801DD002008BDC1
:1017F00004F036FA20B1C2680121936A984708BD07
:1018000008BD00BF6401002008B5084B1868407C83
:10181000012801DD002008BD04F022FA20B1C268D1
:101820000221936A984708BD08BD00BF64010020EB
:1018300008B5084B1868407C012801DD002008BD70
:1018400004F00EFA20B1C2680921936A984708BDD6
:1018500008BD00BF6401002008B548F22803C2F2A9
:101860000203082153F82000C268936A984708BD14
:1018700008B5064B1868407C04F0F2F920B1C26844
:101880000221D36A984708BD08BD00BF640100204B
:1018900048F22803C2F2020353F8200001694868A5
:1018A000704700BF48F22803C2F2020353F8200039
:1018B00001690868704700BF10B5012004F0D0F935
:1018C00080B1C2680321946AA047041E0ADD00208B
:1018D00004F0C6F960B1C36803219A6A9047A04238
:1018E00006DD10BD0020002404F0BAF90028F2D172
:1018F000204610BDC8B130F0010317D030F003030B
:1019000001D10820704730F00703FAD030F00F0300
:10191000F7D030F01F03F4D030F0FF03F1D020F403
:10192000FF7323F0010119B910207047012070479F
:1019300020F47F6222F00F03002BF5D020F4FF414A
:1019400021F07F02002AEFD0000C0304002B0CBF13
:1019500010202020704700BF40F24013C2F2000365
:101960001A68186010467047F0B5054683B00C46FB
:10197000002A37D0224E3368B3F90A10A14231DC75
:10198000B3F90E0084422DDCB3F90810A94229DC1A
:10199000B3F90C00854225DC0E2A25D8DF6B3868A8
:1019A000019201F02BF82146074628460AF0C8FCB0
:1019B000019A0146134802EB0213DAB20368384673
:1019C00098473668104F717C104A57F821601168AB
:1019D000F36808409F6900F0FFFF2946034622464E
:1019E0003046B84703B0F0BD587C074ADE6B52F86A
:1019F00020003368C16822468E692946B047F1E766
:101A000064010020480100202880022040010020BD
:101A1000F0B5054683B00C46002A47D0244E336803
:101A2000B3F90A708F4241DCB3F90E70B9423DDC64
:101A3000B3F90870874239DCB3F90C30984235DCD1
:101A400001920AF07DFC07463068C16B086800F01F
:101A5000D5FF326892F811C0019A5FFA80FE014604
:101A600048F6890300F47F4002FB0EF6C8F68803AF
:101A700002FB00F0A3FB066EA3FB00600D4E01F419
:101A80007F0156F82C6002FB01F28EEA0000A3FBF6
:101A9000021387EAD007F16887EAD3008F6900F064
:101AA0009BFF2946034622463046B84703B0F0BDA7
:101AB0006401002028800220F0B5274D2B68B3F97F
:101AC0000A608E4283B00C46074633DCB3F90E1031
:101AD0008C422FDCB3F90800B8422BDCB3F90C10B0
:101AE0008F4227DC002A27D00F2A31D0DE6B3068E6
:101AF000019200F083FF2A68936B0646186800F095
:101B00007DFF01460198154B00EB00121B68D2B215
:101B10003046984712490A68104000F05DFF2D6872
:101B200010490346687C51F82000C268394695691F
:101B30002246A84703B0F0BD5D7C9B6B09481B683B
:101B400050F82500C16822468D693946A847F1E75B
:101B50005D7CDB6BF2E700BF6401002048010020E0
:101B6000400100202880022010B50C4C2368596BDE
:101B700081420FD0597C5863094B53F821201169D9
:101B80000B68984721680A7C02F00403DAB212B9A4
:101B9000896B086010BDCB6B186010BD640100201C
:101BA0002880022010B50C4C2368196B81420FD09D
:101BB000597C1863094B53F8212011690B68984729
:101BC00021680A7C02F00403DAB212B9C96B08601A
:101BD00010BD8B6B186010BD6401002028800220AE
:101BE00070B4084B1B681A7C80EA0201490705D5CE
:101BF0009C6BD96B26680D6825600E6018741046C2
